:020000040000FA
:04000000ABEF09F069
:08000800236E010E06D0236EE9
:10001000060E03D0236E040E00D00A6E2450205C1E
:1000200002E123501F5C040ED8B0010ED8B4020EBA
:100030000A14D8A4010E1200086A276E286A0096D6
:100040000850D8B40086050E076E270E246E100ED9
:100050000CD8030E246EE80E08D8246A640E05D866
:10006000246A0A0E02D8275008D0236E2850206E2A
:1000700027501F6EEBEC01F01F501F6E074E0096CD
:10008000085003E0075CD8B008D01F50D8A40096F1
:1000900000B603D0300FDCEF00F0120005C01FF0F7
:1000A00006C020F0010E236E246A0F0EEA6E02C015
:1000B000E9FF00002AD8D8A015D0232EFAD7FF0ECA
:1000C0002426D8B0F6D71F26D8A02026D8A0120004
:1000D000640E236E246AEDD70F0EEA6E02C0E9FFAC
:1000E00014D8FEE256D82D6A080E246E53D80DD8C7
:1000F000D8B02D3E2332242EF9D730AA2D6A30BA3B
:10010000239E48D8D88023501200120EE9260950A9
:10011000EF1202C0E9FFEF1430BC0918FF0F120004
:100120002B6E0F0EEA6EE26E0250E96E120FE16E58
:10013000800E0A16080E2C6ED890D8B00A3E12D83F
:100140002B322C2EFAD7000030BA0A300BD800D050
:1001500000D000D0D88006D80650246E055055EC4B
:1001600001F0120030AE0BD0EF50091030AC09187E
:10017000EF6EE7500910D8A00918E76E0BD0EF50CA
:100180000910D8A0091830BC0918EF6E091CE71631
:1001900001D00A8C30501F0B000F206E2F50050F1E
:1001A000D8B0202A0AAC62EF01F00A9C1F6E020E42
:1001B00046EC02F062EF01F001BA90EF00F001B2FC
:1001C00002D001B0FFEF00F0008800A8009800BA4C
:1001D00003D0008A33D827E2009444D8C58642D899
:1001E000C95000B407D000B804D0C588C5B8FED740
:1001F00000B819D8D890236E1DD0008800A80098A8
:1002000000BC05D0FE0B0A6E008CD89013D000BE47
:1002100006D02B6E008E14D8D8B005D02B5014D831
:1002200002E200A807D0C584C5B4FED7009C009E9A
:10023000009A00942D80D8A02D9012000DD801D0E6
:1002400005D80A5000BA0109C96E0AD0948694886C
:10025000C580C5B0FED71200C582C5B2FED7120058
:10026000C7B4FED72368C5501F0B00D0D890D8B4B0
:100270001200232EF8D7D8801200AA6AA96EA66AA7
:10028000A680A850A94AAA2A1200AA6AA86EA66A3D
:10029000A684550EA76EAA0EA76EA682A6B2FED79A
:1002A000A694A94AAA2A1200246A236EFF0E2326C6
:1002B000242200D0D8A01200030E206EE30E02D834
:1002C000F5D7206AF40F1F6E201EFE0ED8A003D0B3
:1002D0001F26D8B0FDD71F260000203EF9D700000A
:1002E0001FB000D01FB000D01200010F2C6E0A0EFC
:1002F000236E246A70D82C2EFDD727501200010FD0
:10030000066E0A0E276E286A296A2A6A04D8062E03
:10031000F8D72750120022502A18800BF46E22AE14
:1003200006D0D880000E1F562056215622562AAEDF
:1003300006D0D880000E2756285629562A56236AFA
:10034000246A256A266A376A386A396A3A6A2A50FC
:1003500029102810271023E0200EF36ED8901F36A6
:100360002036213622363736383639363A36275057
:10037000375C28503858295039582A503A5809E3E0
:100380002750375E2850385A2950395A2A503A5A3D
:10039000D8802336243625362636F32EDFD7F4AE22
:1003A00006D0D880000E235624562556265623C044
:1003B0001FF024C020F025C021F026C022F037C055
:1003C00027F038C028F039C029F03AC02AF01200CE
:1003D000206A246A236E286A276A100EF36E20347E
:1003E000273628362350275C2450285805E323500D
:1003F000275E2450285AD8801F362036F32EEFD798
:100400001F501200200E2B6E376A386A396A3A6A1A
:10041000D8901FA00ED0275037262850D8B0283C9F
:1004200038262950D8B0293C39262A50D8B02A3C41
:100430003A263A32393238323732223221322032B9
:100440001F322B2EE5D71200236A246A04D02032F3
:100450001F3223362436FF0FFAE224C020F0235047
:100460001F6E12001F6E22BE02D81F5012001F1EE8
:10047000201E211E221E1F2AD8B0202AD8B0212AD1
:10048000D8B0222A1200D89020321F32FF0FFBE290
:100490001F501200FC0EDBCFE6FFFD0EDBCFE6FFA8
:1004A000FE0EDBCFE6FFFF0EDBCFE6FFDD52DD52B7
:1004B000DD52DD521200FE0EDBCFE6FFFF0EDBCF7A
:1004C000E6FFDD52DD52120014BE15D11352D8B42E
:1004D00012D13EC02BF03E8C7E0E135C2C6E7E0E35
:1004E000136E1A6A196A186A7F0E176EF30E165C7D
:1004F000040ED8A0050E155C350ED8A0360E145C7F
:1005000003E3B4EC07F004D0132AB4EC07F02C0694
:1005100016C01FF015C020F014C021F013C022F047
:10052000710E1A6E5F0E196E550E186E800E176ED4
:10053000B6EC07F01FC01AF020C019F021C018F067
:1005400022C017F0B8EC08F0C60E1A6EF50E196E40
:100550001F0E186E800E176EB6EC07F016C023F053
:1005600015C024F014C025F013C026F01FC016F0EB
:1005700020C015F021C014F022C013F08A0E1A6EAC
:10058000120E196E790E186E7D0E176EB8EC08F00B
:10059000F60E1A6E460E196E550E186E7E0E176EFA
:1005A000B6EC07F023C01AF024C019F025C018F0EB
:1005B00026C017F050EC08F016C023F015C024F048
:1005C00014C025F013C026F02250136E176E215070
:1005D000146E186E2050156E196E1F50166E1A6E1E
:1005E000B8EC08F016C031F015C032F014C033F08A
:1005F00013C034F023C01AF024C019F025C018F03D
:1006000026C017F0B8EC08F01FC01AF020C019F08F
:1006100021C018F022C017F0B8EC08F031C01AF071
:1006200032C019F033C018F034C017F0176617063F
:10063000B4EC07F01FC01AF020C019F021C018F068
:1006400022C017F0B6EC07F02C5256E016C031F07D
:1006500015C032F014C033F013C034F02CC016F0C3
:10066000000E16BEFF0E156E146E136E68EC09F0C8
:1006700016C01FF015C020F014C021F013C022F0E6
:10068000830E1A6E800E196EDE0E186E720E176EC5
:10069000B8EC08F031C01AF032C019F033C018F0CD
:1006A00034C017F0B6EC07F016C031F015C032F0C8
:1006B00014C033F013C034F01FC016F020C015F082
:1006C00021C014F022C013F01A6A800E196E310E88
:1006D000186E7E0E176EB8EC08F031C01AF032C0FA
:1006E00019F033C018F034C017F0B6EC07F02BBC8B
:1006F00003D03E9C01D03E8A165012003A6A16C0C2
:1007000022F015C021F014C020F013501F6E05E038
:1007100014AE03D03A80800E201A20BE21D0010EE4
:10072000225C000E2158000E20587F0E1F5818E33F
:10073000166A156A146A7F0E136E22C01AF021C061
:1007400019F020C018F01FC017F050EC08F016C0C8
:1007500022F015C021F014C020F013C01FF03A821F
:100760000A0E166E890E156E340E146E7C0E136E04
:1007700022C01AF021C019F020C018F01FC017F0D5
:10078000B8EC08F022C01AF021C019F020C018F00F
:100790001FC017F0B8EC08F07C0E1A6E790E196EB7
:1007A000350E186E810E176EB6EC07F022C01AF0E7
:1007B00021C019F020C018F01FC017F0B8EC08F0E5
:1007C00022C01AF021C019F020C018F01FC017F085
:1007D000B8EC08F03F0E1A6E020E196E330E186E4A
:1007E000830E176EB6EC07F022C01AF021C019F084
:1007F00020C018F01FC017F0B8EC08F022C01AF0A3
:1008000021C019F020C018F01FC017F0B8EC08F094
:10081000330E1A6E8C0E196E1E0E186E830E176E26
:10082000B6EC07F016C026F015C025F014C024F071
:1008300013C023F02250166E2150156E2050146EF6
:100840001F50136E22C01AF021C019F020C018F0FA
:100850001FC017F0B8EC08F01B0E1A6EE40E196EEC
:10086000350E186E820E176EB6EC07F022C01AF025
:1008700021C019F020C018F01FC017F0B8EC08F024
:1008800022C01AF021C019F020C018F01FC017F0C4
:10089000B8EC08F0A40E1A6EDB0E196E670E186E17
:1008A000830E176EB6EC07F022C01AF021C019F0C3
:1008B00020C018F01FC017F0B8EC08F022C01AF0E2
:1008C00021C019F020C018F01FC017F0B8EC08F0D4
:1008D000330E1A6E8C0E196E1E0E186E830E176E66
:1008E000B6EC07F016C02AF015C029F014C028F0A5
:1008F00013C027F022C016F021C015F020C014F05C
:100900001FC013F026C01AF025C019F024C018F03B
:1009100023C017F0B8EC08F02AC01AF029C019F06B
:1009200028C018F027C017F050EC08F016C01AF0D5
:1009300015C019F014C018F013C017F03AA20AD06D
:10094000DB0E166E0F0E156E490E146E7F0E136EB3
:10095000B4EC07F03AA002D0800E141A1650120020
:1009600016C032F015C033F014C034F013C031F0AB
:100970001BD816C01CF015C01DF014C01EF013C00B
:100980001BF032C016F033C015F034C014F031C083
:1009900013F00CD81CC01AF01DC019F01EC018F0BE
:1009A0001BC017F050EF08F0010E01D0000E276EAB
:1009B0003EC029F03E8C2A6A276602D014BE2A8ED9
:1009C000149E880E13603E8A16C01FF015C020F0DA
:1009D00014C021F013C022F0830E1A6EF90E196EA6
:1009E000220E186E7F0E176EB8EC08F03E9C08ECD5
:1009F00009F03E8C16A004D0162A000E15221422EF
:100A0000070E1614286E030E286404D0800E2A1ACE
:100A1000040E285E136A68EC09F01350266E6DE030
:100A200016C023F015C024F014C025F01A6A0F0E6A
:100A3000196EC90E186E7E0E176EB8EC08F01FC046
:100A40001AF020C019F021C018F022C017F0B6EC3F
:100A500007F016C01FF015C020F014C021F013C01D
:100A600022F023C016F024C015F025C014F026C0D3
:100A700013F01A6AA20E196EDA0E186E6E0E176E49
:100A8000B8EC08F01FC01AF020C019F021C018F00F
:100A900022C017F0B6EC07F016C01FF015C020F00A
:100AA00014C021F013C022F023C016F024C015F0AA
:100AB00025C014F026C013F0200E1A6EA20E196E77
:100AC000850E186E5C0E176EB8EC08F01FC01AF099
:100AD00020C019F021C018F022C017F0B6EC07F0C2
:100AE0001350226E176E1450216E186E1550206E22
:100AF000196E16501F6E1A6E0CD02250136E176EA0
:100B00002150146E186E2050156E196E1F50166EFF
:100B10001A6EB8EC08F016C023F015C024F014C00B
:100B200025F013C026F028302818010B271851E0B3
:100B3000CE0E1A6EF50E196E4C0E186E6F0E176EE5
:100B4000B8EC08F01A0E1A6E060E196EB60E186E74
:100B5000750E176EB6EC07F023C01AF024C019F01A
:100B600025C018F026C017F0B8EC08F0A50E1A6ED4
:100B7000AA0E196E2A0E186E7A0E176EB6EC07F0D2
:100B800023C01AF024C019F025C018F026C017F0B1
:100B9000B8EC08F023C01AF024C019F025C018F0F2
:100BA00026C017F0B8EC08F023C01AF024C019F0E2
:100BB00025C018F026C017F017661706B4EC07F02A
:100BC0003E9C1A6A196A186A7F0E176EB6EC07F017
:100BD0005AD0F90E1A6E680E196E360E186E6C0E1B
:100BE000176EB8EC08F0C00E1A6E070E196ED00E14
:100BF000186E720E176EB6EC07F023C01AF024C000
:100C000019F025C018F026C017F0B8EC08F0840ED3
:100C10001A6E880E196E080E186E780E176EB6ECE6
:100C200007F023C01AF024C019F025C018F026C020
:100C300017F0B8EC08F0AB0E1A6EAA0E196E186E0B
:100C40007C0E176EB6EC07F023C01AF024C019F022
:100C500025C018F026C017F0B8EC08F01FC01AF035
:100C600020C019F021C018F022C017F0B8EC08F02D
:100C70003E9C1FC01AF020C019F021C018F022C0FD
:100C800017F0B6EC07F0800E275202E028B22A1ABD
:100C90002ABE141A29BC3E8C1650120014BEB1D0C4
:100CA0001352D8B4AFD013C028F03EC029F03E8C08
:100CB0007F0E136E1A6A196A186A176EB4EC07F081
:100CC00016C01FF015C020F014C021F013C022F090
:100CD000130E1A6ECB0E196E030E186E840E176E5D
:100CE000B6EC07F01FC01AF020C019F021C018F0B0
:100CF00022C017F0B8EC08F0BC0E1A6E5A0E196E2E
:100D0000050E186E860E176EB6EC07F01FC01AF0AF
:100D100020C019F021C018F022C017F0B8EC08F07C
:100D2000830E1A6E300E196E720E186E850E176EC7
:100D3000B6EC07F016C023F015C024F014C025F05F
:100D400013C026F01FC016F020C015F021C014F00B
:100D500022C013F08E0E1A6ED70E196E6B0E186E1F
:100D6000810E176EB8EC08F0B50E1A6E290E196ECA
:100D70004E0E186E840E176EB6EC07F01FC01AF0F8
:100D800020C019F021C018F022C017F0B8EC08F00C
:100D9000800E1A6E300E196E720E186E840E176E5B
:100DA000B6EC07F023C01AF024C019F025C018F0E3
:100DB00026C017F050EC08F01FC01AF020C019F040
:100DC00021C018F022C017F0B8EC08F01A6A196AAE
:100DD000186A7F0E176EB6EC07F028B00AD0F30E33
:100DE0001A6E040E196E350E186E7F0E176EB8EC63
:100DF00008F07F0E28262830136E29BC03D03E9CB5
:100E000001D03E8A1650120018501418406E40BE91
:100E100030D018BE17D01750135CD8A0000CD8A43F
:100E2000010C1850145CD8A0000CD8A4010C195067
:100E3000155CD8A0000CD8A4010C1A50165CD8A0E0
:100E4000000C010C1350175CD8A0000CD8A4010CA6
:100E50001450185CD8A0000CD8A4010C1550195CD3
:100E6000D8A0000CD8A4010C16501A5CD8A0000C15
:100E7000010C14AE010C000C18501418406E40BE4A
:100E800034D018BE19D01750135CD8A0000CD8A4C9
:100E9000010C1850145CD8A0000CD8A4010C1950F7
:100EA000155CD8A0000CD8A4010C1A50165CD8A070
:100EB000000CD8A4010C000C1350175CD8A0000C37
:100EC000D8A4010C1450185CD8A0000CD8A4010CB4
:100ED0001550195CD8A0000CD8A4010C16501A5C4F
:100EE000D8A0000CD8A4010C000C14AE010C000C0E
:100EF00014501818406E40BE34D014BE19D0135090
:100F0000175CD8A0000CD8A4010C1450185CD8A011
:100F1000000CD8A4010C1550195CD8A0000CD8A462
:100F2000010C16501A5CD8A0000CD8A4010C000CBF
:100F30001750135CD8A0000CD8A4010C1850145CF6
:100F4000D8A0000CD8A4010C1950155CD8A0000C36
:100F5000D8A4010C1A50165CD8A0000CD8A4010C1F
:100F6000000C18AE010C000C800E181A1750135C00
:100F70003D6E19E23D6C13C03FF017C013F03FC047
:100F800017F014C03FF018C014F03FC018F015C09F
:100F90003FF019C015F03FC019F016C03FF01AC05D
:100FA00016F03FC01AF01A0E3D6078D0175276E066
:100FB0003C6A14503F6E1818416E148E188E080E3D
:100FC0003D5E08E31AC03CF019C01AF018C019F0D1
:100FD000186AF5D73D2607E0D890183219321A3230
:100FE0003C323D2EF9D741AE35D01A50165E19501D
:100FF000155A1850145A07E2D880000E1656155686
:101000001456800E3F1A3C6C04E01606000E155A6A
:10101000145A040E3D6E14660DD015C014F016C09F
:1010200015F03CC016F03C6A080E135E2DE33D2E11
:10103000F2D72AD014BE08D0D8903C3616361536D2
:101040001436132EF7D720D03EAC26D03CAE24D099
:101050003C6A11D01A501626195015221850142225
:1010600006E31432153216323C32134A0FD03EAC2E
:1010700013D03CAE11D0163E0FD0153E0DD0143E0D
:101080000BD0D8801690EDD7136A02D03E82136839
:10109000166A156A800E146E3FAE149E165012002A
:1010A0001450396E1818416E175053E0135254E023
:1010B000135E7F0E03E2132603E24DD013264EE2A9
:1010C00016C037F015C038F0398E188E180E3F6EE6
:1010D000166A156A146A0BD01A50375C19503858C2
:1010E00011E3386E396A1A50375E0BD004E218509B
:1010F000395CF2E007E31A50375E1950385A18503D
:10110000395AD880163615361436373638363936C9
:101110003F2EECD714BE07D013521DE04132130608
:101120003F2A4136E3D73EAC1FD007E21A50375E64
:101130001950385A1850395A17E3163E15D0153E33
:1011400013D0143E11D0143215321632133E0CD087
:1011500005D03E8604D03E84136A02D03E821368D6
:10116000166A156A800E146E41AE149E1650120057
:101170001450396E1818416E1350D8A417503CE023
:1011800013267E0E03E3135E03E338D0135E33E3CE
:1011900016C037F015C038F0398E188E166A156AE9
:1011A000146A180E3F6E39323832373206E31A505D
:1011B00016261950152218501422143215321632E0
:1011C0003F2EF1D714BE07D01636153614361352FB
:1011D00012E0130639343EAC17D016E3163E14D095
:1011E000153E12D0143E10D0D8801432153216326B
:1011F000133E0AD003D03E84136A02D03E821368A5
:10120000166A156A800E146E41AE149E16501200B6
:1012100014C041F07F0E135C3F6E3FE3148E136ADF
:10122000376A17083F6E0BE2080E3F2638E314C0FA
:1012300013F015C014F016C015F0166A0CD0080E85
:101240003F5E08E316C037F015C016F014C015F065
:10125000146AF5D73F263F5208E0D8901332143273
:101260001532163237323F2EF8D713BE18D03EACA7
:101270000BD037AE09D0163E07D0153E05D0143E30
:1012800003D0142A13BE0BD041AE10D0D880000E6C
:10129000165615561456135609D0000E02D03E822B
:1012A000FF0E136E146E156E166E139E16501200FE
:1012B000136E146A156A166A13C03CF016C013F058
:1012C0003CC016F015C03CF014C015F03CC014F042
:1012D000960E3F6E416A13AE07D0D880000E1656A8
:1012E000155614561356418E135218E03EAC0DD0CD
:1012F00016AE0BD0153E09D0143E07D0133E05D0D4
:10130000D8801332143215323F2A080E3F2615C0FA
:1013100016F014C015F013C014F015D0146613D0D5
:10132000080E3F5E155005E1080E3F5E165011E0B5
:10133000166A146E16C015F0166A05D0D8901636C7
:10134000153614363F0614AEF9D73FC013F041AE40
:10135000149E16501200F86A400E3E6E006AAB6A88
:10136000280EC66E040EC86E800EC76E070EB46ED1
:101370000F0EC16E2EEEC0F0840ED56EF29EF29A64
:101380000EEEFFF0ED6AE950EA10FCE1EF6A2F0E75
:10139000926E070E936E870E946E956A966A3F0E54
:1013A000976E200E986E866B856B946B010E966F10
:1013B000900E956F976B0A0E8C6F8E6B8F6B8B9563
:1013C000906B06013B6B00018B91B66BB56BB86BF4
:1013D000B76B8B9B010EB96F010EBA6FCC6BCB6BE9
:1013E0000B0E8D6F8B998B97CF6BD06BD26BD86BAD
:1013F000D76BD66BD56B0101236B010E0801206FF3
:101400000101296B286B2B6B2A6B0501256B246B63
:10141000236B226B296B286B276B266B2D6B2C6B38
:101420002B6B2A6B316B306B2F6B2E6B336B326BEC
:10143000376B366B356B346B08011F6B1E6B1D6B86
:101440001C6B790E0501386F3A6B396B01012F6BFC
:101450002E6B2D6B2C6B0801276B010E0001846F26
:101460000801306BA30E01014B6FA20E4C6FAB0E47
:101470004D6FAA0E4E6F0001876B800E875DD8B04E
:101480004EEF0AF002EE1EF0D8908735E926000EE6
:10149000EA22EE6AEF6A872BD8A4EFD7876B800E1B
:1014A000875DD8B060EF0AF003EE1EF0D890873564
:1014B000E926000EEA22EE6AEF6A872BD8A4EFD75E
:1014C000876B800E875DD8B072EF0AF004EE1EF0D5
:1014D000D8908735E926000EEA22EE6AEF6A872B5C
:1014E000D8A4EFD7876B150E875DD8B084EF0AF0CC
:1014F00001EE78F0D8908735E926000EEA22EE6AF0
:10150000EF6A872BD8A4EFD7876B290E875DD8B0F9
:1015100096EF0AF001EEA2F0D8908735E926000E8A
:10152000EA22EE6AEF6A872BD8A4EFD7876B150EF5
:10153000875DD8B0A8EF0AF001EEF4F0D8908735B7
:10154000E926000EEA22EE6AEF6A872BD8A4EFD7CD
:1015500072EFD3F00801796B00018653D8A48AEFAB
:101560000BF001013895020E245D0001D8A4BEEFF6
:101570000AF0010138850001CDEF0AF0030E0101E8
:10158000245D0001D8A4CAEF0AF0010138850001EA
:10159000CCEF0AF0010138950001D896010138A579
:1015A000D8860001D8B654EF0BF0850E026E800E7F
:1015B000096E306ABC0E2F6E066A056A200E016E37
:1015C000240E90EC00F0500E90EC00F0530E90ECD6
:1015D00000F0520E90EC00F0460E90EC00F0310E50
:1015E00090EC00F0300E90EC00F0330E90EC00F038
:1015F0002C0E90EC00F0340E90EC00F02C0E90ECE1
:1016000000F0310E90EC00F02C0E90EC00F0310E5A
:1016100090EC00F02C0E90EC00F0310E90EC00F00D
:101620002A0E90EC00F0320E90EC00F0300E90ECB0
:1016300000F00D0E90EC00F00A0E90EC00F0800E21
:10164000026E040E096E400E306EBC0E2F6E066ADE
:10165000320E056E4EEC00F0D8A088EF0BF0520869
:10166000D8A4F8D74EEC00F0D8A088EF0BF04D08C6
:10167000D8A4F0D74EEC00F0D8A088EF0BF04308C8
:10168000D8A4E8D70B6AD8804EEC00F0D8A088EF39
:101690000BF008EE32F00B5023C0EBFF0B2A0B507F
:1016A0004008F1E188EF0BF0800E026E040E096E27
:1016B000400E306EBC0E2F6E070E066ED00E056EFD
:1016C0004EEC00F0D8A02EEFA4F05208D8A4F8D722
:1016D0004EEC00F0D8A02EEFA4F04D08D8A4F0D71F
:1016E0004EEC00F0D8A02EEFA4F04308D8A4E8D721
:1016F0000B6AD8804EEC00F0D8A02EEFA4F008EED4
:1017000032F00B5023C0EBFF0B2A0B504008F1E1E5
:10171000A3EF0CF0470E0801326F500E336F520EDC
:10172000346F4D0E356F430E366F2C0E376F300E03
:10173000386F310E396F310E3A6F340E3B6F330E06
:101740003C6F370E3D6F2E0E3E6F300E3F6F300EEA
:10175000406F300E416F2C0E426F410E436F2C0EC6
:10176000446F340E456F320E466F340E476F340EA1
:10177000486F2E0E496F300E4A6F300E4B6F300E91
:101780004C6F300E4D6F2C0E4E6F4E0E4F6F2C0E59
:10179000506F300E516F380E526F330E536F300E44
:1017A000546F300E556F2E0E566F300E576F300E31
:1017B000586F300E596F300E5A6F2C0E5B6F570EEC
:1017C0005C6F2C0E5D6F776B06EE3CF0D8900601D7
:1017D0003B35E926000EEA22EECF1FF0EFCF20F0D6
:1017E000030E75EC01F00801776F77C85EF8776B30
:1017F00006EE3CF0D89006013B35E926000EEA22C1
:10180000EECF1FF0EFCF20F0020E75EC01F00801D3
:10181000776F77C85FF82E0E606F776B06EE3CF03F
:10182000D89006013B35E926000EEA22EECF1FF0E4
:10183000EFCF20F0010E75EC01F00801776F77C84B
:1018400061F8776B06EE3CF0D89006013B35E9264F
:10185000000EEA22EECF1FF0EFCF20F0000E75EC65
:1018600001F00801776F77C862F82C0E636F776B11
:1018700007EE2CF0D89006013B35E926000EEA224F
:10188000EECF1FF0EFCF20F0020E75EC01F0080153
:10189000776F77C864F8776B07EE2CF0D890060165
:1018A0003B35E926000EEA22EECF1FF0EFCF20F005
:1018B000010E75EC01F00801776F77C865F8776B5A
:1018C00007EE2CF0D89006013B35E926000EEA22FF
:1018D000EECF1FF0EFCF20F0000E75EC01F0080105
:1018E000776F77C866F82E0E676F380E686F350E03
:1018F000696F2C0E6A6F320E6B6F300E6C6F300E8C
:101900006D6F380E6E6F300E6F6F380E706F2C0E5D
:10191000716F2C0E726F2A0E736F310E746F360E4C
:10192000756F360E766F06013B2B780E3B5D00011E
:10193000D8A09DEF0CF006013B6B0001010E246E58
:10194000900E55EC01F00801316B0001400E0801CA
:10195000315D0001D8B0E6EF0CF008EE32F008017E
:101960003151EBCF0BF000EE42F031510BC0EBFFE9
:1019700008EE32F03151EB500F6EA40EF66E190ED8
:10198000F76E2368232A235009080001D8A0DCEF52
:101990000CF00900F55009000F5CF4E123C00BF0D6
:1019A000DCEF0CF0300C310C320C330C340C350CF9
:1019B000360C370C380C390C00EE42F0080131516E
:1019C0000BC0EBFF312B0001D8A4BFD712000801D8
:1019D0007A6B00010A0E08017A5D0001D8B041EF70
:1019E0000DF00101235108017A5D0001D8B01CEF10
:1019F0000DF008017A510101235D316E326AD8A0E1
:101A00003206310404EE1EF0D890E836E926000EC6
:101A1000EA22EECF0BF0EFCF0CF008EE7DF0D8907D
:101A200008017A35E926000EEA220BC0EEFF0CC051
:101A3000EFFF00013BEF0DF07F0E01012325326A1D
:101A4000316E323608017A51315C04EE1EF0D890C6
:101A5000E836E926000EEA22EECF0BF0EFCF0CF0CD
:101A600008EE7DF0D8907A35E926000EEA220BC008
:101A7000EEFF0CC0EFFF000108017A2B0001D8A493
:101A8000A8D708017A6B00010A0E08017A5D0001EF
:101A9000D8B0E2EF0DF004EE1EF0D890010123352E
:101AA000E926000EEA22EECF1FF0EFCF20F0020E63
:101AB00075EC01F00B6E030E0B5C0001D8A494EFE3
:101AC0000DF008EE7DF0D89008017A35E926000E79
:101AD000EA22EECF1FF0EFCF20F0020E75EC01F0FE
:101AE0000B6E0B520001D8A493EF0DF008EE7DF0C1
:101AF000D89008017A35E926000EEA22EECF0FF0E1
:101B0000EFCF10F0680E0F240B6E010E10200C6E3C
:101B100008EE7DF0D8907A35E926000EEA220BC057
:101B2000EEFF0CC0EFFF000104EE1EF0D8900101A3
:101B30002335E926000EEA22EECF1FF0EFCF20F08A
:101B4000020E75EC01F00B6E0B520001D8A4DDEF14
:101B50000DF008EE7DF0D89008017A35E926000EE8
:101B6000EA22EECF1FF0EFCF20F0020E75EC01F06D
:101B70000B6E030E0B5C0001D8A4DCEF0DF008EE39
:101B80007DF0D89008017A35E926000EEA22EECFE2
:101B90000FF0EFCF10F00F5068080B6E010E1054CD
:101BA0000C6E08EE7DF0D8907A35E926000EEA2218
:101BB0000BC0EEFF0CC0EFFF000108017A2B000103
:101BC000D8A461D708017C6B7B6B7A6B00010A0E8D
:101BD00008017A5D0001D8B002EF0EF008EE7DF04A
:101BE000D89008017A35E926000EEA22EECF0BF0F4
:101BF000EFCF0CF00B507B270C507C237A2B00018D
:101C0000D8A4E4D77CC820F07BC81FF0246A0A0E51
:101C1000236EEBEC01F008017B6F20C07CF804EE32
:101C20001EF0D89001012335E926000EEA22EECFFE
:101C30000BF0EFCF0CF00B5008017B5D0C507C5982
:101C40000001D8B03AEF0EF004EE1EF0D89001017A
:101C50002335E926000EEA22EECF0BF0EFCF0CF091
:101C600008017B510B5C916F7C510C58926F000105
:101C70004DEF0EF004EE1EF0D89001012335E92659
:101C8000000EEA22EECF0BF0EFCF0CF00B50080164
:101C90007B5D916F0C507C59926F0001080192534B
:101CA0000001D8A46AEF0EF0030E0801915D000157
:101CB000D8B06AEF0EF004EE1EF0D8900101233583
:101CC000E926000EEA22EECF7BF8EFCF7CF8000188
:101CD0006FEF0EF0010E08017C6F680E7B6F000144
:101CE0007BC8DEFF7CC8DEFF120018EE95F05BECCF
:101CF00002F018EE93F05BEC02F008019351955D51
:101D0000945196590001D8B096EF0EF00801955104
:101D1000935D976F96519459986F97516808976F94
:101D2000010E9855986F00019DEF0EF00801935138
:101D3000955D976F94519659986F000108019851DD
:101D4000010A680ED8B497190001D8A4ADEF0EF0BF
:101D5000010E0801986F670E976F000197C8DEFFAC
:101D600098C8DEFF1200FF0EDB50DD5201013887FC
:101D7000E8A0389718EE9BF05BEC02F018EE99F0B3
:101D80005BEC02F0080199519B5D9A519C5900014E
:101D9000D8B0DBEF0EF008019B51995D9D6F9C510F
:101DA0009A599E6F9D5168089F6F010E9E55A06FB6
:101DB0000001E8EF0EF0080199519B5D9D6F9A516B
:101DC0009C599E6F9D5168089F6F010E9E55A06F94
:101DD000000108019F519D5DA0519E590001D8B09E
:101DE000F8EF0EF09EC8A2F89DC8A1F8FCEF0EF027
:101DF000A0C8A2F89FC8A1F8D896010138A7D88634
:101E00000001D8B62DEF0FF0080199519B5D9A5152
:101E10009C590001D8B01EEF0FF008019F519D5D45
:101E2000A0519E590001D8B01AEF0FF0520E886FE2
:101E30001CEF0FF04C0E886F2DEF0FF008019F5133
:101E40009D5DA0519E590001D8B02BEF0FF04C0EB4
:101E5000886F2DEF0FF0520E886F0801A251010A12
:101E6000680ED8B4A1190001D8A43CEF0FF0010E00
:101E70000801A26F670EA16F0001A1C8DEFFA2C812
:101E8000DEFF120018EEAFF05BEC02F004EE1EF085
:101E9000D89001012335E926000EEA22EECF0BF09F
:101EA000EFCF0CF00BC0DEFF0CC0DEFFAFC8DEFFD3
:101EB000B0C8DEFFDE6A000156DF18EEA3F05BEC6F
:101EC00002F0A3C813F0A4C814F05AEC09F0DB0E1A
:101ED0001A6E0F0E196E490E186E800E176EB8EC42
:101EE00008F016C0AEF815C0ADF814C0ACF813C0B9
:101EF000ABF81A6A196A340E186E860E176EAEC8E1
:101F000016F0ADC815F0ACC814F0ABC813F050EC27
:101F100008F016C0AEF815C0ADF814C0ACF813C088
:101F2000ABF8AEC816F0ADC815F0ACC814F0ABC82D
:101F300013F0D4EC04F016C0AAF815C0A9F814C028
:101F4000A8F813C0A7F80801A89F03EE1EF0D890C8
:101F500001012335E926000EEA22EECF0BF0EFCF88
:101F60000CF00BC013F00CC014F05AEC09F0AAC826
:101F70001AF0A9C819F0A8C818F0A7C817F0B8EC4B
:101F800008F008EC09F015C0A6F80801A56FA5C86F
:101F9000DEFFA6C8DEFF00011200D8968BADD88602
:101FA000D8B6D8EF0FF00801BA6BB96B00018B9D62
:101FB00004EE1EF0D89001012335E926000EEA2236
:101FC000EECFB1F8EFCFB2F8B2C820F0B1C81FF031
:101FD000020E75EC01F00801B46BB36F01012353DD
:101FE0000001D8B405EF10F0010123050B6E04EEDB
:101FF0001EF0D8900B34E926000EEA22EECFB5F899
:10200000EFCFB6F8000109EF10F01CC5B5F81DC5FB
:10201000B6F8B6C820F0B5C81FF0020E75EC01F096
:102020000801B86BB76FB751B35D0B6EB851B459B7
:102030000C6E0B50030A0C100001D8A427EF10F00F
:102040000801B5516808B56F010EB655B66F0001AD
:102050000801B351B75D0B6EB451B8590C6E0B50FB
:10206000030A0C100001D8A43BEF10F0680E080121
:10207000B127010EB22300010801B151B55DB25183
:10208000B6590001D8B060EF10F00801B92B040E6A
:10209000BA5D0001D8A05DEF10F08B8104EE1EF058
:1020A000D89001012335E926000EEA22EECF89F00F
:1020B000EFCF8AF000015FEF10F00801BA6B00016A
:1020C0000801B551B15DB651B2590001D8B084EFE5
:1020D00010F00801BA2B040EB95D0001D8A081EF01
:1020E00010F08B8104EE1EF0D89001012335E92613
:1020F000000EEA22EECF89F0EFCF8AF0000183EFE5
:1021000010F00801B96B0001120018EED6F05BEC7C
:1021100002F018EEBCF04AEC02F018EED4F05BECE2
:1021200002F0BCC813F0BDC814F0BEC815F0BFC89B
:1021300016F05CEC09F016C0C3F815C0C2F814C064
:10214000C1F813C0C0F8D6C8DEFFD7C8DEFFD4C8B8
:10215000DEFFD5C8DEFFDE6A06DE18EED8F05BECE7
:1021600002F00801D9530001D8A4BEEF10F00B0E05
:102170000801D85D0001D8A0AFEF11F00101405176
:102180000801BC5D010141510801BD5901014251E5
:102190000801BE59010143510801BF59BF51010156
:1021A0004319D8B0800A0001D8B8A5EF11F0D9C8FA
:1021B00014F0D8C813F05AEC09F016C0C7F815C0CF
:1021C000C6F814C0C5F813C0C4F8DB0E166E0F0EA7
:1021D000156E490E146E800E136EC7C81AF0C6C86D
:1021E00019F0C5C818F0C4C817F0B8EC08F016C04C
:1021F00034F015C033F014C032F013C031F01A6A55
:10220000196A340E186E860E176E34C016F033C07D
:1022100015F032C014F031C013F050EC08F016C0C5
:10222000C7F815C0C6F814C0C5F813C0C4F8080133
:10223000D9530001D8A42EEF11F0050E0801D85D86
:102240000001D8B02EEF11F0C3C8CFF8C2C8CEF845
:10225000C1C8CDF8C0C8CCF874EF11F00801D9534B
:102260000001D8A43BEF11F0AB0E0801D85D0001CE
:10227000D8A045EF11F0C3C8CFF8C2C8CEF8C1C886
:10228000CDF8C0C8CCF873EF11F0C7C816F0C6C8B7
:1022900015F0C5C814F0C4C813F0D6EC04F016C08D
:1022A000D3F815C0D2F814C0D1F813C0D0F8080183
:1022B000D19FC3C816F0C2C815F0C1C814F0C0C879
:1022C00013F0D3C81AF0D2C819F0D1C818F0D0C88A
:1022D00017F050EC08F016C0CFF815C0CEF814C0B7
:1022E000CDF813C0CCF80001CFC816F0CEC815F059
:1022F000CDC814F0CCC813F008EC09F013C0CBF82B
:1023000014C0CAF815C0C9F80801C86FD896CBBF69
:10231000D8860001D8B6A2EF11F03D0E0801C85DC5
:10232000860EC959010ECA59000ECB590001D8A01A
:10233000A2EF11F00801CB6B010ECA6F860EC96FB8
:102340003C0EC86F0001ADEF11F0BFC8CBF8BEC89E
:10235000CAF8BDC8C9F8BCC8C8F8B7EF11F0BFC803
:10236000CBF8BEC8CAF8BDC8C9F8BCC8C8F8C8C848
:10237000DEFFC9C8DEFFCAC8DEFFCBC8DEFF120021
:10238000A4C0DDF8A3C0DCF8A2C0DBF8A1C0DAF875
:10239000A8C0E1F8A7C0E0F8A6C0DFF8A5C0DEF845
:1023A000ACC0E5F8ABC0E4F8AAC0E3F8A9C0E2F815
:1023B000B0C0E9F8AFC0E8F8AEC0E7F8ADC0E6F8E5
:1023C0001A6A7C0E196E120E186E920E176E99C054
:1023D00013F09AC014F09BC015F09CC016F05CEC92
:1023E00009F050EC08F016C0EDF815C0ECF814C078
:1023F000EBF813C0EAF8D05158EC09F0EDC81AF028
:10240000ECC819F0EBC818F0EAC817F0B6EC07F002
:1024100016C0EDF815C0ECF814C0EBF813C0EAF8DC
:10242000530E01015E5D0001D8A41AEF12F0800E78
:102430000801EB1B00011A6A7C0E196E120E186E51
:10244000920E176E9DC013F09EC014F09FC015F041
:10245000A0C016F05CEC09F050EC08F016C0F1F8E2
:1024600015C0F0F814C0EFF813C0EEF8D15158ECD5
:1024700009F0F1C81AF0F0C819F0EFC818F0EEC86A
:1024800017F0B6EC07F016C0F1F815C0F0F814C05C
:10249000EFF813C0EEF8570E0101685D0001D8A4F3
:1024A00055EF12F0800E0801EF1B0001D05158ECDF
:1024B00009F0DB0E1A6E0F0E196E490E186E800EA3
:1024C000176EB8EC08F016C034F015C033F014C025
:1024D00032F013C031F01A6A196A340E186E860E83
:1024E000176E34C016F033C015F032C014F031C08E
:1024F00013F050EC08F016C03FF915C03EF914C0B7
:102500003DF913C03CF93FC916F03EC915F03DC96D
:1025100014F03CC913F0D4EC04F016C03FF915C018
:102520003EF914C03DF913C03CF9E9C816F0E8C8FB
:1025300015F0E7C814F0E6C813F0E1C81AF0E0C8D7
:1025400019F0DFC818F0DEC817F0B4EC07F016C0B9
:1025500034F015C033F014C032F013C031F034C081
:1025600016F033C015F032C014F031C013F03FC97B
:102570001AF03EC919F03DC918F03CC917F0B8EC83
:1025800008F016C00FF915C00EF914C00DF913C0EC
:102590000CF9E5C816F0E4C815F0E3C814F0E2C879
:1025A00013F0DDC81AF0DCC819F0DBC818F0DAC87F
:1025B00017F0B4EC07F016C013F915C012F914C0E7
:1025C00011F913C010F9F1C816F0F0C815F0EFC8F2
:1025D00014F0EEC813F0E1C81AF0E0C819F0DFC833
:1025E00018F0DEC817F0B4EC07F016C034F015C0D0
:1025F00033F014C032F013C031F034C016F033C0E1
:1026000015F032C014F031C013F03FC91AF03EC9C2
:1026100019F03DC918F03CC917F0B8EC08F016C025
:102620001BF915C01AF914C019F913C018F9EDC82F
:1026300016F0ECC815F0EBC814F0EAC813F0DDC8CA
:102640001AF0DCC819F0DBC818F0DAC817F0B4ECDF
:1026500007F016C017F915C016F914C015F913C004
:1026600014F9DDC816F0DCC815F0DBC814F0DAC8C0
:1026700013F0EDC81AF0ECC819F0EBC818F0EAC86E
:1026800017F0B4EC07F016C027F915C026F914C0EE
:1026900025F913C024F9E1C816F0E0C815F0DFC829
:1026A00014F0DEC813F0F1C81AF0F0C819F0EFC842
:1026B00018F0EEC817F0B4EC07F016C034F015C0EF
:1026C00033F014C032F013C031F034C016F033C010
:1026D00015F032C014F031C013F03FC91AF03EC9F2
:1026E00019F03DC918F03CC917F0B8EC08F016C055
:1026F0002BF915C02AF914C029F913C028F917C9F4
:10270000F7F816C9F6F815C9F5F80801F59F14C9C8
:10271000F4F82BC9FBF82AC9FAF829C9F9F8F99F86
:1027200028C9F8F8FBC816F0FAC815F0F9C814F073
:10273000F8C813F0F7C81AF0F6C819F0F5C818F081
:10274000F4C817F004EC07F001080001D8B4B3EFA7
:1027500013F0F7C843F9F6C842F9F5C841F9F4C8CF
:1027600040F9BBEF13F0FBC843F9FAC842F9F9C8C6
:1027700041F9F8C840F90A0E166ED70E156E230EF1
:10278000146E780E136E43C91AF042C919F041C98C
:1027900018F040C917F004EC07F00108D8B4DCEFDA
:1027A00013F009013B6B010E3A6F860E396F3C0E38
:1027B000386F00011FEF17F01BC916F01AC915F08A
:1027C00019C914F018C913F00FC91AF00EC919F07D
:1027D0000DC918F00CC917F0B8EC08F016C0F7F8DE
:1027E00015C0F6F814C0F5F813C0F4F817C916F0C0
:1027F00016C915F015C914F014C913F013C91AF04D
:1028000012C919F011C918F010C917F0B8EC08F086
:1028100016C0FBF815C0FAF814C0F9F813C0F8F8A0
:10282000F7C816F0F6C815F0F5C814F0F4C813F0A0
:10283000FBC81AF0FAC819F0F9C818F0F8C817F070
:10284000B6EC07F016C003F915C002F914C001F97F
:1028500013C000F90FC916F00EC915F00DC914F018
:102860000CC913F00FC91AF00EC919F00DC918F0F0
:102870000CC917F0B8EC08F016C0F7F815C0F6F858
:1028800014C0F5F813C0F4F813C916F012C915F006
:1028900011C914F010C913F013C91AF012C919F0B4
:1028A00011C918F010C917F0B8EC08F016C0FBF801
:1028B00015C0FAF814C0F9F813C0F8F8F7C816F004
:1028C000F6C815F0F5C814F0F4C813F0FBC81AF0F8
:1028D000FAC819F0F9C818F0F8C817F0B6EC07F004
:1028E00016C0FFF815C0FEF814C0FDF813C0FCF8C0
:1028F00003C916F002C915F001C914F000C913F09C
:10290000FFC81AF0FEC819F0FDC818F0FCC817F08F
:1029100050EC08F016C007F915C006F914C005F907
:1029200013C004F90FC916F00EC915F00DC914F043
:102930000CC913F027C91AF026C919F025C918F0D7
:1029400024C917F0B8EC08F016C0F7F815C0F6F86F
:1029500014C0F5F813C0F4F813C916F012C915F035
:1029600011C914F010C913F02BC91AF02AC919F0B3
:1029700029C918F028C917F0B8EC08F016C0FBF800
:1029800015C0FAF814C0F9F813C0F8F8F7C816F033
:10299000F6C815F0F5C814F0F4C813F0FBC81AF027
:1029A000FAC819F0F9C818F0F8C817F0B4EC07F035
:1029B00016C00BF915C00AF914C009F913C008F9BB
:1029C0000BC916F00AC915F009C914F008C913F0AB
:1029D000FFC81AF0FEC819F0FDC818F0FCC817F0BF
:1029E00050EC08F016C00BF915C00AF914C009F92B
:1029F00013C008F9010137530001D8B427EF15F0CF
:102A0000020E0101375D0001D8A425EF15F0166A0A
:102A1000156A146A136A0BC91AF00AC919F009C9B0
:102A200018F008C917F004EC07F00108D8B41FEF3C
:102A300015F04E0E0101366F000122EF15F0500E19
:102A40000101366F000125EF15F00101376B000120
:102A500001013891166A156A146A136A0BC91AF0D3
:102A60000AC919F009C918F008C917F03CEC07F0B9
:102A700001080001D8B449EF15F04E0E0101365D92
:102A80000001D8A446EF15F001013881000153EF91
:102A900015F0500E0101365D0001D8A452EF15F07B
:102AA00001013881000107C916F006C915F005C9F2
:102AB00014F004C913F01A6A196A186A176A04EC48
:102AC00007F03B6E07C916F006C915F005C914F0EA
:102AD00004C913F01A6A196A186A7F0E176E3CEC63
:102AE00007F0010A3B14D8B4AFEF15F0FFC816F099
:102AF000FEC815F0FDC814F0FCC813F04EEC06F04B
:102B000016C0F7F815C0F6F814C0F5F813C0F4F8BD
:102B10000BC9FBF80AC9FAF809C9F9F80801F99FC5
:102B200008C9F8F8F7C816F0F6C815F0F5C814F09B
:102B3000F4C813F0FBC81AF0FAC819F0F9C818F075
:102B4000F8C817F0B8EC08F016C037F915C036F918
:102B500014C035F913C034F90001D5EF16F01BC9C4
:102B600016F01AC915F019C914F018C913F01BC9C9
:102B70001AF01AC919F019C918F018C917F0B8ECE9
:102B800008F016C0F7F815C0F6F814C0F5F813C031
:102B9000F4F817C916F016C915F015C914F014C9C0
:102BA00013F017C91AF016C919F015C918F014C98D
:102BB00017F0B8EC08F016C0FBF815C0FAF814C00E
:102BC000F9F813C0F8F8F7C816F0F6C815F0F5C80C
:102BD00014F0F4C813F0FBC81AF0FAC819F0F9C8D9
:102BE00018F0F8C817F0B6EC07F016C02FF915C0AA
:102BF0002EF914C02DF913C02CF9F1C816F0F0C845
:102C000015F0EFC814F0EEC813F0E9C81AF0E8C8E0
:102C100019F0E7C818F0E6C817F0B4EC07F016C0D2
:102C200034F015C033F014C032F013C031F034C0AA
:102C300016F033C015F032C014F031C013F03FC9A4
:102C40001AF03EC919F03DC918F03CC917F0B8ECAC
:102C500008F016C023F915C022F914C021F913C0D9
:102C600020F9EDC816F0ECC815F0EBC814F0EAC86E
:102C700013F0E5C81AF0E4C819F0E3C818F0E2C888
:102C800017F0B4EC07F016C01FF915C01EF914C0F8
:102C90001DF913C01CF923C916F022C915F021C96A
:102CA00014F020C913F023C91AF022C919F021C960
:102CB00018F020C917F0B8EC08F016C0F7F815C0E6
:102CC000F6F814C0F5F813C0F4F81FC916F01EC9C1
:102CD00015F01DC914F01CC913F01FC91AF01EC944
:102CE00019F01DC918F01CC917F0B8EC08F016C08F
:102CF000FBF815C0FAF814C0F9F813C0F8F8F7C8D3
:102D000016F0F6C815F0F5C814F0F4C813F0FBC8B7
:102D10001AF0FAC819F0F9C818F0F8C817F0B6ECAC
:102D200007F016C033F915C032F914C031F913C0D9
:102D300030F92FC916F02EC915F02DC914F02CC981
:102D400013F033C91AF032C919F031C918F030C97B
:102D500017F004EC07F00108D8B4C3EF16F02FC940
:102D600016F02EC915F02DC914F02CC913F04EEC35
:102D700006F016C037F915C036F914C035F913C07E
:102D800034F9D5EF16F033C916F032C915F031C950
:102D900014F030C913F04EEC06F016C037F915C028
:102DA00036F914C035F913C034F9600E166E5F0E93
:102DB000156E290E146E960E136E37C91AF036C9A9
:102DC00019F035C918F034C917F0B8EC08F016C07E
:102DD00037F915C036F914C035F913C034F9166A3D
:102DE0001E0E156E430E146E8F0E136E37C91AF039
:102DF00036C919F035C918F034C917F004EC07F0DA
:102E00000108D8B40CEF17F00901376B1E0E366FAE
:102E1000430E356F8F0E346F000137C916F036C977
:102E200015F035C914F034C913F008EC09F013C0DB
:102E30003BF914C03AF915C039F90901386F00019E
:102E400038C9DEFF39C9DEFF3AC9DEFF3BC9DEFF04
:102E5000120019EE4AF04AEC02F019EE44F05BEC75
:102E600002F044C913F045C914F05AEC09F04A0EB7
:102E70001A6E9F0E196E240E186E810E176EB8EC26
:102E800008F016C049F915C048F914C047F913C035
:102E900046F949C916F048C915F047C914F046C9A2
:102EA00013F008EC09F015C045F90901446F4DC94C
:102EB00022F04CC921F04BC920F04AC91FF02A6A00
:102EC000296A030E286EE80E276E02EC02F022C07B
:102ED0004DF921C04CF920C04BF91FC04AF9166AC0
:102EE000156A146A7F0E136E49C91AF048C919F0A1
:102EF00047C918F046C917F004EC07F001080001B3
:102F0000D8B4A4EF17F04DC916F04CC915F04BC951
:102F100014F04AC913F05CEC09F049C91AF048C929
:102F200019F047C918F046C917F050EC08F008EC42
:102F300009F013C053F914C052F915C051F9090131
:102F4000506F0001ABEF17F00901536B526B170E76
:102F5000516F340E506F0001D896090153BFD886C7
:102F60000001D8B6C8EF17F0090153530AE15251D6
:102F700008E1350E505D170E51590001D8A0C8EF79
:102F800017F00901536B526B170E516F340E506FCF
:102F9000000151C94FF950C94EF94EC9DEFF4FC962
:102FA000DEFF120019EE54F04AEC02F019EE58F070
:102FB0004AEC02F019EE5CF04AEC02F019EE60F017
:102FC0004AEC02F001013899166A156A146A136A0C
:102FD00057C91AF056C919F055C918F054C917F055
:102FE00004EC07F001080001D8B40EEF18F0166ADF
:102FF000156A146A136A5FC91AF05EC919F05DC9CF
:1030000018F05CC917F004EC07F00108D8B40BEF16
:1030100018F00101388900011FEF18F009015C5315
:103020000001D8B41EEF18F0D89609015DAFD8861C
:103030000001D8B61EEF18F0010138890001166AA8
:10304000156A146A136A5BC91AF05AC919F059C98A
:1030500018F058C917F004EC07F00108D8B448EF8D
:1030600018F0166A156A146A136A63C91AF062C9FD
:1030700019F061C918F060C917F004EC07F00108F5
:10308000D8B445EF18F001013889000159EF18F064
:10309000090160530001D8B458EF18F0D89609011F
:1030A00061AFD8860001D8B658EF18F00101388911
:1030B0000001DB0E09016F6F0F0E6E6F490E6D6F11
:1030C000800E6C6FDB0E736F0F0E726F490E716F97
:1030D000810E706FDB0E776F0F0E766F490E756F76
:1030E0007E0E746F63C916F062C915F061C914F0E1
:1030F00060C913F008EC09F09E6F9E5158EC09F07E
:1031000016C0A2F915C0A1F914C0A0F913C09FF907
:10311000A2C916F0A1C915F0A0C914F09FC913F0F7
:103120006FC91AF06EC919F06DC918F06CC917F0A3
:10313000B8EC08F016C034F015C033F014C032F00B
:1031400013C031F01A6A196A340E186E860E176EA3
:1031500034C016F033C015F032C014F031C013F093
:1031600050EC08F016C0A2F915C0A1F914C0A0F9DE
:1031700013C09FF9A2C916F0A1C915F0A0C914F097
:103180009FC913F0D4EC04F016C0A2F915C0A1F940
:1031900014C0A0F913C09FF963C9AEF962C9ADF9B3
:1031A00061C9ACF9AC9F60C9ABF95FC9B2F95EC93E
:1031B000B1F95DC9B0F9B09F5CC9AFF95BC9B6F9A7
:1031C0005AC9B5F959C9B4F9B49F58C9B3F957C91F
:1031D000BAF956C9B9F955C9B8F9B89F54C9B7F978
:1031E000AEC916F0ADC915F0ACC914F0ABC913F0F7
:1031F000B6C91AF0B5C919F0B4C918F0B3C917F0B7
:10320000B4EC07F016C0A6F915C0A5F914C0A4F9CE
:1032100013C0A3F9B2C916F0B1C915F0B0C914F0C2
:10322000AFC913F0BAC91AF0B9C919F0B8C918F082
:10323000B7C917F0B4EC07F016C034F015C033F07E
:1032400014C032F013C031F034C016F033C015F0A2
:1032500032C014F031C013F0A2C91AF0A1C919F09C
:10326000A0C918F09FC917F0B8EC08F016C0AAF969
:1032700015C0A9F914C0A8F913C0A7F9A6C916F07A
:10328000A5C915F0A4C914F0A3C913F0A6C91AF072
:10329000A5C919F0A4C918F0A3C917F0B8EC08F033
:1032A00016C07FF915C07EF914C07DF913C07CF9F2
:1032B000AAC916F0A9C915F0A8C914F0A7C913F036
:1032C000AAC91AF0A9C919F0A8C918F0A7C917F016
:1032D000B8EC08F016C083F915C082F914C081F962
:1032E00013C080F983C916F082C915F081C914F0A2
:1032F00080C913F07FC91AF07EC919F07DC918F092
:103300007CC917F0B6EC07F016C083F915C082F936
:1033100014C081F913C080F983C916F082C915F071
:1033200081C914F080C913F04EEC06F016C08FF975
:1033300015C08EF914C08DF913C08CF9166ACC0E25
:10334000156E580E146E8F0E136E8FC91AF08EC93B
:1033500019F08DC918F08CC917F0B8EC08F016C038
:103360008FF915C08EF914C08DF913C08CF98FC96F
:1033700016F08EC915F08DC914F08CC913F01A6AB5
:10338000196A7A0E186E890E176E78EC07F03B6E8C
:10339000E86A010138B9010E3B140001D8B40AEF04
:1033A0001DF0A6C97FF9A5C97EF9A4C97DF9090157
:1033B0007D9FA3C97CF9AAC983F9A9C982F9A8C9C3
:1033C00081F9819FA7C980F97FC916F07EC915F0E0
:1033D0007DC914F07CC913F083C91AF082C919F0B1
:1033E00081C918F080C917F050EC08F016C083F9B5
:1033F00015C082F914C081F913C080F983C916F091
:1034000082C915F081C914F080C913F07EEC03F075
:1034100016C08BF915C08AF914C089F913C088F950
:10342000166A156A340E146E860E136E8BC91AF066
:103430008AC919F089C918F088C917F0B8EC08F0E2
:1034400016C034F015C033F014C032F013C031F0A0
:1034500034C016F033C015F032C014F031C013F090
:103460006FC91AF06EC919F06DC918F06CC917F060
:1034700050EC08F016C08BF915C08AF914C089F910
:1034800013C088F9166A500E156E430E146E8F0E17
:10349000136E8BC91AF08AC919F089C918F088C946
:1034A00017F0B8EC08F016C07FF915C07EF914C00B
:1034B0007DF913C07CF9166A156A146A136A63C928
:1034C0001AF062C919F061C918F060C917F004EC6C
:1034D00007F001080001D8B4BCEF1BF0166A156AAA
:1034E000146A136A5FC91AF05EC919F05DC918F051
:1034F0005CC917F004EC07F00108D8B41EEF1BF00C
:10350000166A156A146A136AA6C91AF0A5C919F0D1
:10351000A4C918F0A3C917F004EC07F00108D8B447
:10352000D8EF1AF0166A156A146A136AAAC91AF053
:10353000A9C919F0A8C918F0A7C917F004EC07F039
:103540000108D8B4BEEF1AF0166A156A070E146E99
:10355000870E136E8BC91AF08AC919F089C918F041
:1035600088C917F0B4EC07F016C08BF915C08AF9BA
:1035700014C089F913C088F9D6EF1AF0166A156AD3
:10358000340E146E850E136E8BC91AF08AC919F0A9
:1035900089C918F088C917F0B6EC07F016C08BF986
:1035A00015C08AF914C089F913C088F91CEF1BF003
:1035B000166A156A146A136AAAC91AF0A9C919F019
:1035C000A8C918F0A7C917F004EC07F00108D8B48F
:1035D00004EF1BF0166A156A070E146E870E136E41
:1035E0008BC91AF08AC919F089C918F088C917F06F
:1035F000B6EC07F016C08BF915C08AF914C089F92A
:1036000013C088F91CEF1BF0166A156A340E146E8D
:10361000850E136E8BC91AF08AC919F089C918F082
:1036200088C917F0B4EC07F016C08BF915C08AF9F9
:1036300014C089F913C088F9BAEF1BF0166A156A2D
:10364000146A136AA6C91AF0A5C919F0A4C918F01A
:10365000A3C917F004EC07F00108D8B476EF1BF00B
:10366000166A156A146A136AAAC91AF0A9C919F068
:10367000A8C918F0A7C917F004EC07F00108D8B4DE
:103680005CEF1BF0166A156A340E146E850E136E0D
:103690008BC91AF08AC919F089C918F088C917F0BE
:1036A000B6EC07F016C08BF915C08AF914C089F979
:1036B00013C088F974EF1BF0166A156A070E146EB2
:1036C000870E136E8BC91AF08AC919F089C918F0D0
:1036D00088C917F0B4EC07F016C08BF915C08AF949
:1036E00014C089F913C088F9BAEF1BF0166A156A7D
:1036F000146A136AAAC91AF0A9C919F0A8C918F05E
:10370000A7C917F004EC07F00108D8B4A2EF1BF02A
:10371000166A156A340E146E850E136E8BC91AF074
:103720008AC919F089C918F088C917F0B4EC07F0F4
:1037300016C08BF915C08AF914C089F913C088F92D
:10374000BAEF1BF0166A156A070E146E870E136E19
:103750008BC91AF08AC919F089C918F088C917F0FD
:10376000B6EC07F016C08BF915C08AF914C089F9B8
:1037700013C088F908EF1DF0166A156A146A136AF7
:103780005FC91AF05EC919F05DC918F05CC917F07D
:1037900004EC07F00108D8B46CEF1CF0166A156A47
:1037A000146A136AA6C91AF0A5C919F0A4C918F0B9
:1037B000A3C917F004EC07F00108D8B426EF1CF0F9
:1037C000166A156A146A136AAAC91AF0A9C919F007
:1037D000A8C918F0A7C917F004EC07F00108D8B47D
:1037E0000CEF1CF0166A156A070E146E870E136E26
:1037F0008BC91AF08AC919F089C918F088C917F05D
:10380000B6EC07F016C08BF915C08AF914C089F917
:1038100013C088F924EF1CF0166A156A340E146E72
:10382000850E136E8BC91AF08AC919F089C918F070
:1038300088C917F0B4EC07F016C08BF915C08AF9E7
:1038400014C089F913C088F96AEF1CF0166A156A6A
:10385000146A136AAAC91AF0A9C919F0A8C918F0FC
:10386000A7C917F004EC07F00108D8B452EF1CF018
:10387000166A156A070E146E870E136E8BC91AF03E
:103880008AC919F089C918F088C917F0B4EC07F093
:1038900016C08BF915C08AF914C089F913C088F9CC
:1038A0006AEF1CF0166A156A340E146E850E136EDC
:1038B0008BC91AF08AC919F089C918F088C917F09C
:1038C000B6EC07F016C08BF915C08AF914C089F957
:1038D00013C088F908EF1DF0166A156A146A136A96
:1038E000A6C91AF0A5C919F0A4C918F0A3C917F000
:1038F00004EC07F00108D8B4C4EF1CF0166A156A8E
:10390000146A136AAAC91AF0A9C919F0A8C918F04B
:10391000A7C917F004EC07F00108D8B4AAEF1CF00F
:10392000166A156A340E146E850E136E8BC91AF062
:103930008AC919F089C918F088C917F0B4EC07F0E2
:1039400016C08BF915C08AF914C089F913C088F91B
:10395000C2EF1CF0166A156A070E146E870E136EFE
:103960008BC91AF08AC919F089C918F088C917F0EB
:10397000B6EC07F016C08BF915C08AF914C089F9A6
:1039800013C088F908EF1DF0166A156A146A136AE5
:10399000AAC91AF0A9C919F0A8C918F0A7C917F03F
:1039A00004EC07F00108D8B4F0EF1CF0166A156AB1
:1039B000340E146E850E136E8BC91AF08AC919F075
:1039C00089C918F088C917F0B6EC07F016C08BF952
:1039D00015C08AF914C089F913C088F908EF1DF0E1
:1039E000166A156A070E146E870E136E8BC91AF0CD
:1039F0008AC919F089C918F088C917F0B4EC07F022
:103A000016C08BF915C08AF914C089F913C088F95A
:103A1000DCEF25F063C916F062C915F061C914F036
:103A200060C913F06FC91AF06EC919F06DC918F0AA
:103A30006CC917F0B8EC08F016C034F015C033F0BC
:103A400014C032F013C031F01A6A196A340E186EBD
:103A5000860E176E34C016F033C015F032C014F065
:103A600031C013F050EC08F016C063F915C062F9CC
:103A700014C061F913C060F95FC916F05EC915F092
:103A80005DC914F05CC913F06FC91AF06EC919F062
:103A90006DC918F06CC917F0B8EC08F016C034F016
:103AA00015C033F014C032F013C031F01A6A196A2D
:103AB000340E186E860E176E34C016F033C015F033
:103AC00032C014F031C013F050EC08F016C05FF9AA
:103AD00015C05EF914C05DF913C05CF95BC916F03E
:103AE0005AC915F059C914F058C913F06FC91AF022
:103AF0006EC919F06DC918F06CC917F0B8EC08F070
:103B000016C034F015C033F014C032F013C031F0D9
:103B10001A6A196A340E186E860E176E34C016F0C3
:103B200033C015F032C014F031C013F050EC08F07F
:103B300016C05BF915C05AF914C059F913C058F9E9
:103B400057C916F056C915F055C914F054C913F0E9
:103B50006FC91AF06EC919F06DC918F06CC917F069
:103B6000B8EC08F016C034F015C033F014C032F0D1
:103B700013C031F01A6A196A340E186E860E176E69
:103B800034C016F033C015F032C014F031C013F059
:103B900050EC08F016C057F915C056F914C055F985
:103BA00013C054F957C916F056C915F055C914F089
:103BB00054C913F05FC91AF05EC919F05DC918F055
:103BC0005CC917F0B4EC07F016C07FF915C07EF998
:103BD00014C07DF913C07CF97FC916F07EC915F0B9
:103BE0007DC914F07CC913F073C91AF072C919F0B9
:103BF00071C918F070C917F050EC08F016C083F9BD
:103C000015C082F914C081F913C080F983C916F078
:103C100082C915F081C914F080C913F008EC09F0CD
:103C200015C09DF909019C6F9CC913F09DC914F042
:103C30005AEC09F073C91AF072C919F071C918F079
:103C400070C917F0B8EC08F016C06BF915C06AF926
:103C500014C069F913C068F97FC916F07EC915F060
:103C60007DC914F07CC913F06BC91AF06AC919F048
:103C700069C918F068C917F0B4EC07F016C06BF901
:103C800015C06AF914C069F913C068F968530001D6
:103C9000D8B46DEF1EF0D896090169AFD88600013F
:103CA000D8B66DEF1EF06BC916F06AC915F069C978
:103CB00014F068C913F073C91AF072C919F071C908
:103CC00018F070C917F0B6EC07F016C06BF915C004
:103CD0006AF914C069F913C068F95FC916F05EC9C2
:103CE00015F05DC914F05CC913F057C91AF056C934
:103CF00019F055C918F054C917F0B4EC07F016C004
:103D00007FF915C07EF914C07DF913C07CF97FC915
:103D100016F07EC915F07DC914F07CC913F073C983
:103D20001AF072C919F071C918F070C917F050EC87
:103D300008F016C083F915C082F914C081F913C0C8
:103D400080F983C916F082C915F081C914F080C9C1
:103D500013F008EC09F015C09DF909019C6F9CC98E
:103D600013F09DC914F05AEC09F073C91AF072C926
:103D700019F071C918F070C917F0B8EC08F016C046
:103D800067F915C066F914C065F913C064F97FC9F5
:103D900016F07EC915F07DC914F07CC913F067C90F
:103DA0001AF066C919F065C918F064C917F0B4ECC7
:103DB00007F016C067F915C066F914C065F913C09D
:103DC00064F964530001D8B408EF1FF0D8960901D4
:103DD00065AFD8860001D8B608EF1FF067C916F0A6
:103DE00066C915F065C914F064C913F073C91AF0F7
:103DF00072C919F071C918F070C917F0B6EC07F064
:103E000016C067F915C066F914C065F913C064F9E6
:103E100063C97FF962C97EF961C97DF90901605101
:103E2000D8B43E84D8A460057C6F7FC916F07EC9E3
:103E300015F07DC914F07CC913F077C91AF076C962
:103E400019F075C918F074C917F0B6EC07F016C070
:103E50007FF915C07EF914C07DF913C07CF97FC9C4
:103E600016F07EC915F07DC914F07CC913F0B0ECD2
:103E700004F016C07FF915C07EF914C07DF913C097
:103E80007CF95BC983F95AC982F959C981F958513A
:103E9000D8B43E84D8A45805806F83C916F082C96F
:103EA00015F081C914F080C913F077C91AF076C9EA
:103EB00019F075C918F074C917F0B6EC07F016C000
:103EC00083F915C082F914C081F913C080F983C940
:103ED00016F082C915F081C914F080C913F0B0EC56
:103EE00004F016C083F915C082F914C081F913C01B
:103EF00080F983C916F082C915F081C914F080C910
:103F000013F07FC91AF07EC919F07DC918F07CC979
:103F100017F050EC08F016C07BF915C07AF914C000
:103F200079F913C078F97BC916F07AC915F079C907
:103F300014F078C913F064EC02F016C07BF915C0D8
:103F40007AF914C079F913C078F95BC916F05AC927
:103F500015F059C914F058C913F063C91AF062C9B1
:103F600019F061C918F060C917F0B4EC07F016C079
:103F70007FF915C07EF914C07DF913C07CF97C531C
:103F80000001D8B4CFEF1FF0D89609017DAFD886D5
:103F90000001D8B6CFEF1FF0800E09017D1B000194
:103FA0007DBF0DD0DC0E09017F5D240E7E59340EDD
:103FB0007D59500E7C590001D8B0F3EF1FF063C952
:103FC00016F062C915F061C914F060C913F0D4ECA1
:103FD00004F016C087F915C086F914C085F913C01E
:103FE00084F927EF20F05BC916F05AC915F059C9BA
:103FF00014F058C913F063C91AF062C919F061C905
:1040000018F060C917F0B4EC07F016C07FF915C0BE
:104010007EF914C07DF913C07CF97FC916F07EC902
:1040200015F07DC914F07CC913F07BC91AF07AC968
:1040300019F079C918F078C917F050EC08F016C0DB
:1040400087F915C086F914C085F913C084F96BC9C6
:1040500016F06AC915F069C914F068C913F067C988
:104060001AF066C919F065C918F064C917F004ECB4
:1040700007F00108D8B416EF22F06BC97FF96AC9BE
:104080007EF969C97DF968C97CF9166A156A146AEE
:10409000136A7BC91AF07AC919F079C918F078C97E
:1040A00017F004EC07F00108D8B485EF20F07FC9C1
:1040B00016F07EC915F07DC914F07CC913F07BC9D8
:1040C0001AF07AC919F079C918F078C917F050ECCC
:1040D00008F016C083F915C082F914C081F913C025
:1040E00080F983C916F082C915F081C914F080C91E
:1040F00013F07EEC03F016C083F915C082F914C0EA
:1041000081F913C080F993EF21F009017853000180
:10411000D8A4E9EF20F0166A156A146A136A7FC9F9
:104120001AF07EC919F07DC918F07CC917F004ECAB
:1041300007F00108D8B4ADEF20F06FC983F96EC95C
:1041400082F96DC981F909016C51D8B43E84D8A4B3
:104150006C05806F0001E7EF20F009017C5300013E
:10416000D8B4E1EF20F0D89609017DAFD8860001E0
:10417000D8B6E1EF20F0166A156A146A136A6FC99F
:104180001AF06EC919F06DC918F06CC917F0B4ECCB
:1041900007F016C034F015C033F014C032F013C06D
:1041A00031F034C083F933C082F932C081F9315023
:1041B000D8B43E84D8A431040901806F0001E6EF31
:1041C00020F009018B6B8A6B896B886B000193EF80
:1041D00021F0090178530001D8B493EF21F0D8966B
:1041E000090179AFD8860001D8B693EF21F0090113
:1041F0007C530001D8B44DEF21F0D89609017DAF72
:10420000D8860001D8B64DEF21F07FC916F07EC9DF
:1042100015F07DC914F07CC913F07BC91AF07AC976
:1042200019F079C918F078C917F050EC08F016C0E9
:1042300083F915C082F914C081F913C080F983C9CC
:1042400016F082C915F081C914F080C913F07EEC14
:1042500003F016C083F915C082F914C081F913C0A8
:1042600080F983C916F082C915F081C914F080C99C
:1042700013F06FC91AF06EC919F06DC918F06CC946
:1042800017F0B4EC07F016C083F915C082F914C01A
:1042900081F913C080F993EF21F07FC916F07EC930
:1042A00015F07DC914F07CC913F07BC91AF07AC9E6
:1042B00019F079C918F078C917F050EC08F016C059
:1042C00083F915C082F914C081F913C080F983C93C
:1042D00016F082C915F081C914F080C913F07EEC84
:1042E00003F016C083F915C082F914C081F913C018
:1042F00080F983C916F082C915F081C914F080C90C
:1043000013F06FC91AF06EC919F06DC918F06CC9B5
:1043100017F0B6EC07F016C083F915C082F914C087
:1043200081F913C080F983C916F082C915F081C9DB
:1043300014F080C913F073C91AF072C919F071C969
:1043400018F070C917F050EC08F016C07FF915C0CE
:104350007EF914C07DF913C07CF97FC916F07EC9BF
:1043600015F07DC914F07CC913F008EC09F015C0F4
:104370009DF909019C6F9CC913F09DC914F05AEC7A
:1043800009F073C91AF072C919F071C918F070C92F
:1043900017F0B8EC08F016C08BF915C08AF914C0F4
:1043A00089F913C088F983C916F082C915F081C94B
:1043B00014F080C913F08BC91AF08AC919F089C9A1
:1043C00018F088C917F0B4EC07F016C08BF915C0C7
:1043D0008AF914C089F913C088F988530001D8B448
:1043E00014EF22F0D896090189AFD8860001D8B61B
:1043F00014EF22F08BC916F08AC915F089C914F0A0
:1044000088C913F073C91AF072C919F071C918F08C
:1044100070C917F0B6EC07F016C08BF915C08AF911
:1044200014C089F913C088F9E5EF23F067C97FF953
:1044300066C97EF965C97DF9800E09017D1B64C9D5
:104440007CF9166A156A146A136A7BC91AF07AC96C
:1044500019F079C918F078C917F004EC07F00108D1
:104460000001D8B462EF22F07FC916F07EC915F0C2
:104470007DC914F07CC913F07BC91AF07AC919F010
:1044800079C918F078C917F050EC08F016C083F914
:1044900015C082F914C081F913C080F983C916F0E0
:1044A00082C915F081C914F080C913F07EEC03F0C5
:1044B00016C083F915C082F914C081F913C080F9C0
:1044C00064EF23F0090178530001D8A4BAEF22F079
:1044D000166A156A146A136A7FC91AF07EC919F040
:1044E0007DC918F07CC917F004EC07F00108D8B4B6
:1044F0008AEF22F06FC983F96EC982F96DC981F91B
:1045000009016C51D8B43E84D8A46C05806F0001B9
:10451000B8EF22F009017C530001D8B4B2EF22F0C9
:10452000D89609017DAFD8860001D8B6B2EF22F047
:104530006FC90EF06EC90DF06DC90CF0800E0C1A2B
:104540006CC90BF00EC083F90DC082F90CC081F963
:104550000B50D8B43E84D8A40B040901806F00012D
:10456000B7EF22F009018B6B8A6B896B886B0001B6
:1045700064EF23F0090178530001D8B464EF23F00D
:10458000D896090179AFD8860001D8B664EF23F038
:1045900009017C530001D8B41EEF23F0D89609011D
:1045A0007DAFD8860001D8B61EEF23F07FC916F084
:1045B0007EC915F07DC914F07CC913F07BC91AF0CF
:1045C0007AC919F079C918F078C917F050EC08F0D9
:1045D00016C083F915C082F914C081F913C080F99F
:1045E00083C916F082C915F081C914F080C913F08F
:1045F0007EEC03F016C083F915C082F914C081F96E
:1046000013C080F983C916F082C915F081C914F06E
:1046100080C913F06FC91AF06EC919F06DC918F08E
:104620006CC917F0B4EC07F016C083F915C082F915
:1046300014C081F913C080F964EF23F07FC916F02C
:104640007EC915F07DC914F07CC913F07BC91AF03E
:104650007AC919F079C918F078C917F050EC08F048
:1046600016C083F915C082F914C081F913C080F90E
:1046700083C916F082C915F081C914F080C913F0FE
:104680007EEC03F016C083F915C082F914C081F9DD
:1046900013C080F983C916F082C915F081C914F0DE
:1046A00080C913F06FC91AF06EC919F06DC918F0FE
:1046B0006CC917F0B6EC07F016C083F915C082F983
:1046C00014C081F913C080F983C916F082C915F0AE
:1046D00081C914F080C913F073C91AF072C919F0B6
:1046E00071C918F070C917F050EC08F016C07FF9C6
:1046F00015C07EF914C07DF913C07CF97FC916F08E
:104700007EC915F07DC914F07CC913F008EC09F0DE
:1047100015C09DF909019C6F9CC913F09DC914F047
:104720005AEC09F073C91AF072C919F071C918F07E
:1047300070C917F0B8EC08F016C08BF915C08AF9EB
:1047400014C089F913C088F983C916F082C915F01D
:1047500081C914F080C913F08BC91AF08AC919F005
:1047600089C918F088C917F0B4EC07F016C08BF9A6
:1047700015C08AF914C089F913C088F9885300015B
:10478000D8B4E5EF23F0D896090189AFD8860001A7
:10479000D8B6E5EF23F08BC916F08AC915F089C9A0
:1047A00014F088C913F073C91AF072C919F071C9ED
:1047B00018F070C917F0B6EC07F016C08BF915C0E9
:1047C0008AF914C089F913C088F9166A156A340E7B
:1047D000146E860E136E8BC91AF08AC919F089C936
:1047E00018F088C917F0B8EC08F016C08BF915C09E
:1047F0008AF914C089F913C088F98BC916F08AC9DF
:1048000015F089C914F088C913F06FC91AF06EC980
:1048100019F06DC918F06CC917F050EC08F016C00B
:104820008BF915C08AF914C089F913C088F9166A82
:10483000156A330E146E870E136E8BC91AF08AC96F
:1048400019F089C918F088C917F004EC07F00108BD
:10485000D8B433EF24F009018B6B800E8A6F330ECE
:10486000896F870E886F00016BC916F06AC915F051
:1048700069C914F068C913F067C91AF066C919F05C
:1048800065C918F064C917F004EC07F00108D8B442
:10489000FAEF24F087C916F086C915F085C914F01F
:1048A00084C913F087C91AF086C919F085C918F0B0
:1048B00084C917F0B8EC08F016C07FF915C07EF96E
:1048C00014C07DF913C07CF96BC916F06AC915F0E4
:1048D00069C914F068C913F06BC91AF06AC919F0F4
:1048E00069C918F068C917F0B8EC08F016C083F968
:1048F00015C082F914C081F913C080F97FC916F080
:104900007EC915F07DC914F07CC913F083C91AF073
:1049100082C919F081C918F080C917F0B8EC08F005
:1049200016C07FF915C07EF914C07DF913C07CF95B
:104930005BC916F05AC915F059C914F058C913F0DB
:1049400063C91AF062C919F061C918F060C917F09B
:10495000B4EC07F016C083F915C082F914C081F9D0
:1049600013C080F983C916F082C915F081C914F00B
:1049700080C913F083C91AF082C919F081C918F0EF
:1049800080C917F0B8EC08F016C083F915C082F999
:1049900014C081F913C080F97FC916F07EC915F0E3
:1049A0007DC914F07CC913F083C91AF082C919F0CB
:1049B00081C918F080C917F0B6EC07F016C08FF95E
:1049C00015C08EF914C08DF913C08CF98FC916F07B
:1049D0008EC915F08DC914F08CC913F04EEC06F099
:1049E00016C08FF915C08EF914C08DF913C08CF95B
:1049F000A8EF25F087C916F086C915F085C914F00F
:104A000084C913F087C91AF086C919F085C918F04E
:104A100084C917F0B8EC08F016C07FF915C07EF90C
:104A200014C07DF913C07CF967C916F066C915F08A
:104A300065C914F064C913F067C91AF066C919F0A2
:104A400065C918F064C917F0B8EC08F016C083F90E
:104A500015C082F914C081F913C080F97FC916F01E
:104A60007EC915F07DC914F07CC913F083C91AF012
:104A700082C919F081C918F080C917F0B8EC08F0A4
:104A800016C07FF915C07EF914C07DF913C07CF9FA
:104A90005BC916F05AC915F059C914F058C913F07A
:104AA00063C91AF062C919F061C918F060C917F03A
:104AB000B4EC07F016C083F915C082F914C081F96F
:104AC00013C080F983C916F082C915F081C914F0AA
:104AD00080C913F083C91AF082C919F081C918F08E
:104AE00080C917F0B8EC08F016C083F915C082F938
:104AF00014C081F913C080F97FC916F07EC915F082
:104B00007DC914F07CC913F083C91AF082C919F069
:104B100081C918F080C917F0B6EC07F016C08FF9FC
:104B200015C08EF914C08DF913C08CF98FC916F019
:104B30008EC915F08DC914F08CC913F04EEC06F037
:104B400016C08FF915C08EF914C08DF913C08CF9F9
:104B5000166A156A480E146E850E136E8FC91AF008
:104B60008EC919F08DC918F08CC917F004EC07F044
:104B70000108D8B4C1EF25F009018F6B8E6B8D6BE6
:104B80008C6B0001320E166EA50E156E420E146E61
:104B9000950E136E8FC91AF08EC919F08DC918F0D1
:104BA0008CC917F0B8EC08F016C08FF915C08EF953
:104BB00014C08DF913C08CF98DBF0DD0400E0901C2
:104BC0008F5DD70E8E59340E8D59900E8C59000181
:104BD000D8B000EF26F08FC916F08EC915F08DC938
:104BE00014F08CC913F008EC09F013C093F914C049
:104BF00092F915C091F90901906F000108EF26F0B4
:104C00000901936B020E926FD30E916F5D0E906F40
:104C100000018BC916F08AC915F089C914F088C93A
:104C200013F008EC09F013C097F914C096F915C0F9
:104C300095F90901946F97C922F096C921F095C999
:104C400020F094C91FF02A6A0F0E296E420E286EBA
:104C5000400E276E02EC02F022C097F921C096F9AF
:104C600020C095F91FC094F99B6B9A6B996B986B58
:104C700090519425986F91519521996F9251962159
:104C80009A6F935197219B6F98C9DEFF99C9DEFFF8
:104C90009AC9DEFF9BC9DEFF00011200010E06016A
:104CA0003D6F4D0E3C6F010E3F6F2C0E3E6F010E9F
:104CB000416F2C0E406F010E436F2C0E426F010EA0
:104CC000456F2C0E446F010E476F2C0E466F010E80
:104CD000496F2C0E486F010E4B6F2C0E4A6F010E60
:104CE0004D6F900E4C6F010E4F6FF40E4E6F020E13
:104CF000516F580E506F020E536FBC0E526F030E61
:104D0000556F200E546F030E576F840E566F030EAF
:104D1000596FE80E586F030E5B6FE80E5A6F030E63
:104D20005D6FE80E5C6F030E5F6FE80E5E6F030E43
:104D3000616FE80E606F030E636FE80E626F030E23
:104D4000656FE80E646F030E676FE80E666F030E03
:104D5000696FE80E686F030E6B6FE80E6A6F030EE3
:104D60006D6FE80E6C6F030E6F6FE80E6E6F030EC3
:104D7000716FE80E706F030E736FE80E726F040EA2
:104D8000756F4C0E746F040E776FB00E766F050E54
:104D9000796F140E786F050E7B6F780E7A6F050EA3
:104DA0007D6FDC0E7C6F050E7F6F780E7E6F050EBB
:104DB000816F140E806F040E836FB00E826F030E2E
:104DC000856FE80E846F030E876FDE0E866F030E0D
:104DD000896FD40E886F030E8B6FCA0E8A6F030E15
:104DE0008D6FD40E8C6F030E8F6FDE0E8E6F030EE1
:104DF000916FE80E906F040E936F4C0E926F040E3D
:104E0000956FB00E946F040E976FB00E966F040EF0
:104E1000996FB00E986F040E9B6FB00E9A6F040ED0
:104E20009D6FB00E9C6F040E9F6FB00E9E6F040EB0
:104E3000A16FB00EA06F040EA36FB00EA26F040E90
:104E4000A56FB00EA46F030EA76FE80EA66F030E3A
:104E5000A96FDE0EA86F030EAB6FD40EAA6F030E00
:104E6000AD6FCA0EAC6F030EAF6FD40EAE6F030EF4
:104E7000B16FDE0EB06F030EB36FE80EB26F030EAC
:104E8000B56F840EB46F030EB76F200EB66F020EAF
:104E9000B96FBC0EB86F020EBB6F580EBA6F020E20
:104EA000BD6F580EBC6F020EBF6F580EBE6F020E64
:104EB000C16F580EC06F020EC36F580EC26F020E44
:104EC000C56F580EC46F020EC76F580EC66F020E24
:104ED000C96F580EC86F020ECB6F580ECA6F020E04
:104EE000CD6F580ECC6F020ECF6F580ECE6F020EE4
:104EF000D16F580ED06F020ED36F580ED26F020EC4
:104F0000D56F580ED46F020ED76F580ED66F020EA3
:104F1000D96F580ED86F020EDB6F580EDA6F020E83
:104F2000DD6F580EDC6F020EDF6F580EDE6F020E63
:104F3000E16F8A0EE06F020EE36F8A0EE26F020EDF
:104F4000E56F8A0EE46F020EE76F8A0EE66F020EBF
:104F5000E96F8A0EE86F020EEB6F8A0EEA6F020E9F
:104F6000ED6F8A0EEC6F020EEF6F8A0EEE6F020E7F
:104F7000F16F8A0EF06F020EF36F8A0EF26F020E5F
:104F8000F56F8A0EF46F020EF76F260EF66F020EA3
:104F9000F96F260EF86F020EFB6F260EFA6F020EE7
:104FA000FD6F260EFC6F020EFF6F260EFE6F020EC7
:104FB0000701016F260E006F020E036F260E026FAF
:104FC000020E056F260E046F020E076F260E066F87
:104FD000020E096F260E086F020E0B6F260E0A6F67
:104FE000020E0D6F260E0C6F020E0F6F260E0E6F47
:104FF000020E116F260E106F020E136F260E126F27
:10500000020E156F260E146F010E176FF40E166F39
:10501000010E196FC20E186F010E1B6F900E1A6FE2
:10502000010E1D6F5E0E1C6F010E1F6F2C0E1E6F8A
:10503000010E216F2C0E206F010E236F2C0E226F9C
:10504000010E256F2C0E246F010E276F2C0E266F7C
:10505000010E296F2C0E286F010E2B6F2C0E2A6F5C
:105060002D6B2C6B2F6B140E2E6F316B280E306F47
:10507000336B3C0E326F356B500E346F376B640EF2
:10508000366F396B780E386F3B6B8C0E3A6F3D6B19
:10509000A00E3C6F3F6BB40E3E6F416BC80E406F6D
:1050A000436BB40E426F456BA00E446F476B8C0E82
:1050B000466F496B780E486F4B6B640E4A6F4D6BB1
:1050C000500E4C6F4F6B3C0E4E6F516B280E506F55
:1050D000536B140E526F556B546B576B050E566F16
:1050E000596B0A0E586F5B6B0A0E5A6F5D6B0A0E96
:1050F0005C6F5F6B0A0E5E6F616B0A0E606F636BB5
:105100000A0E626F656B0A0E646F676B0A0E666F3C
:10511000696B0F0E686F6B6B140E6A6F6D6B190EF7
:105120006C6F6F6B1E0E6E6F716B230E706F736BF7
:10513000280E726F756B0A0E746F776B0F0E766F99
:10514000796B140E786F7B6B190E7A6F7D6B1E0E68
:105150007C6F7F6B230E7E6F816B280E806F836B5D
:105160002D0E826F856B320E846F876B370E866FC4
:10517000896B3C0E886F8B6B3D0E8A6F8D6B3E0E7C
:105180008C6F8F6B3D0E8E6F916B3C0E906F936B9F
:105190003B0E926F956B3A0E946F976B3B0E966F2A
:1051A000996B460E986F9B6B500E9A6F9D6B5A0EC3
:1051B0009C6F9F6B640E9E6FA16B6E0EA06FA36BB6
:1051C000780EA26FA56B820EA46FA76B8C0EA66FD4
:1051D000A96B960EA86FAB6BA00EAA6FAD6BAA0E53
:1051E000AC6FAF6BB40EAE6FB16BBE0EB06FB36B86
:1051F000C80EB26FB56BD20EB46FB76BD30EB66F6D
:10520000B96BD40EB86FBB6BD30EBA6FBD6BD40E37
:10521000BC6FBF6BD30EBE6FC16BD40EC06FC36BC0
:10522000D50EC26FC56BD40EC46FC76BD50EC66FDB
:10523000C96BD60EC86FCB6BDC0ECA6FCD6BF00E90
:10524000CC6F010ECF6F040ECE6F010ED16F180E12
:10525000D06F010ED36F2C0ED26F010ED56F400EA2
:10526000D46F010ED76F540ED66F010ED96F5E0E3C
:10527000D86F010EDB6F5E0EDA6F010EDD6F5E0E12
:10528000DC6F010EDF6F5E0EDE6F010EE16F630EED
:10529000E06FE36BE26BE56B0A0EE46FE76B140EF5
:1052A000E66FE96B1E0EE86FEB6B280EEA6FED6B95
:1052B000320EEC6FEF6B3C0EEE6FF16B460EF06F43
:1052C000F36B500EF26FF56B5A0EF46FF76B5F0EC7
:1052D000F66FF96B5F0EF86FFB6B5F0EFA6FFD6B8D
:1052E0005F0EFC6FFF6B5F0EFE6F0801016B5F0EC0
:1052F000006F036B5F0E026F056B5F0E046F076B31
:105300005F0E066F096B590E086F0B6B530E0A6F19
:105310000D6B4D0E0C6F0F6B470E0E6F116B410E28
:10532000106F136B3B0E126F156B350E146F176BEE
:105330002F0E166F196B290E186F1B6B230E1A6F29
:1053400000011200A30E0901DC6FA20EDD6FAB0E8F
:10535000DE6FAA0EDF6F01014F510A0DF3CF31F05E
:10536000F4CF32F0505131240B6E0BC0BBF95151C8
:105370000A0DF3CF31F0F4CF32F0525131240B6EDD
:105380000BC0BCF953510A0DF3CF31F0F4CF32F01A
:10539000545131240B6E0BC0BDF956510A0DF3CF99
:1053A00031F0F4CF32F0575131240B6E0BC0BEF9FF
:1053B00058510A0DF3CF31F0F4CF32F05951312466
:1053C0000B6E0BC0BFF95A510A0DF3CF31F0F4CF79
:1053D00032F05B5131240B6E0BC0C0F95C510A0DE9
:1053E000F3CF31F0F4CF32F05D5131240B6E0BC0AE
:1053F000C1F94E0E5E5D0001D8A403EF2AF06FC123
:10540000C2F909EF2AF00A0E01016F250B6E0BC0DD
:10541000C2F9000101015F510A0DF3CF31F0F4CF61
:1054200032F0605131240B6E0BC0C3F961510A0D8B
:10543000F3CF31F0F4CF32F0625131240B6E0BC058
:10544000C4F963510A0DF3CF31F0F4CF32F0645157
:1054500031240B6E0BC0C5F965510A0DF3CF31F045
:10546000F4CF32F0665131240B6E0BC0C6F9450EF5
:10547000685D0001D8A446EF2AF0140E01016725EB
:105480000B6E0BC0C7F900014CEF2AF01E0E010194
:1054900067250B6E0BC0C7F90001010169510A0DA8
:1054A000F3CF31F0F4CF32F06A5131240B6E0BC0E0
:1054B000C8F96B510A0DF3CF31F0F4CF32F06C51D3
:1054C00031240B6E0BC0C9F970510A0DF3CF31F0C6
:1054D000F4CF32F0715131240B6E0BC0CAF9725106
:1054E0000A0DF3CF31F0F4CF32F0735131240B6E4B
:1054F0000BC0CBF974510A0DF3CF31F0F4CF32F079
:10550000755131240B6E0BC0CCF976510A0DF3CFD7
:1055100031F0F4CF32F0775131240B6E0BC0CDF95E
:1055200005011E510A0DF3CF31F0F4CF32F01F51B7
:1055300031240B6E0BC0CEF920510A0DF3CF31F0A0
:10554000F4CF32F0215131240B6E0BC0CFF9EA0EAB
:105550000901D06FD16B0001160E0901D15D000168
:10556000D8B042EF2BF0D896BEBFD886D8B6D2EFCF
:105570002AF0FE0EBB5DFF0EBC59010EBD59000E98
:10558000BE59D8A0D2EF2AF0AA6A450EA96E010E24
:1055900046EC01F0010EB96F010E0801286F000101
:1055A0003DEF2BF0D896BEBFD886D8B620EF2BF0B3
:1055B000000EBE5DD8A020EF2BF011E1000EBD5D06
:1055C000D8A020EF2BF00BE1FF0EBC5DD8A020EFA0
:1055D0002BF005E1FE0EBB5DD8A020EF2BF0BB2B1E
:1055E000000EBC23BD23BE23FF0EBB5D0901D26F9D
:1055F000FF0E0001BC590901D36F000E0001BD5917
:105600000901D46F000E0001BE590901D56FD3C93D
:10561000D7F9D2C9D6F9DF51FFEC00F0D751FFEC32
:1056200000F0D651FFEC00F009EEBBF0D151EB5089
:10563000FDEC00F0050E54EC01F000013CEF2BF006
:10564000BB2B000EBC23BD23BE23BCC0D7F9BBC0FF
:10565000D6F90901DD51FFEC00F0D751FFEC00F065
:10566000D651FFEC00F009EEBBF0D151EB50FDEC50
:1056700000F0050E54EC01F000010901D12B0001EE
:10568000D8A469D7BEC0D8F9BDC0D9F9BCC0DAF971
:10569000BBC0DBF90901DD51FFEC00F00001C05196
:1056A000FFEC00F0BF51FFEC00F00901D851FDEC18
:1056B00000F0050E54EC01F0DD51FFEC00F0010E9E
:1056C0000001BF25316E000EC021326E3250FFEC5A
:1056D00000F03150FFEC00F00901D951FDEC00F071
:1056E000050E54EC01F0DD51FFEC00F0020E00015C
:1056F000BF25316E000EC021326E3250FFEC00F03B
:105700003150FFEC00F00901DA51FDEC00F0050E1C
:1057100054EC01F0DD51FFEC00F0030E0001BF2559
:10572000316E000EC021326E3250FFEC00F031506D
:10573000FFEC00F00901DB51FDEC00F0050E54EC2C
:1057400001F0000112000A0E8C5DD8A4B6EF2BF018
:1057500026ECBDF0DE6ADE6A9D0EDE6E200EDE6E89
:10576000010EDE6EE4ECA8F0B7EF32F00B0E8C5DAC
:10577000D8A4C9EF2BF0DFECBCF0DE6ADE6A2F0E96
:10578000DE6E0C0EDE6E020EDE6EE4ECA8F0B7EFFD
:1057900032F00C0E8C5DD8A4DCEF2BF0DFECBCF00B
:1057A000DE6ADE6A2D0EDE6E1B0EDE6E020EDE6E11
:1057B000E4ECA8F0B7EF32F00D0E8C5DD8A4EFEF5B
:1057C0002BF0DFECBCF0DE6ADE6A2B0EDE6E0E0E16
:1057D000DE6E020EDE6EE4ECA8F0B7EF32F0140ECF
:1057E0008C5DD8A401EF2CF026ECBDF0DE6ADE6AF9
:1057F0009F0EDE6E140EDE6EDE6AE4ECA8F0B7EFEC
:1058000032F0150E8C5DD8A41DEF2CF059ECBDF0D4
:10581000DE6ADE6A250EDE6E1B0EDE6EDE6AE4ECEC
:10582000A8F0DE6ADE6A330EDE6E0E0EDE6E0C0E41
:10583000DE6EE4ECA8F0B7EF32F0160E8C5DD8A463
:1058400039EF2CF059ECBDF0DE6ADE6A270EDE6E11
:105850000C0EDE6EDE6AE4ECA8F0DE6ADE6A350E5F
:10586000DE6E1B0EDE6E0C0EDE6EE4ECA8F0B7EF03
:1058700032F0170E8C5DD8A455EF2CF059ECBDF02A
:10588000DE6ADE6A270EDE6E0C0EDE6EDE6AE4EC89
:10589000A8F0DE6ADE6A330EDE6E0E0EDE6E0C0ED1
:1058A000DE6EE4ECA8F0B7EF32F01E0E8C5DD8A4EB
:1058B00068EF2CF026ECBDF0DE6ADE6AA30EDE6E29
:1058C000110EDE6E010EDE6EE4ECA8F0B7EF32F0E2
:1058D0001F0E8C5DD8A484EF2CF059ECBDF0DE6A6D
:1058E000DE6A250EDE6E1B0EDE6EDE6AE4ECA8F0CC
:1058F000DE6ADE6A970EDE6E210EDE6E0C0EDE6E46
:10590000E4ECA8F0B7EF32F0200E8C5DD8A4A0EF45
:105910002CF059ECBDF0DE6ADE6A250EDE6E1B0E41
:10592000DE6EDE6AE4ECA8F0DE6ADE6A950EDE6EFC
:10593000210EDE6E0C0EDE6EE4ECA8F0B7EF32F056
:10594000210E8C5DD8A4BCEF2CF059ECBDF0DE6AC2
:10595000DE6A250EDE6E1B0EDE6EDE6AE4ECA8F05B
:10596000DE6ADE6A930EDE6E210EDE6E0C0EDE6ED9
:10597000E4ECA8F0B7EF32F0220E8C5DD8A4D8EF9B
:105980002CF059ECBDF0DE6ADE6A250EDE6E1B0ED1
:10599000DE6EDE6AE4ECA8F0DE6ADE6A990EDE6E88
:1059A000210EDE6E0C0EDE6EE4ECA8F0B7EF32F0E6
:1059B000230E8C5DD8A4F4EF2CF059ECBDF0DE6A18
:1059C000DE6A270EDE6E0C0EDE6EDE6AE4ECA8F0F8
:1059D000DE6ADE6A950EDE6E210EDE6E0C0EDE6E67
:1059E000E4ECA8F0B7EF32F0240E8C5DD8A410EFF1
:1059F0002DF059ECBDF0DE6ADE6A270EDE6E0C0E6D
:105A0000DE6EDE6AE4ECA8F0DE6ADE6A930EDE6E1D
:105A1000210EDE6E0C0EDE6EE4ECA8F0B7EF32F075
:105A2000250E8C5DD8A42CEF2DF059ECBDF0DE6A6C
:105A3000DE6A270EDE6E0C0EDE6EDE6AE4ECA8F087
:105A4000DE6ADE6A970EDE6E210EDE6E0C0EDE6EF4
:105A5000E4ECA8F0B7EF32F0260E8C5DD8A448EF46
:105A60002DF059ECBDF0DE6ADE6A270EDE6E0C0EFC
:105A7000DE6EDE6AE4ECA8F0DE6ADE6A990EDE6EA7
:105A8000210EDE6E0C0EDE6EE4ECA8F0B7EF32F005
:105A9000270E8C5DD8A464EF2DF059ECBDF0DE6AC2
:105AA000DE6A230EDE6E0E0EDE6EDE6AE4ECA8F019
:105AB000DE6ADE6A930EDE6E210EDE6E0C0EDE6E88
:105AC000E4ECA8F0B7EF32F0280E8C5DD8A480EF9C
:105AD0002DF059ECBDF0DE6ADE6A230EDE6E0E0E8E
:105AE000DE6EDE6AE4ECA8F0DE6ADE6A950EDE6E3B
:105AF000210EDE6E0C0EDE6EE4ECA8F0B7EF32F095
:105B0000290E8C5DD8A49CEF2DF059ECBDF0DE6A17
:105B1000DE6A230EDE6E0E0EDE6EDE6AE4ECA8F0A8
:105B2000DE6ADE6A970EDE6E210EDE6E0C0EDE6E13
:105B3000E4ECA8F0B7EF32F02A0E8C5DD8A4B8EFF1
:105B40002DF059ECBDF0DE6ADE6A230EDE6E0E0E1D
:105B5000DE6EDE6AE4ECA8F0DE6ADE6A990EDE6EC6
:105B6000210EDE6E0C0EDE6EE4ECA8F0B7EF32F024
:105B7000320E8C5DD8A4CBEF2DF026ECBDF0DE6AA2
:105B8000DE6A030EDE6E340EDE6E020EDE6EE4ECB6
:105B9000A8F0B7EF32F0330E8C5DD8A4F1EF2DF002
:105BA00059ECBDF0DE6ADE6A030EDE6E0A0EDE6EB2
:105BB0000C0EDE6EE4ECA8F0DE6ADE6A290EDE6E04
:105BC000480EDE6E0D0EDE6EE4ECA8F0DE6ADE6AD4
:105BD000330EDE6E0E0EDE6EDE6AE4ECA8F0B7EF7A
:105BE00032F0340E8C5DD8A417EF2EF059ECBDF0D6
:105BF000DE6ADE6A030EDE6E0A0EDE6E0C0EDE6EEE
:105C0000E4ECA8F0DE6ADE6A290EDE6E480EDE6E77
:105C10000D0EDE6EE4ECA8F0DE6ADE6A2F0EDE6E9C
:105C20000C0EDE6EDE6AE4ECA8F0B7EF32F0350E53
:105C30008C5DD8A446EF2EF059ECBDF0DE6ADE6A2A
:105C4000030EDE6E0A0EDE6E0C0EDE6EE4ECA8F0C5
:105C5000DE6ADE6A290EDE6E480EDE6E0D0EDE6E28
:105C6000E4ECA8F0DE6ADE6A030EDE6E070EDE6E7E
:105C7000DE6AE4ECA8F0DE6ADE6A410EDE6E450EF6
:105C8000DE6EDE6AE4ECA8F0B7EF32F0360E8C5D23
:105C9000D8A476EF2EF059ECBDF0DE6ADE6A030E72
:105CA000DE6E0A0EDE6E0C0EDE6EE4ECA8F0DE6A2E
:105CB000DE6A290EDE6E480EDE6E0D0EDE6EE4EC40
:105CC000A8F0DE6ADE6A030EDE6E060EDE6EDE6AA7
:105CD000E4ECA8F0DE6ADE6A190EDE6E440EDE6EBB
:105CE000010EDE6EE4ECA8F0B7EF32F0370E8C5DFB
:105CF000D8A4A5EF2EF059ECBDF0DE6ADE6A030EE3
:105D0000DE6E0A0EDE6E0C0EDE6EE4ECA8F0DE6ACD
:105D1000DE6A290EDE6E480EDE6E0D0EDE6EE4ECDF
:105D2000A8F0DE6ADE6A310EDE6E200EDE6EDE6AFE
:105D3000E4ECA8F0DE6ADE6A030EDE6E470EDE6E6D
:105D4000DE6AE4ECA8F0B7EF32F0380E8C5DD8A430
:105D5000D4EF2EF059ECBDF0DE6ADE6A030EDE6E83
:105D6000060EDE6E0C0EDE6EE4ECA8F0DE6ADE6A75
:105D7000190EDE6E440EDE6E0D0EDE6EE4ECA8F043
:105D8000DE6ADE6A310EDE6E200EDE6EDE6AE4EC66
:105D9000A8F0DE6ADE6A030EDE6E470EDE6EDE6A95
:105DA000E4ECA8F0B7EF32F0390E8C5DD8A403EF25
:105DB0002FF059ECBDF0DE6ADE6A330EDE6E0E0E99
:105DC000DE6EDE6AE4ECA8F0DE6ADE6A650EDE6E88
:105DD000DE6A0C0EDE6EE4ECA8F0DE6ADE6A670EA8
:105DE000DE6E100EDE6E0C0EDE6EE4ECA8F0DE6AE7
:105DF000DE6A690EDE6E210EDE6E0C0EDE6EE4ECE7
:105E0000A8F0B7EF32F03A0E8C5DD8A420EF2FF057
:105E1000DFECBCF0DE6ADE6A030EDE6E340EDE6E90
:105E2000010EDE6EE4ECA8F0DE6ADE6A170EDE6EAE
:105E30002F0EDE6E040EDE6EE4ECA8F0B7EF32F04B
:105E40003C0E8C5DD8A433EF2FF026ECBDF0DE6A5B
:105E5000DE6A140EDE6E200EDE6E010EDE6EE4ECE7
:105E6000A8F0B7EF32F03D0E8C5DD8A446EF2FF0CE
:105E7000DFECBCF0DE6ADE6A140EDE6E200EDE6E33
:105E8000020EDE6EE4ECA8F0B7EF32F03E0E8C5D51
:105E9000D8A489EF2FF059ECBDF0DE6ADE6A8B0ED4
:105EA000DE6E220EDE6EDE6AE4ECA8F0DE6ADE6AEA
:105EB000240EDE6E350EDE6E010EDE6EE4ECA8F012
:105EC000DE6ADE6A8A0EDE6E3C0EDE6EDE6AE4ECB0
:105ED000A8F0DE6ADE6A200EDE6E140EDE6E0C0E98
:105EE000DE6EE4ECA8F0DE6ADE6A240EDE6E270EBB
:105EF000DE6E0D0EDE6EE4ECA8F0DE6ADE6A220EC7
:105F0000DE6E2E0EDE6E0C0EDE6EE4ECA8F0B7EF49
:105F100032F03F0E8C5DD8A4B9EF2FF059ECBDF0F4
:105F2000DE6ADE6A8B0EDE6E220EDE6E0C0EDE6E1A
:105F3000E4ECA8F0DE6ADE6A240EDE6E350EDE6E5C
:105F40000D0EDE6EE4ECA8F0DE6ADE6A8A0EDE6E0E
:105F50003C0EDE6E0C0EDE6EE4ECA8F0DE6ADE6A4D
:105F60000B0EDE6E360EDE6EDE6AE4ECA8F0B7EFE6
:105F700032F0400E8C5DD8A4E9EF2FF059ECBDF063
:105F8000DE6ADE6A0B0EDE6E360EDE6EDE6AE4EC74
:105F9000A8F0DE6ADE6A200EDE6E140EDE6E0C0ED7
:105FA000DE6EE4ECA8F0DE6ADE6A240EDE6E270EFA
:105FB000DE6E0D0EDE6EE4ECA8F0DE6ADE6A220E06
:105FC000DE6E2E0EDE6E0C0EDE6EE4ECA8F0B7EF89
:105FD00032F0460E8C5DD8A4FCEF2FF026ECBDF01D
:105FE000DE6ADE6AA50EDE6E0F0EDE6E010EDE6E5E
:105FF000E4ECA8F0B7EF32F0470E8C5DD8A40FEFB9
:1060000030F0DFECBCF0DE6ADE6A180EDE6E1E0ECB
:10601000DE6E010EDE6EE4ECA8F0B7EF32F0480E53
:106020008C5DD8A46DEF30F0DFECBCF0DE6ADE6A88
:10603000EB0EDE6E2A0EDE6EDE6AE4ECA8F0010ED8
:10604000B95DD8A439EF30F0DE6A0F0EDE6E380E7F
:10605000DE6E040EDE6EC0ECBCF0DE6ADE6A4D0E53
:10606000DE6E3F0EDE6E060EDE6EE4ECA8F06BEF29
:1060700030F0020EB95DD8A453EF30F0DE6A0F0E97
:10608000DE6E380EDE6E040EDE6EC0ECBCF0DE6A34
:10609000DE6A590EDE6E450EDE6E060EDE6EE4EC36
:1060A000A8F06BEF30F0030EB95DD8A46BEF30F0C1
:1060B000DE6A0F0EDE6E380EDE6E040EDE6EC0EC93
:1060C000BCF0DE6ADE6A550EDE6E380EDE6E060E3F
:1060D000DE6EE4ECA8F0B7EF32F0490E8C5DD8A488
:1060E0008AEF30F0DE6ADE6A570EDE6E360EDE6E46
:1060F000010EDE6EE4ECA8F0DE6ADE6A230EDE6ED0
:106100000E0EDE6E030EDE6EE4ECA8F0DFECBCF0EB
:10611000B7EF32F04A0E8C5DD8A4A7EF30F0DFEC79
:10612000BCF0DE6ADE6A550EDE6E380EDE6E010EE3
:10613000DE6EE4ECA8F0DE6ADE6A630EDE6E2C0E24
:10614000DE6E030EDE6EE4ECA8F0B7EF32F04B0E1D
:106150008C5DD8A4BAEF30F0DFECBCF0DE6ADE6A0A
:10616000170EDE6E2F0EDE6E030EDE6EE4ECA8F070
:10617000B7EF32F04C0E8C5DD8A4D7EF30F0DFECE7
:10618000BCF0DE6ADE6A410EDE6E410EDE6E020E8D
:10619000DE6EE4ECA8F0DE6ADE6A110EDE6E180E2A
:1061A000DE6E030EDE6EE4ECA8F0B7EF32F04D0EBB
:1061B0008C5DD8A4EAEF30F0DFECBCF0DE6ADE6A7A
:1061C000160EDE6E250EDE6E010EDE6EE4ECA8F01D
:1061D000B7EF32F0500E8C5DD8A4FDEF30F026EC16
:1061E000BDF0DE6ADE6AED0EDE6E1F0EDE6E010EA3
:1061F000DE6EE4ECA8F0B7EF32F0510E8C5DD8A45F
:1062000019EF31F0DFECBCF0DE6ADE6AE90EDE6E1B
:106210001C0EDE6EDE6AE4ECA8F0DE6ADE6AED0ECD
:10622000DE6E1F0EDE6E040EDE6EE4ECA8F0B7EF3D
:1062300032F0520E8C5DD8A435EF31F0DFECBCF0BB
:10624000DE6ADE6AEB0EDE6E2A0EDE6EDE6AE4ECDD
:10625000A8F0DE6ADE6AED0EDE6E1F0EDE6E040E44
:10626000DE6EE4ECA8F0B7EF32F0530E8C5DD8A4EC
:1062700052EF31F0DFECBCF0DE6ADE6A890EDE6ED2
:10628000200EDE6E010EDE6EE4ECA8F0DE6ADE6A41
:10629000ED0EDE6E1F0EDE6E040EDE6EE4ECA8F078
:1062A000B7EF32F0540E8C5DD8A489EF31F0DFECFB
:1062B000BCF0DE6ADE6AA30EDE6E110EDE6EDE6AF2
:1062C000E4ECA8F0DE6ADE6A080EDE6E130EDE6E07
:1062D000030EDE6EE4ECA8F0010ECF5DD8A47DEFD6
:1062E00031F0DE6ADE6AF50EDE6E390EDE6E060E07
:1062F000DE6EE4ECA8F087EF31F0DE6ADE6AF70EBE
:10630000DE6E390EDE6E060EDE6EE4ECA8F0B7EF40
:1063100032F0550E8C5DD8A4B7EF31F0DFECBCF055
:10632000DE6ADE6A020EDE6E240EDE6E010EDE6EA8
:10633000E4ECA8F0010E865DD8A4ABEF31F0DE6A84
:10634000DE6AF50EDE6E390EDE6E060EDE6EE4ECF3
:10635000A8F0B5EF31F0DE6ADE6AF70EDE6E390EB8
:10636000DE6E060EDE6EE4ECA8F0B7EF32F0560EED
:106370008C5DD8A4D4EF31F0DFECBCF0DE6ADE6ACD
:10638000120EDE6E150EDE6E010EDE6EE4ECA8F06F
:10639000DE6ADE6AED0EDE6E1F0EDE6E040EDE6E4F
:1063A000E4ECA8F0B7EF32F0570E8C5DD8A4F1EF13
:1063B00031F0DFECBCF0DE6ADE6A470EDE6E240EE2
:1063C000DE6E010EDE6EE4ECA8F0DE6ADE6AED0E33
:1063D000DE6E1F0EDE6E040EDE6EE4ECA8F0B7EF8C
:1063E00032F0580E8C5DD8A40EEF32F0DFECBCF02A
:1063F000DE6ADE6A030EDE6E340EDE6E010EDE6EC7
:10640000E4ECA8F0DE6ADE6AED0EDE6E1F0EDE6ED4
:10641000040EDE6EE4ECA8F0B7EF32F05A0E8C5D9D
:10642000D8A45EEF32F0DE6ADE6A1B0EDE6E0D0E61
:10643000DE6E030EDE6EE4ECA8F0DE6ADE6A630E4A
:10644000DE6E190EDE6E0A0EDE6EE4ECA8F0DE6A79
:10645000DE6AD70EDE6E6E0EDE6E090EDE6EE4ECC8
:10646000A8F0DE6ADE6AD90EDE6E6E0EDE6E0B0EF0
:10647000DE6EE4ECA8F0DE6ADE6A4F0EDE6E3F0EE2
:10648000DE6E0E0EDE6EE4ECA8F0DE6ADE6ADF0E73
:10649000DE6E780EDE6E0E0EDE6EE4ECA8F0DE6AC6
:1064A000DE6ADB0EDE6E6D0EDE6E0E0EDE6EE4EC70
:1064B000A8F0C80E54EC01F0B7EF32F05B0E8C5D23
:1064C000D8A4B5EF32F0DE6ADE6A1B0EDE6E0D0E6A
:1064D000DE6E030EDE6EE4ECA8F0DE6ADE6AE10E2C
:1064E000DE6E3F0EDE6E0A0EDE6EE4ECA8F0DE6AB3
:1064F000DE6AD70EDE6E6E0EDE6E080EDE6EE4EC29
:10650000A8F0DE6ADE6AD90EDE6E6E0EDE6E0C0E4E
:10651000DE6EE4ECA8F0DE6ADE6ADF0EDE6E800E70
:10652000DE6E0A0EDE6EE4ECA8F0DE6ADE6ADB0EDA
:10653000DE6E650EDE6E0A0EDE6EE4ECA8F0DE6A3C
:10654000DE6A4F0EDE6E3F0EDE6E0E0EDE6EE4EC89
:10655000A8F0DE6ADE6ADD0EDE6E650EDE6E0E0E01
:10656000DE6EE4ECA8F0B7EF32F0B8EF32F01200D4
:106570000101389F00018B83DDECCEF0010E246E0B
:10658000F40E55EC01F0206A8CC01FF0000E75EC83
:1065900001F00B6E0B52D8B4D2EF32F08CC08DF0FC
:1065A000DDEF32F0280E8C5DD8A4DBEF32F08CC02A
:1065B0008DF0DDEF32F00B0E8D6FA3EC2BF00B0E98
:1065C00008012A6FDC0E296F2AC8D7FF29C8D6FF19
:1065D000F2940901F86BF76B010E246EF40E55EC82
:1065E00001F00001820E026E800E096E306A540EB8
:1065F0002F6E066A0B0E056E4EEC00F0D8A00BEF66
:1066000033F00901F96F6C0EF95D0001D8A40BEFAE
:1066100033F0AFEF5CF0F2A41BEF33F00B0E080188
:106620002A6FDC0E296F2AC8D7FF29C8D6FFF2943B
:106630000901F74BF82B0001030E0901F85D000179
:10664000D8A02FEF33F0D8A42DEF33F0850E090139
:10665000F75D0001D8A02FEF33F02EECA4F001017C
:10666000389D0001986B80A03BEF33F00101388D1D
:10667000030E0001986F81A243EF33F00101388DC2
:10668000040E0001986F80AA4BEF33F00101388DA2
:10669000010E0001986F82A253EF33F00101388D93
:1066A000020E0001986F82A05BEF33F00101388D7C
:1066B000050E0001986FD896010138BDD8860001FB
:1066C000D8B601EF34F00901F46B0001100E090196
:1066D000F45D0001D8B078EF33F0F36A09EEE4F02E
:1066E0000901F451F3CFEBFFF42B0001D8A4EDD74F
:1066F000810E026E010E096E400E306E200E2F6E5E
:10670000066A7B0E056E0B6AD8804EEC00F0D8A0AE
:1067100068D709EEE4F00B5023C0EBFF0B2A0B50B7
:106720001008F2E10901F46B00010D0E0901F45D9E
:106730000001D8B001EF34F009EEE4F00901F451A2
:10674000EB500B6E030E0B5C0001D8A4FCEF33F092
:10675000030E0901F42509EEE4F0EB50F66F206A10
:10676000F6C91FF0080E24EC02F0F56F800EF55DFF
:106770000001D8A4C3EF33F0010E986F0101388FE8
:106780000001FCEF33F0400E0901F55D0001D8A4D3
:10679000D1EF33F0020E986F0101388F0001FCEF4A
:1067A00033F0200E0901F55D0001D8A4DFEF33F0CE
:1067B000030E986F0101388F0001FCEF33F0100ECB
:1067C0000901F55D0001D8A4EDEF33F0040E986FD8
:1067D0000101388F0001FCEF33F0080E0901F55D6F
:1067E0000001D8A4FBEF33F0050E986F0101388F3C
:1067F0000001FCEF33F0986B0901F42B0001D8A4E1
:1068000093D7010E985DD8A44AEF34F05B0E8C5DEF
:10681000D8A40DEF34F02EEFA4F0420EF66E680E01
:10682000F76E2368232A23500B08D8A02DEF34F0ED
:106830000900F55009008C5DF5E123C094F02DEFBF
:1068400034F0630C0C0C150C160C1F0C200C210CD6
:10685000220C250C290C4A0C4C0C3A0E8C5DD8B03D
:1068600034EF34F08CC02FF8280E8C5DD8A43BEFA9
:1068700034F022EF35F0206A8CC01FF0000E75EC6A
:1068800001F00B6E0B52D8B448EF34F022EF35F024
:106890001BEF35F0020E985DD8A46EEF34F08CC07B
:1068A0001FF00A0EE8EC01F08C6F8C510A0DF3CF4B
:1068B00031F0F4CF32F00A0E31248C6F280E8C5D4B
:1068C000D8A465EF34F0320E8C6F640E8C5DD8A4C2
:1068D0006CEF34F00A0E8C6F1BEF35F0030E985DF1
:1068E000D8A491EF34F08CC01FF00A0EE8EC01F050
:1068F0008C6F8C510A0DF3CF31F0F4CF32F00A0EC9
:10690000315C8C6F280E8C5DD8A489EF34F01E0E9C
:106910008C6F8C53D8A48FEF34F05A0E8C6F1BEF12
:1069200035F0040E985DD8A4D1EF34F08C2B0E0E08
:106930008C5DD8A49EEF34F00A0E8C6F180E8C5D1F
:10694000D8A4A5EF34F0140E8C6F2B0E8C5DD8A458
:10695000ACEF34F01E0E8C6F3B0E8C5DD8A4B3EF01
:1069600034F0320E8C6F410E8C5DD8A4BAEF34F047
:106970003C0E8C6F4E0E8C5DD8A4C1EF34F0460EE9
:106980008C6F590E8C5DD8A4C8EF34F0500E8C6F0C
:106990005C0E8C5DD8A4CFEF34F05A0E8C6F1BEFD9
:1069A00035F0050E985DD8A411EF35F08C07090E6F
:1069B0008C5DD8A4DEEF34F00D0E8C6F130E8C5D61
:1069C000D8A4E5EF34F0170E8C6F1D0E8C5DD8A4A3
:1069D000ECEF34F02A0E8C6F310E8C5DD8A4F3EFFF
:1069E00034F03A0E8C6F3B0E8C5DD8A4FAEF34F085
:1069F000400E8C6F450E8C5DD8A401EF35F04D0E26
:106A00008C6F4F0E8C5DD8A408EF35F0580E8C6F4C
:106A1000590E8C5DD8A40FEF35F05B0E8C6F1BEF19
:106A200035F09853D8A419EF35F0F1EF32F01BEFA1
:106A300035F0F1EF32F0DDECCEF0A3EC2BF0F1EF1E
:106A400032F012003A0E8C5DD8A429EF35F098EFA1
:106A500035F03E0E8C5DD8A430EF35F098EF35F070
:106A60003F0E8C5DD8A437EF35F098EF35F0400E2F
:106A70008C5DD8A43EEF35F098EF35F0470E8C5D75
:106A8000D8A445EF35F098EF35F04A0E8C5DD8A4C8
:106A90004CEF35F098EF35F04D0E8C5DD8A453EFE8
:106AA00035F098EF35F0510E8C5DD8A45AEF35F0E3
:106AB00098EF35F0520E8C5DD8A461EF35F098EF69
:106AC00035F0530E8C5DD8A468EF35F098EF35F0B3
:106AD000540E8C5DD8A46FEF35F098EF35F0550E5D
:106AE0008C5DD8A476EF35F098EF35F0560E8C5DBE
:106AF000D8A47DEF35F098EF35F0570E8C5DD8A413
:106B000084EF35F098EF35F0580E8C5DD8A48BEFFC
:106B100035F098EF35F05B0E8C5DD8A492EF35F030
:106B200098EF35F0AAEC0AF0010EDE6E13EC48F097
:106B3000856BD8968BA3D886D8B6A1EF35F0DDEC5F
:106B4000CEF00901FA933A0E00018C5DD8A4ABEFA8
:106B500035F041EF36F03D0E8C5DD8A4B2EF35F044
:106B600041EF36F03E0E8C5DD8A4B9EF35F041EF21
:106B700036F03F0E8C5DD8A4C0EF35F041EF36F013
:106B8000400E8C5DD8A4C7EF35F041EF36F0430ED0
:106B90008C5DD8A4CEEF35F041EF36F0470E8C5D1A
:106BA000D8A4D5EF35F041EF36F0480E8C5DD8A46F
:106BB000DCEF35F041EF36F0490E8C5DD8A4E3EF01
:106BC00035F041EF36F04A0E8C5DD8A4EAEF35F08F
:106BD00041EF36F04B0E8C5DD8A4F1EF35F041EF6C
:106BE00036F04C0E8C5DD8A4F8EF35F041EF36F05E
:106BF0004D0E8C5DD8A4FFEF35F041EF36F0510E0D
:106C00008C5DD8A406EF36F041EF36F0520E8C5D65
:106C1000D8A40DEF36F041EF36F0530E8C5DD8A4BA
:106C200014EF36F041EF36F0540E8C5DD8A41BEF14
:106C300036F041EF36F0550E8C5DD8A422EF36F0D9
:106C400041EF36F0560E8C5DD8A429EF36F041EFB7
:106C500036F0570E8C5DD8A430EF36F041EF36F0A9
:106C6000580E8C5DD8A437EF36F041EF36F05B0E4E
:106C70008C5DD8A43EEF36F040EF36F00901FA8380
:106C80000001D8960901FAA3D8860001D8B6F3EF1F
:106C900036F08E53D8A451EF36F08CC08EF05DEFF5
:106CA00036F08F53D8A45DEF36F08E518C5DD8B49A
:106CB0005DEF36F08CC08FF08B85010E905DD8A40F
:106CC000F3EF36F0D8968BA5D886D8B6F3EF36F02A
:106CD0008CC091F004EE1EF0D89001012335E92616
:106CE000000EEA22EECF0BF0EFCF0CF00001955131
:106CF0000B5C96510C58D8A097EF36F004EE1EF0BE
:106D0000D89001012335E926000EEA22EECF0BF0E0
:106D1000EFCF0CF0000195510B5C0A013C6F0001B4
:106D200096510C580A013D6F0001ADEF36F004EEAC
:106D30001EF0D89001012335E926000EEA22EECF9D
:106D40000BF0EFCF0CF00B500001955D0A013C6F8A
:106D50000C50000196590A013D6F00010A013D5394
:106D60000001D8A4BDEF36F05B0E0A013C5D0001C6
:106D7000D8B0BDEF36F08EC08CF0010E0A013D5D3B
:106D80000001D8A0D0EF36F0D8A4CEEF36F00E0E2A
:106D90000A013C5D0001D8A0D0EF36F08EC08CF027
:106DA0000A013D530001D8A4DDEF36F05B0E0A0165
:106DB0003C5D0001D8A0E9EF36F0010E0A013D5D0F
:106DC0000E0ED8B43C5D0001D8B0E9EF36F08FC0AC
:106DD0008CF08C51915DD8B4F1EF36F08B83DDEC03
:106DE000CEF0F3EF36F00B0E8C5DD8A4ECEF37F05D
:106DF000DE6AFCEC8EF0010E985DD8A408EF37F047
:106E0000D8968BB3D886D8B608EF37F0B8EF32F003
:106E1000050E985DD8A41BEF37F0D8968BB3D886B3
:106E2000D8B61BEF37F08DC03BFA8CC08DF03BCA53
:106E30008CF08B8307D6040E985DD8A422EF37F030
:106E40005AEC68F0D8968BA3D886D8B634EF37F0D2
:106E50000901FA91DE6ADE6A270EDE6E180EDE6E1A
:106E6000DE6A0001E4ECA8F021ECBFF003EE1EF0B6
:106E7000D89001012335E926000EEA22EECF0BF06F
:106E8000EFCF0CF00BC0DEFF0CC0DEFF00010AEC00
:106E90007AF0FF0EDB50DD520901FA81E8A0FA9189
:106EA000D896FAA1D8860001D8B6A0EF37F0010134
:106EB00023530001D8B483EF37F003EE1EF0D890CF
:106EC00001012335E926000EEA22EECF0BF0EFCFC9
:106ED0000CF00BC0DEFF0CC0DEFF23050F6E03EECF
:106EE0001EF0D8900F34E926000EEA22EECF0BF008
:106EF000EFCF0CF00BC0DEFF0CC0DEFF00010EEC8C
:106F00007BF09EEF37F003EE1EF0D89001012335A1
:106F1000E926000EEA22EECF0BF0EFCF0CF00BC00B
:106F2000DEFF0CC0DEFF1CC40BF01DC40CF00BC058
:106F3000DEFF0CC0DEFF00010EEC7BF0E7EF37F068
:106F4000010123530001D8B4CCEF37F003EE1EF05B
:106F5000D89001012335E926000EEA22EECF0BF08E
:106F6000EFCF0CF00BC0DEFF0CC0DEFF23050F6E71
:106F700003EE1EF0D8900F34E926000EEA22EECF81
:106F80000BF0EFCF0CF00BC0DEFF0CC0DEFF0001FA
:106F9000D0EC7AF0E7EF37F003EE1EF0D890010165
:106FA0002335E926000EEA22EECF0BF0EFCF0CF0EE
:106FB0000BC0DEFF0CC0DEFF1CC40BF01DC40CF0C8
:106FC0000BC0DEFF0CC0DEFF0001D0EC7AF08B932B
:106FD00022EF35F011EF48F00C0E8C5DD8A4FEEFD7
:106FE00038F0DE6AFCEC8EF0010E985DD8A403EF59
:106FF00038F0D8968BB3D886D8B601EF38F0B8EF12
:1070000032F019EF38F0020E985DD8A40FEF38F087
:10701000DDECCEF08B83BDEFA2F019EF38F0030E5C
:10702000985DD8A419EF38F0DDECCEF08B83BDEF7E
:10703000A2F0040E985DD8A420EF38F05AEC68F066
:10704000050E985DD8A434EF38F0D8968BB3D88667
:10705000D8B634EF38F08DC03BFA8CC08DF03BCA07
:107060008CF08B8322EF35F0D8968BA3D886D8B6D8
:1070700046EF38F00901FA91DE6ADE6A250EDE6E0F
:10708000180EDE6EDE6A0001E4ECA8F021ECBFF021
:1070900002EE1EF0D89001012335E926000EEA2207
:1070A000EECF0BF0EFCF0CF00BC0DEFF0CC0DEFF1D
:1070B00000010AEC7AF0FF0EDB50DD520901FA8183
:1070C000E8A0FA91D896FAA1D8860001D8B6B2EF16
:1070D00038F0010123530001D8B495EF38F002EEE7
:1070E0001EF0D89001012335E926000EEA22EECFEA
:1070F0000BF0EFCF0CF00BC0DEFF0CC0DEFF230562
:107100000F6E02EE1EF0D8900F34E926000EEA2230
:10711000EECF0BF0EFCF0CF00BC0DEFF0CC0DEFFAC
:1071200000010EEC7BF0B0EF38F002EE1EF0D890CC
:1071300001012335E926000EEA22EECF0BF0EFCF56
:107140000CF00BC0DEFF0CC0DEFF1CC30BF01DC338
:107150000CF00BC0DEFF0CC0DEFF00010EEC7BF07C
:10716000F9EF38F0010123530001D8B4DEEF38F015
:1071700002EE1EF0D89001012335E926000EEA2226
:10718000EECF0BF0EFCF0CF00BC0DEFF0CC0DEFF3C
:1071900023050F6E02EE1EF0D8900F34E926000E84
:1071A000EA22EECF0BF0EFCF0CF00BC0DEFF0CC0ED
:1071B000DEFF0001D0EC7AF0F9EF38F002EE1EF0BD
:1071C000D89001012335E926000EEA22EECF0BF01C
:1071D000EFCF0CF00BC0DEFF0CC0DEFF1CC30BF0CA
:1071E0001DC30CF00BC0DEFF0CC0DEFF0001D0ECB5
:1071F0007AF08B9322EF35F011EF48F00D0E8C5D95
:10720000D8A465EF39F0DE6AFCEC8EF0010E985DD3
:10721000D8A413EF39F0D8968BB3D886D8B613EF2D
:1072200039F0B8EF32F0050E985DD8A427EF39F0A9
:10723000D8968BB3D886D8B627EF39F08DC03BFAF5
:107240008CC08DF03BCA8CF08B8322EF35F0040E9E
:10725000985DD8A42EEF39F05AEC68F0D8968BA33D
:10726000D886D8B648EF39F0DE6ADE6A230EDE6EC5
:107270000E0EDE6E010EDE6EE4ECA8F0DE6ADE6A53
:107280003D0EDE6E860EDE6E060EDE6EE4ECA8F0BF
:1072900004EE1EF0D89001012335E926000EEA2203
:1072A000EECF0BF0EFCF0CF00BC0DEFF0CC0DEFF1B
:1072B000DE6A010EDE6E0A0EDE6E00014CEC7BF023
:1072C0008B9322EF35F011EF48F0150E8C5DD8A4AA
:1072D000FAEF39F0DE6AFCEC8EF0010E985DD8A46E
:1072E0007CEF39F0D8968BB3D886D8B67AEF39F0E0
:1072F000B8EF32F092EF39F0020E985DD8A488EF23
:1073000039F0DDECCEF08B83BDEFA2F092EF39F0D7
:10731000030E985DD8A492EF39F0DDECCEF08B83AC
:10732000BDEFA2F0040E985DD8A499EF39F05AECA5
:1073300068F0050E985DD8A4ADEF39F0D8968BB300
:10734000D886D8B6ADEF39F08DC03BFA8CC08DF041
:107350003BCA8CF08B8322EF35F0D8968BA3D8866E
:10736000D8B6C5EF39F0DE6ADE6ACD0EDE6EDE6AB3
:10737000DE6AE4ECA8F0DE6ADE6A3F0EDE6E860EA0
:10738000DE6E090EDE6EE4ECA8F002EE1EF0D89080
:1073900001012335E926000EEA22EECF0BF0EFCFF4
:1073A0000CF00BC0DEFF0CC0DEFF010EDE6EDE6AED
:1073B000140EDE6E00014CEC7BF004EE1EF0D89053
:1073C00001012335E926000EEA22EECF0BF0EFCFC4
:1073D0000CF00BC0DEFF0CC0DEFFDE6A010EDE6EBD
:1073E0000A0EDE6E00014CEC7BF08B9322EF35F041
:1073F00011EF48F0160E8C5DD8A48FEF3AF0DE6ADC
:10740000FCEC8EF0010E985DD8A411EF3AF0D896FE
:107410008BB3D886D8B60FEF3AF0B8EF32F027EF3B
:107420003AF0020E985DD8A41DEF3AF0DDECCEF0F4
:107430008B83BDEFA2F027EF3AF0030E985DD8A43E
:1074400027EF3AF0DDECCEF08B83BDEFA2F0040E17
:10745000985DD8A42EEF3AF05AEC68F0050E985DCE
:10746000D8A442EF3AF0D8968BB3D886D8B642EF7C
:107470003AF08DC03BFA8CC08DF03BCA8CF08B8308
:1074800022EF35F0D8968BA3D886D8B65BEF3AF0CA
:10749000DE6ADE6AD10EDE6E050EDE6EDE6AE4ECBA
:1074A000A8F0DE6ADE6ACF0EDE6E900EDE6E090E8A
:1074B000DE6EE4ECA8F003EE1EF0D8900101233557
:1074C000E926000EEA22EECF0BF0EFCF0CF00BC056
:1074D000DEFF0CC0DEFF010EDE6EDE6A140EDE6E15
:1074E00000014CEC7BF002EE1EF0D8900101233538
:1074F000E926000EEA22EECF0BF0EFCF0CF00BC026
:10750000DEFF0CC0DEFFDE6ADE6A0C0EDE6E0001FE
:107510004CEC7BF08B9322EF35F011EF48F0170E17
:107520008C5DD8A40DEF3BF0DE6AFCEC8EF0010E12
:10753000985DD8A4A4EF3AF0D8968BB3D886D8B685
:10754000A4EF3AF0B8EF32F0050E985DD8A4B8EF8A
:107550003AF0D8968BB3D886D8B6B8EF3AF08DC04B
:107560003BFA8CC08DF03BCA8CF08B8322EF35F058
:10757000040E985DD8A4BFEF3AF05AEC68F0D896A4
:107580008BA3D886D8B6D8EF3AF0DE6ADE6AD10E81
:10759000DE6E050EDE6EDE6AE4ECA8F0DE6ADE6A00
:1075A0003F0EDE6E860EDE6E090EDE6EE4ECA8F097
:1075B00003EE1EF0D89001012335E926000EEA22E1
:1075C000EECF0BF0EFCF0CF00BC0DEFF0CC0DEFFF8
:1075D000010EDE6EDE6A140EDE6E00014CEC7BF0F6
:1075E00004EE1EF0D89001012335E926000EEA22B0
:1075F000EECF0BF0EFCF0CF00BC0DEFF0CC0DEFFC8
:10760000DE6A010EDE6E0A0EDE6E00014CEC7BF0CF
:107610008B9322EF35F011EF48F01F0E8C5DD8A44C
:107620008EEF3BF0DE6AFCEC8EF0010E985DD8A484
:1076300024EF3BF0D8968BB3D886D8B622EF3BF038
:10764000B8EF32F03AEF3BF0020E985DD8A430EF7D
:107650003BF0DDECCEF08B83BDEFA2F03AEF3BF0D8
:10766000030E985DD8A43AEF3BF0DDECCEF08B83AF
:10767000BDEFA2F0040E985DD8A441EF3BF05AECA8
:1076800068F0050E985DD8A455EF3BF0D8968BB303
:10769000D886D8B655EF3BF08DC03BFA8CC08DF044
:1076A0003BCA8CF08B8322EF35F0D8968BA3D8861B
:1076B000D8B66DEF3BF0DE6ADE6ACD0EDE6EDE6AB6
:1076C000DE6AE4ECA8F0DE6ADE6ACF0EDE6E900EB3
:1076D000DE6E080EDE6EE4ECA8F002EE1EF0D8902E
:1076E00001012335E926000EEA22EECF0BF0EFCFA1
:1076F0000CF00BC0DEFF0CC0DEFF010EDE6EDE6A9A
:10770000140EDE6E00014CEC7BF0020EDE6E8AEC95
:10771000C0F08B9322EF35F011EF48F0200E8C5D16
:10772000D8A40FEF3CF0DE6AFCEC8EF0010E985D01
:10773000D8A4A5EF3BF0D8968BB3D886D8B6A3EFE4
:107740003BF0B8EF32F0BBEF3BF0020E985DD8A4EF
:10775000B1EF3BF0DDECCEF08B83BDEFA2F0BBEFE1
:107760003BF0030E985DD8A4BBEF3BF0DDECCEF010
:107770008B83BDEFA2F0040E985DD8A4C2EF3BF05E
:107780005AEC68F0050E985DD8A4D6EF3BF0D89679
:107790008BB3D886D8B6D6EF3BF08DC03BFA8CC001
:1077A0008DF03BCA8CF08B8322EF35F0D8968BA3FB
:1077B000D886D8B6EEEF3BF0DE6ADE6ACD0EDE6E1E
:1077C000DE6ADE6AE4ECA8F0DE6ADE6AD30EDE6E04
:1077D0008E0EDE6E090EDE6EE4ECA8F002EE1EF0F8
:1077E000D89001012335E926000EEA22EECF0BF0F6
:1077F000EFCF0CF00BC0DEFF0CC0DEFF010EDE6E23
:10780000DE6A140EDE6E00014CEC7BF0010EDE6EC3
:107810008AECC0F08B9322EF35F011EF48F0210E87
:107820008C5DD8A490EF3CF0DE6AFCEC8EF0010E8B
:10783000985DD8A426EF3CF0D8968BB3D886D8B6FE
:1078400024EF3CF0B8EF32F03CEF3CF0020E985DD4
:10785000D8A432EF3CF0DDECCEF08B83BDEFA2F08C
:107860003CEF3CF0030E985DD8A43CEF3CF0DDEC1F
:10787000CEF08B83BDEFA2F0040E985DD8A443EF49
:107880003CF05AEC68F0050E985DD8A457EF3CF038
:10789000D8968BB3D886D8B657EF3CF08DC03BFA5C
:1078A0008CC08DF03BCA8CF08B8322EF35F0D896DC
:1078B0008BA3D886D8B66FEF3CF0DE6ADE6ACD0EB9
:1078C000DE6EDE6ADE6AE4ECA8F0DE6ADE6A3F0E97
:1078D000DE6E860EDE6E090EDE6EE4ECA8F002EEC1
:1078E0001EF0D89001012335E926000EEA22EECFE2
:1078F0000BF0EFCF0CF00BC0DEFF0CC0DEFF010E73
:10790000DE6EDE6A140EDE6E00014CEC7BF0030EC0
:10791000DE6E8AECC0F08B9322EF35F011EF48F069
:10792000220E8C5DD8A41DEF3DF0DE6AFCEC8EF0DB
:10793000010E985DD8A4A7EF3CF0D8968BB3D886FB
:10794000D8B6A5EF3CF0B8EF32F0D2EF3CF0020E23
:10795000985DD8A4B3EF3CF0DDECCEF08B83BDEFA7
:10796000A2F0D2EF3CF0030E985DD8A4BFEF3CF03C
:10797000DDECCEF08B83BDEFA2F0D2EF3CF0040E35
:10798000985DD8A4D1EF3CF08B8104EE1EF0D89026
:1079900001012335E926000EEA22EECF89F0EFCF70
:1079A0008AF00001050E985DD8A4E6EF3CF0D89669
:1079B0008BB3D886D8B6E6EF3CF08DC03BFA8CC0CE
:1079C0008DF03BCA8CF08B8322EF35F0D8968BA3D9
:1079D000D886D8B6FEEF3CF0DE6ADE6ACD0EDE6EEB
:1079E000DE6ADE6AE4ECA8F0DE6ADE6A490EDE6E6C
:1079F000640EDE6E0E0EDE6EE4ECA8F002EE1EF0FB
:107A0000D89001012335E926000EEA22EECF0BF0D3
:107A1000EFCF0CF00BC0DEFF0CC0DEFF010EDE6E00
:107A2000DE6A140EDE6E00014CEC7BF02FEC6CF085
:107A30008B9322EF35F011EF48F0230E8C5DD8A424
:107A400087EF3DF0DE6AFCEC8EF0010E985DD8A465
:107A500032EF3DF0D8968BB3D886D8B632EF3DF0F2
:107A6000B8EF32F0050E985DD8A446EF3DF0D896F9
:107A70008BB3D886D8B646EF3DF08DC03BFA8CC0AC
:107A80008DF03BCA8CF08B8322EF35F0040E985DAD
:107A9000D8A44DEF3DF05AEC68F0D8968BA3D88669
:107AA000D8B666EF3DF0DE6ADE6AD10EDE6E050EF8
:107AB000DE6EDE6AE4ECA8F0DE6ADE6AD30EDE6E0D
:107AC0008E0EDE6E090EDE6EE4ECA8F003EE1EF004
:107AD000D89001012335E926000EEA22EECF0BF003
:107AE000EFCF0CF00BC0DEFF0CC0DEFF010EDE6E30
:107AF000DE6A140EDE6E00014CEC7BF0010EDE6ED1
:107B00008AECC0F08B9322EF35F011EF48F0240E91
:107B10008C5DD8A4F1EF3DF0DE6AFCEC8EF0010E36
:107B2000985DD8A49CEF3DF0D8968BB3D886D8B694
:107B30009CEF3DF0B8EF32F0050E985DD8A4B0EFA1
:107B40003DF0D8968BB3D886D8B6B0EF3DF08DC057
:107B50003BFA8CC08DF03BCA8CF08B8322EF35F062
:107B6000040E985DD8A4B7EF3DF05AEC68F0D896B3
:107B70008BA3D886D8B6D0EF3DF0DE6ADE6AD10E90
:107B8000DE6E050EDE6EDE6AE4ECA8F0DE6ADE6A0A
:107B90003F0EDE6E860EDE6E090EDE6EE4ECA8F0A1
:107BA00003EE1EF0D89001012335E926000EEA22EB
:107BB000EECF0BF0EFCF0CF00BC0DEFF0CC0DEFF02
:107BC000010EDE6EDE6A140EDE6E00014CEC7BF000
:107BD000030EDE6E8AECC0F08B9322EF35F011EFCE
:107BE00048F0250E8C5DD8A473EF3EF0DE6AFCEC05
:107BF0008EF0010E985DD8A408EF3EF0D8968BB3B6
:107C0000D886D8B606EF3EF0B8EF32F01EEF3EF061
:107C1000020E985DD8A414EF3EF0DDECCEF08B831D
:107C2000BDEFA2F01EEF3EF0030E985DD8A41EEF4C
:107C30003EF0DDECCEF08B83BDEFA2F0040E985D3C
:107C4000D8A425EF3EF05AEC68F0050E985DD8A454
:107C500039EF3EF0D8968BB3D886D8B639EF3EF0E0
:107C60008DC03BFA8CC08DF03BCA8CF08B8322EF29
:107C700035F0D8968BA3D886D8B652EF3EF0DE6AA0
:107C8000DE6AD10EDE6E050EDE6EDE6AE4ECA8F072
:107C9000DE6ADE6ACF0EDE6E900EDE6E080EDE6EDF
:107CA000E4ECA8F003EE1EF0D89001012335E9269C
:107CB000000EEA22EECF0BF0EFCF0CF00BC0DEFF90
:107CC0000CC0DEFF010EDE6EDE6A140EDE6E0001F9
:107CD0004CEC7BF0020EDE6E8AECC0F08B9322EF50
:107CE00035F011EF48F0260E8C5DD8A4E7EF3EF09A
:107CF000DE6AFCEC8EF0010E985DD8A488EF3EF0B1
:107D0000D8968BB3D886D8B688EF3EF0B8EF32F06D
:107D1000040E985DD8A49AEF3EF08B8104EE1EF01D
:107D2000D89001012335E926000EEA22EECF89F032
:107D3000EFCF8AF00001050E985DD8A4AFEF3EF0BA
:107D4000D8968BB3D886D8B6AFEF3EF08DC03BFA4D
:107D50008CC08DF03BCA8CF08B8322EF35F0D89627
:107D60008BA3D886D8B6C8EF3EF0DE6ADE6AD10EA5
:107D7000DE6E050EDE6EDE6AE4ECA8F0DE6ADE6A18
:107D8000490EDE6E640EDE6E0E0EDE6EE4ECA8F0C2
:107D900003EE1EF0D89001012335E926000EEA22F9
:107DA000EECF0BF0EFCF0CF00BC0DEFF0CC0DEFF10
:107DB000010EDE6EDE6A140EDE6E00014CEC7BF00E
:107DC0002FEC6CF08B9322EF35F011EF48F0270E7B
:107DD0008C5DD8A452EF3FF0DE6AFCEC8EF0010E11
:107DE000985DD8A4FCEF3EF0D8968BB3D886D8B671
:107DF000FCEF3EF0B8EF32F0050E985DD8A410EF1E
:107E00003FF0D8968BB3D886D8B610EF3FF08DC030
:107E10003BFA8CC08DF03BCA8CF08B8322EF35F09F
:107E2000040E985DD8A417EF3FF05AEC68F0D8968E
:107E30008BA3D886D8B630EF3FF0DE6ADE6A3D0EFF
:107E4000DE6E860EDE6EDE6AE4ECA8F0DE6ADE6AC6
:107E50003F0EDE6E860EDE6E090EDE6EE4ECA8F0DE
:107E600004EE1EF0D89001012335E926000EEA2227
:107E7000EECF0BF0EFCF0CF00BC0DEFF0CC0DEFF3F
:107E8000010EDE6E010EDE6E0A0EDE6E00014CEC9F
:107E90007BF0030EDE6E8AECC0F08B9322EF35F0A0
:107EA00011EF48F0280E8C5DD8A4BDEF3FF0DE6ADC
:107EB000FCEC8EF0010E985DD8A467EF3FF0D896E9
:107EC0008BB3D886D8B667EF3FF0B8EF32F0050E27
:107ED000985DD8A47BEF3FF0D8968BB3D886D8B600
:107EE0007BEF3FF08DC03BFA8CC08DF03BCA8CF02D
:107EF0008B8322EF35F0040E985DD8A482EF3FF01B
:107F00005AEC68F0D8968BA3D886D8B69BEF3FF092
:107F1000DE6ADE6A3D0EDE6E860EDE6EDE6AE4EC42
:107F2000A8F0DE6ADE6AD30EDE6E8E0EDE6E090EFD
:107F3000DE6EE4ECA8F004EE1EF0D89001012335CB
:107F4000E926000EEA22EECF0BF0EFCF0CF00BC0CB
:107F5000DEFF0CC0DEFF010EDE6E010EDE6E0A0ECD
:107F6000DE6E00014CEC7BF0010EDE6E8AECC0F0A0
:107F70008B9322EF35F011EF48F0290E8C5DD8A4D9
:107F800040EF40F0DE6AFCEC8EF0010E985DD8A464
:107F9000D4EF3FF0D8968BB3D886D8B6D2EF3FF067
:107FA000B8EF32F0EAEF3FF0020E985DD8A4E0EFB0
:107FB0003FF0DDECCEF08B83BDEFA2F0EAEF3FF0B7
:107FC000030E985DD8A4EAEF3FF0DDECCEF08B8392
:107FD000BDEFA2F0040E985DD8A4F1EF3FF05AEC8B
:107FE00068F0050E985DD8A405EF40F0D8968BB3E5
:107FF000D886D8B605EF40F08DC03BFA8CC08DF026
:108000003BCA8CF08B8322EF35F0D8968BA3D886B1
:10801000D8B61EEF40F0DE6ADE6A3D0EDE6E860EDA
:10802000DE6EDE6AE4ECA8F0DE6ADE6ACF0EDE6E9B
:10803000900EDE6E080EDE6EE4ECA8F004EE1EF08C
:10804000D89001012335E926000EEA22EECF0BF08D
:10805000EFCF0CF00BC0DEFF0CC0DEFF010EDE6EBA
:10806000010EDE6E0A0EDE6E00014CEC7BF0020E9D
:10807000DE6E8AECC0F08B9322EF35F011EF48F002
:108080002A0E8C5DD8A4B5EF40F0DE6AFCEC8EF0D1
:10809000010E985DD8A455EF40F0D8968BB3D886E2
:1080A000D8B655EF40F0B8EF32F0040E985DD8A482
:1080B00067EF40F08B8104EE1EF0D890010123356C
:1080C000E926000EEA22EECF89F0EFCF8AF0000118
:1080D000050E985DD8A47CEF40F0D8968BB3D88677
:1080E000D8B67CEF40F08DC03BFA8CC08DF03BCA17
:1080F0008CF08B8322EF35F0D8968BA3D886D8B638
:1081000095EF40F0DE6ADE6A3D0EDE6E860EDE6EB4
:10811000DE6AE4ECA8F0DE6ADE6A490EDE6E640E0A
:10812000DE6E0E0EDE6EE4ECA8F004EE1EF0D890CB
:1081300001012335E926000EEA22EECF0BF0EFCF46
:108140000CF00BC0DEFF0CC0DEFF010EDE6E010E78
:10815000DE6E0A0EDE6E00014CEC7BF02FEC6CF054
:108160008B9322EF35F011EF48F0330E8C5DD8A4DD
:1081700048EF41F0DE6AFCEC8EF0010E985DD8A469
:10818000CCEF40F0D8968BB3D886D8B6CAEF40F083
:10819000B8EF32F0F8EF40F0020E985DD8A4D8EFB7
:1081A00040F0DDECCEF08B831BEFA2F0F8EF40F057
:1081B000030E985DD8A4E4EF40F0DDECCEF08B83A5
:1081C0001BEFA2F0F8EF40F0050E985DD8A4F8EF91
:1081D00040F0D8968BB3D886D8B6F8EF40F08DC073
:1081E0003BFA8CC08DF03BCA8CF08B8322EF35F0CC
:1081F000040E985DD8A4FFEF40F05AEC68F0D896D2
:108200008BA3D886D8B63FEF41F0DE6ADE6A3D0E1A
:10821000DE6E860EDE6EDE6AE4ECA8F0DE6ADE6AF2
:108220003D0EDE6E7D0EDE6E090EDE6EE4ECA8F015
:10823000DE6ADE6A430EDE6E8B0EDE6E090EDE6EC9
:10824000E4ECA8F0010E0101465D0001D8A435EF71
:1082500041F0DE6ADE6A6D0EDE6E7D0EDE6E0B0EA6
:10826000DE6EE4ECA8F03FEF41F0DE6ADE6A6B0EF2
:10827000DE6E7D0EDE6E0B0EDE6EE4ECA8F0330ECD
:10828000DE6E0CEC74F08B9322EF35F011EF48F0BA
:10829000340E8C5DD8A4DAEF41F0DE6AFCEC8EF08F
:1082A000010E985DD8A45FEF41F0D8968BB3D886C5
:1082B000D8B65DEF41F0B8EF32F08BEF41F0020E2F
:1082C000985DD8A46BEF41F0DDECCEF08B831BEF13
:1082D000A2F08BEF41F0030E985DD8A477EF41F048
:1082E000DDECCEF08B831BEFA2F08BEF41F0050E9F
:1082F000985DD8A48BEF41F0D8968BB3D886D8B6CA
:108300008BEF41F08DC03BFA8CC08DF03BCA8CF0F6
:108310008B8322EF35F0040E985DD8A492EF41F0E4
:108320005AEC68F0D8968BA3D886D8B6D1EF41F036
:10833000DE6ADE6A3D0EDE6E7D0EDE6E090EDE6EDC
:10834000E4ECA8F0DE6ADE6A430EDE6E8B0EDE6EB3
:10835000090EDE6EE4ECA8F0DE6ADE6AD10EDE6E97
:10836000DE6ADE6AE4ECA8F0010E0101465D000160
:10837000D8A4C7EF41F0DE6ADE6A6D0EDE6E7D0EB8
:10838000DE6E0B0EDE6EE4ECA8F0D1EF41F0DE6A9B
:10839000DE6A6B0EDE6E7D0EDE6E0B0EDE6EE4ECC4
:1083A000A8F0340EDE6E0CEC74F08B9322EF35F0F7
:1083B00011EF48F0350E8C5DD8A46CEF42F0DE6A08
:1083C000FCEC8EF0010E985DD8A4F1EF41F0D89648
:1083D0008BB3D886D8B6EFEF41F0B8EF32F01DEF8F
:1083E00042F0020E985DD8A4FDEF41F0DDECCEF036
:1083F0008B831BEFA2F01DEF42F0030E985DD8A413
:1084000009EF42F0DDECCEF08B831BEFA2F01DEF05
:1084100042F0050E985DD8A41DEF42F0D8968BB3BC
:10842000D886D8B61DEF42F08DC03BFA8CC08DF0D7
:108430003BCA8CF08B8322EF35F0040E985DD8A4F4
:1084400024EF42F05AEC68F0D8968BA3D886D8B6C1
:1084500063EF42F0DE6ADE6A3D0EDE6E7D0EDE6E9A
:10846000090EDE6EE4ECA8F0DE6ADE6A430EDE6E14
:108470008B0EDE6E090EDE6EE4ECA8F0DE6ADE6ABC
:10848000CD0EDE6EDE6ADE6AE4ECA8F0010E0101BC
:10849000465D0001D8A459EF42F0DE6ADE6A6D0E37
:1084A000DE6E7D0EDE6E0B0EDE6EE4ECA8F063EF8A
:1084B00042F0DE6ADE6A6B0EDE6E7D0EDE6E0B0E45
:1084C000DE6EE4ECA8F0350EDE6E0CEC74F08B93EF
:1084D00022EF35F011EF48F0360E8C5DD8A4F6EFA0
:1084E00042F0DE6AFCEC8EF0010E985DD8A483EFBA
:1084F00042F0D8968BB3D886D8B681EF42F0B8EF69
:1085000032F0AFEF42F0020E985DD8A48FEF42F048
:10851000DDECCEF08B831BEFA2F0AFEF42F0030E49
:10852000985DD8A49BEF42F0DDECCEF08B831BEF7F
:10853000A2F0AFEF42F0050E985DD8A4AFEF42F085
:10854000D8968BB3D886D8B6AFEF42F08DC03BFA41
:108550008CC08DF03BCA8CF08B8322EF35F0040E7B
:10856000985DD8A4B6EF42F05AEC68F0D8968BA389
:10857000D886D8B6EDEF42F0DE6ADE6A3D0EDE6EDA
:108580007D0EDE6E090EDE6EE4ECA8F0DE6ADE6AB9
:10859000430EDE6E8B0EDE6E090EDE6EE4ECA8F08E
:1085A000010E0101465D0001D8A4E3EF42F0DE6A4E
:1085B000DE6A6D0EDE6E7D0EDE6E0B0EDE6EE4ECA0
:1085C000A8F0EDEF42F0DE6ADE6A6B0EDE6E7D0E25
:1085D000DE6E0B0EDE6EE4ECA8F0360EDE6E0CECFA
:1085E00074F08B9322EF35F011EF48F0370E8C5D6D
:1085F000D8A480EF43F0DE6AFCEC8EF0010E985DAB
:10860000D8A40DEF43F0D8968BB3D886D8B60BEF2D
:1086100043F0B8EF32F039EF43F0020E985DD8A482
:1086200019EF43F0DDECCEF08B831BEFA2F039EFB6
:1086300043F0030E985DD8A425EF43F0DDECCEF0B7
:108640008B831BEFA2F039EF43F0050E985DD8A4A1
:1086500039EF43F0D8968BB3D886D8B639EF43F0CC
:108660008DC03BFA8CC08DF03BCA8CF08B8322EF1F
:1086700035F0040E985DD8A440EF43F05AEC68F052
:10868000D8968BA3D886D8B677EF43F0DE6ADE6A39
:108690003D0EDE6E7D0EDE6E090EDE6EE4ECA8F0A1
:1086A000DE6ADE6A430EDE6E8B0EDE6E090EDE6E55
:1086B000E4ECA8F0010E0101465D0001D8A46DEFC5
:1086C00043F0DE6ADE6A6D0EDE6E7D0EDE6E0B0E30
:1086D000DE6EE4ECA8F077EF43F0DE6ADE6A6B0E44
:1086E000DE6E7D0EDE6E0B0EDE6EE4ECA8F0370E55
:1086F000DE6E0CEC74F08B9322EF35F011EF48F046
:10870000380E8C5DD8A4D9EF43F0DE6AFCEC8EF015
:10871000010E985DD8A497EF43F0D8968BB3D88616
:10872000D8B695EF43F0B8EF32F0C3EF43F0020E46
:10873000985DD8A4A3EF43F0DDECCEF08B831BEF64
:10874000A2F0C3EF43F0030E985DD8A4AFEF43F05F
:10875000DDECCEF08B831BEFA2F0C3EF43F0050EF0
:10876000985DD8A4C3EF43F0D8968BB3D886D8B61B
:10877000C3EF43F08DC03BFA8CC08DF03BCA8CF048
:108780008B8322EF35F0040E985DD8A4CAEF43F036
:108790005AEC68F0D8968BA3D886D8B6D0EF43F0C1
:1087A000380EDE6E0CEC74F08B9322EF35F011EF87
:1087B00048F0390E8C5DD8A44FEF44F0DE6AFCEC33
:1087C0008EF0010E985DD8A4F0EF43F0D8968BB3ED
:1087D000D886D8B6EEEF43F0B8EF32F01CEF44F095
:1087E000020E985DD8A4FCEF43F0DDECCEF08B8355
:1087F0001BEFA2F01CEF44F0030E985DD8A408EF25
:1088000044F0DDECCEF08B831BEFA2F01CEF44F0C4
:10881000050E985DD8A41CEF44F0D8968BB3D8868B
:10882000D8B61CEF44F08DC03BFA8CC08DF03BCA2B
:108830008CF08B8322EF35F0040E985DD8A423EFE3
:1088400044F05AEC68F0D8968BA3D886D8B646EF99
:1088500044F0DE6ADE6A3D0EDE6E860EDE6EDE6A95
:10886000E4ECA8F0DE6ADE6A650EDE6E420EDE6EB5
:108870000E0EDE6EE4ECA8F0DE6ADE6A670EDE6ED7
:10888000500EDE6E0E0EDE6EE4ECA8F0390EDE6EDB
:108890000CEC74F08B9322EF35F011EF48F03A0EA8
:1088A0008C5DD8A458EF44F009EF9EF011EF48F02A
:1088B0003D0E8C5DD8A4AEEF44F0D8968BA3D8863D
:1088C000D8B6A7EF44F0DDECCEF0D8968BBBD886B7
:1088D000D8B66FEF44F0B66BB56BB86BB76B0801E9
:1088E00027530001D8A477EF44F079EC6CF0DE6AEE
:1088F000DE6A890EDE6EDE6ADE6AE4ECA8F0DE6A0D
:10890000DE6A8A0EDE6E0F0EDE6E030EDE6EE4ECA5
:10891000A8F0DE6ADE6AD70EDE6E840EDE6E020E10
:10892000DE6EE4ECA8F0DE6ADE6AD90EDE6E840E3E
:10893000DE6E060EDE6EE4ECA8F0DE6ADE6A1A0E6B
:10894000DE6E790EDE6E040EDE6EE4ECA8F05FECF7
:108950006FF08B9322EF35F011EF48F03E0E8C5DF7
:10896000D8A4EFEF44F0D8968BA3D886D8B6CDEF35
:1089700044F0D8968BBBD886D8B6C3EF44F0B66B1C
:10898000B56BB86BB76BDDECCEF008012753000177
:10899000D8A4CDEF44F079EC6CF00101395300011B
:1089A000D8A4DFEF44F0DE6ADE6A0C0EDE6E820EC3
:1089B000DE6E040EDE6EE4ECA8F0E9EF44F0DE6A51
:1089C000DE6A0A0EDE6E820EDE6E040EDE6EE4ECF1
:1089D000A8F0010EDE6E1DEC84F011EF48F03F0EA2
:1089E0008C5DD8A412EF45F0D8968BA3D886D8B664
:1089F0000EEF45F0D8968BBBD886D8B604EF45F07D
:108A0000B66BB56BB86BB76BDDECCEF008012753D6
:108A10000001D8A40EEF45F079EC6CF00BEF8AF072
:108A200011EF48F0400E8C5DD8A437EF45F0D89692
:108A30008BA3D886D8B631EF45F0D8968BBBD886B5
:108A4000D8B627EF45F0B66BB56BB86BB76BDDECFE
:108A5000CEF0080127530001D8A431EF45F079EC9E
:108A60006CF0010EDE6E1DEC84F011EF48F0470E45
:108A70008C5DD8A449EF45F0DE6ADE6A180EDE6E22
:108A8000DE6ADE6AE4ECA8F08B831DEF84F011EF60
:108A900048F0480E8C5DD8A462EF45F0DE6AFCEC2D
:108AA0008EF0010E985DD8A45EEF45F0D8968BB39A
:108AB000D886D8B65EEF45F0B8EF32F0D9EFA4F023
:108AC00011EF48F0490E8C5DD8A437EF46F0D896E8
:108AD0008BA3D886D8B676EF45F0010E0101486F1A
:108AE000680E476F010E4A6F680E496F0001DE6A1B
:108AF000FCEC8EF0010E985DD8A489EF45F0D89675
:108B00008BB3D886D8B687EF45F0B8EF32F00DEFCB
:108B100046F0020E985DD8A4E1EF45F004EE1EF099
:108B2000D89001012335E926000EEA22EECF47F165
:108B3000EFCF48F10001DDECCEF0DE6ADE6A5B0EBD
:108B4000DE6E360EDE6EDE6AE4ECA8F0DE6ADE6A09
:108B50005B0EDE6E360EDE6E040EDE6EE4ECA8F00A
:108B6000DE6ADE6A5B0EDE6E360EDE6E090EDE6ECD
:108B7000E4ECA8F0DE6ADE6A5B0EDE6E360EDE6EB8
:108B80000E0EDE6EE4ECA8F00A013E6B0001150E3D
:108B90000A013E5D0001D8B0DDEF45F084ECD2F073
:108BA000C80E54EC01F093ECD2F0C80E54EC01F076
:108BB0000A013E2B0001D8A4E9D7DDECCEF00DEF81
:108BC00046F0030E985DD8A401EF46F0010148512C
:108BD000010A680ED8B447190001D8B4FFEF45F078
:108BE00004EE1EF0D89001012335E926000EEA229A
:108BF000EECF49F1EFCF4AF10001DDECCEF00DEF01
:108C000046F0040E985DD8A408EF46F00DEF46F04C
:108C1000050E985DD8A40DEF46F00DEC90F0DE6ADD
:108C2000DE6A3F0EDE6E860EDE6E090EDE6EE4EC50
:108C3000A8F08B8304EE1EF0D89001012335E926BD
:108C4000000EEA22EECF0BF0EFCF0CF00BC0DEFFF0
:108C50000CC0DEFFDE6A010EDE6E0A0EDE6E000163
:108C60004CEC7BF08B9322EF35F011EF48F04A0E7D
:108C70008C5DD8A444EF46F0DDECCEF055EC98F0D6
:108C8000B8EF32F011EF48F04B0E8C5DD8A4BDEF79
:108C900046F0DE6AFCEC8EF0010E985DD8A459EF28
:108CA00046F0D8968BB3D886D8B659EF46F0B8EFD1
:108CB00032F0040E985DD8A460EF46F05AEC68F0EC
:108CC000020E985DD8A4B7EF46F0AA6A4F0EA96EBF
:108CD000000E46EC01F00A0E54EC01F0AA6A500EA8
:108CE000A96E000E46EC01F00A0E54EC01F0AA6ADF
:108CF000510EA96E000E46EC01F00A0E54EC01F084
:108D0000AA6A520EA96E000E46EC01F00A0E54EC4F
:108D100001F0AA6A530EA96E000E46EC01F00A0E8D
:108D200054EC01F0AA6A540EA96E000E46EC01F054
:108D30000A0E54EC01F0AA6A550EA96E000E46EC1C
:108D400001F00A0E54EC01F0AA6A560EA96E000E4C
:108D500046EC01F00A0E54EC01F00101296B286B7E
:108D60002B6B2A6B08011F6B1E6B1D6B1C6B0001AC
:108D700001EC7EF08B9311EF48F04C0E8C5DD8A483
:108D800057EF47F0DE6AFCEC8EF0010E985DD8A438
:108D9000D4EF46F0D8968BB3D886D8B6D2EF46F04B
:108DA000B8EF32F007EF47F0020E985DD8A4E0EF7D
:108DB00046F0DDECCEF08B83BDEFA2F007EF47F07D
:108DC000030E985DD8A4ECEF46F0DDECCEF08B837B
:108DD000BDEFA2F007EF47F0040E985DD8A4F3EFC3
:108DE00046F007EF47F0050E985DD8A407EF47F06F
:108DF000D8968BB3D886D8B607EF47F08DC03BFA2C
:108E00008CC08DF03BCA8CF08B8322EF35F0D89666
:108E10008BA3D886D8B62DEF47F0DE6ADE6ACD0E7A
:108E2000DE6EDE6ADE6AE4ECA8F0DE6ADE6A3F0E21
:108E3000DE6E860EDE6E090EDE6EE4ECA8F0DE6AF3
:108E4000DE6A3D0EDE6E900EDE6EDE6AE4ECA8F0A9
:108E500001012D6B2C6B2F6B2E6B00012CC1DEFFE3
:108E60002DC1DEFF010EDE6E010EDE6E140EDE6E13
:108E70004CEC7BF004EE1EF0D89001012335E9267E
:108E8000000EEA22EECF0BF0EFCF0CF00BC0DEFFAE
:108E90000CC0DEFFDE6A010EDE6E0A0EDE6E000121
:108EA0004CEC7BF08B9322EF35F011EF48F04D0E38
:108EB0008C5DD8A460EF47F08CEFA6F011EF48F07E
:108EC000510E8C5DD8A46DEF47F0DDECCEF087EC51
:108ED00095F0B8EF32F011EF48F0520E8C5DD8A447
:108EE0007AEF47F0DDECCEF0E5EC96F0B8EF32F03B
:108EF00011EF48F0530E8C5DD8A487EF47F0DDECFE
:108F0000CEF0C7EC91F0B8EF32F011EF48F0540E0C
:108F10008C5DD8A4B4EF47F0CF2B020ECF5DD8A460
:108F20009FEF47F0CF6BDE6ADE6AF70EDE6E370E1C
:108F3000DE6E060EDE6EE4ECA8F0A9EF47F0DE6A06
:108F4000DE6AF50EDE6E370EDE6E060EDE6EE4ECC9
:108F5000A8F0010E246E2C0E55EC01F0DDECCEF0E5
:108F6000B8EF32F011EF48F0550E8C5DD8A4E1EF68
:108F700047F0862B020E865DD8A4CCEF47F0866BB7
:108F8000DE6ADE6AF70EDE6E390EDE6E060EDE6E0D
:108F9000E4ECA8F0D6EF47F0DE6ADE6AF50EDE6E8E
:108FA000390EDE6E060EDE6EE4ECA8F0010E246EC5
:108FB0002C0E55EC01F0DDECCEF0B8EF32F011EFF5
:108FC00048F0560E8C5DD8A4EEEF47F0DDECCEF005
:108FD00057ECA3F0B8EF32F011EF48F0570E8C5D6C
:108FE000D8A4FBEF47F0DDECCEF076EC93F0B8EFD1
:108FF00032F011EF48F0580E8C5DD8A408EF48F01D
:10900000DDECCEF07AEC94F0B8EF32F011EF48F0EE
:109010005B0E8C5DD8A40FEF48F011EF48F0B8EF6D
:1090200032F022EF35F0FF0EDB50DD520901FA89F4
:10903000E8A0FA990101232B800E235D0001D8A43A
:1090400024EF48F00101236B0001D8960901FAA929
:10905000D8860001D8B6C3EF54F00901FA950A0189
:109060003F6B0001D8960901FAB5D8860001D8B641
:109070004FEF48F000EE42F00A013F51EB500B6E0B
:109080002C0E0B5C0001D8A44BEF48F00901FA85C7
:1090900000014DEF48F00A013F2B0001E2D70A0121
:1090A0003F2900EE42F0EBCF0BF00BC043FA020E6B
:1090B0003F2500EE42F0EBCF0BF00BC044FA030E5D
:1090C0003F2500EE42F0EBCF0BF00BC045FA040E4B
:1090D0003F2500EE42F0EBCF0BF00BC046FA050E39
:1090E0003F2500EE42F0EBCF0BF00BC047FA060E27
:1090F0003F2500EE42F0EBCF0BF00BC048FA070E15
:109100003F2500EE42F0EBCF0BF00BC049FA080E02
:109110003F2500EE42F0EBCF0BF00BC04AFA090EF0
:109120003F2500EE42F0EBCF0BF00BC04BFA0A0EDE
:109130003F2500EE42F0EBCF0BF00BC04CFA0901DB
:10914000FA950A01406B00010A0E0A01405D000118
:10915000D8B0D6EF48F00AEE43F00A014051EB5088
:109160000B6E2C0E0B5C0001D8A4C0EF48F0F36A24
:109170000AEE43F00A014051F3CFEBFF0901FA85F3
:109180000001D8960901FAA5D8860001D8B6D0EF1B
:1091900048F0F36A0AEE43F00A014051F3CFEBFFC7
:1091A00000010A01402B0001D8A4CDD70901FA978C
:1091B0000A01416B0001D8960901FAB7D88600016F
:1091C000D8B627EF49F00AEE43F00A014151EB50BF
:1091D0000B6E2E0E0B5C0001D8A423EF49F0060E97
:1091E0000A01415D0AEE43F0EB5001014F6F050E9D
:1091F0000A01415D0AEE43F0EB500101506F040E8D
:109200000A01415D0AEE43F0EB500101516F030E7C
:109210000A01415D0AEE43F0EB500101526F020E6C
:109220000A01415D0AEE43F0EB500101536F0A0160
:1092300041050AEE43F0EB500101546F0901FA8732
:10924000000125EF49F00A01412B0001B3D70901C4
:10925000FA950A013F2B0001D8960901FAB5D88684
:109260000001D8B649EF49F000EE42F00A013F5143
:10927000EB500B6E2C0E0B5C0001D8A445EF49F0AF
:109280000901FA85000147EF49F00A013F2B00016F
:10929000E2D70A013F2900EE42F0EB500B6E560E6A
:1092A0000B5C0001D8A457EF49F0AEEFBDF00A0106
:1092B0003F2900EE42F0EB500B6E410E0B5C0001BB
:1092C000D8B465EF49F0AEEFBDF00A013F2B0901BC
:1092D000FA950001D8960901FAB5D8860001D8B6EA
:1092E00087EF49F000EE42F00A013F51EB500B6E60
:1092F0002C0E0B5C0001D8A483EF49F00901FA851C
:10930000000185EF49F00A013F2B0001E2D70A0175
:109310003F2900EE42F0EBCF0BF00BC04DFA020EEE
:109320003F2500EE42F0EBCF0BF00BC04EFA030EE0
:109330003F2500EE42F0EBCF0BF00BC04FFA040ECE
:109340003F2500EE42F0EBCF0BF00BC050FA050EBC
:109350003F2500EE42F0EBCF0BF00BC051FA060EAA
:109360003F2500EE42F0EBCF0BF00BC052FA070E98
:109370003F2500EE42F0EBCF0BF00BC053FA080E86
:109380003F2500EE42F0EBCF0BF00BC054FA090E74
:109390003F2500EE42F0EBCF0BF00BC055FA0A0E62
:1093A0003F2500EE42F0EBCF0BF00BC056FA0B0E50
:1093B0003F2500EE42F0EBCF0BF00BC057FA09014E
:1093C000FA950A01406B00010B0E0A01405D000195
:1093D000D8B016EF4AF00AEE4DF00A014051EB50BA
:1093E0000B6E2C0E0B5C0001D8A400EF4AF0F36A60
:1093F0000AEE4DF00A014051F3CFEBFF0901FA8567
:109400000001D8960901FAA5D8860001D8B610EF58
:109410004AF0F36A0AEE4DF00A014051F3CFEBFF38
:1094200000010A01402B0001D8A4CDD70901FA9709
:109430000A01416B0001D8960901FAB7D8860001EC
:10944000D8B676EF4AF00AEE4DF00A014151EB50E2
:109450000B6E2E0E0B5C0001D8A472EF4AF0040EC6
:109460000A01415D0AEE4DF0EB500101566F030E0B
:109470000A01415D0AEE4DF0EB500101576F020EFB
:109480000A01415D0AEE4DF0EB500101586F0A01EF
:1094900041050AEE4DF0EB500101596F0A014129D7
:1094A0000AEE4DF0EB5001015A6F020E0A01412500
:1094B0000AEE4DF0EB5001015B6F030E0A014125EE
:1094C0000AEE4DF0EB5001015C6F040E0A014125DC
:1094D0000AEE4DF0EB5001015D6F0901FA870001C2
:1094E00074EF4AF00A01412B0001A4D7226A216AD5
:1094F000206A58C11FF02A6A010E296E860E286E56
:10950000A00E276E02EC02F022C09CF021C09BF05E
:1095100020C09AF01FC099F0226A216A206A59C1BE
:109520001FF02A6A296A270E286E100E276E02EC99
:1095300002F022C034F021C033F020C032F01FC04E
:1095400031F03150992732509A2333509B233450B5
:109550009C23226A216A206A5AC11FF02A6A296A5A
:10956000030E286EE80E276E02EC02F022C034F0E3
:1095700021C033F020C032F01FC031F031509927A4
:1095800032509A2333509B2334509C23226A216A01
:10959000206A5BC11FF02A6A296A286A640E276E56
:1095A00002EC02F022C034F021C033F020C032F0CF
:1095B0001FC031F03150992732509A2333509B23EA
:1095C00034509C23226A216A206A5CC11FF02A6AF7
:1095D000296A286A0A0E276E02EC02F022C034F0D3
:1095E00021C033F020C032F01FC031F03150992734
:1095F00032509A2333509B2334509C2301015D51F8
:1096000000019925996F000E9A219A6F000E9B21F7
:109610009B6F000E9C219C6F010156510A0DF3CFE8
:1096200031F0F4CF32F0575131240001D06F0A01EC
:109630003F2B0901FA950001D8960901FAB5D886A1
:109640000001D8B639EF4BF000EE42F00A013F516D
:10965000EB500B6E2C0E0B5C0001D8A435EF4BF0D9
:109660000901FA85000137EF4BF00A013F2B000199
:10967000E2D70A013F2900EE42F0EB5001015E6F94
:109680000A013F2B0901FA950001D8960901FAB5A4
:10969000D8860001D8B662EF4BF000EE42F00A0126
:1096A0003F51EB500B6E2C0E0B5C0001D8A45EEF0B
:1096B0004BF00901FA85000160EF4BF00A013F2BE6
:1096C0000001E2D70A013F2900EE42F0EBCF0BF098
:1096D0000BC058FA020E3F2500EE42F0EBCF0BF024
:1096E0000BC059FA030E3F2500EE42F0EBCF0BF012
:1096F0000BC05AFA040E3F2500EE42F0EBCF0BF000
:109700000BC05BFA050E3F2500EE42F0EBCF0BF0ED
:109710000BC05CFA060E3F2500EE42F0EBCF0BF0DB
:109720000BC05DFA070E3F2500EE42F0EBCF0BF0C9
:109730000BC05EFA080E3F2500EE42F0EBCF0BF0B7
:109740000BC05FFA090E3F2500EE42F0EBCF0BF0A5
:109750000BC060FA0A0E3F2500EE42F0EBCF0BF093
:109760000BC061FA0B0E3F2500EE42F0EBCF0BF081
:109770000BC062FA0C0E3F2500EE42F0EBCF0BF06F
:109780000BC063FA0901FA950A01406B00010B0E48
:109790000A01405D0001D8B0F9EF4BF00AEE58F035
:1097A0000A014051EB500B6E2C0E0B5C0001D8A44B
:1097B000E3EF4BF0F36A0AEE58F00A014051F3CFA1
:1097C000EBFF0901FA850001D8960901FAA5D886B0
:1097D0000001D8B6F3EF4BF0F36A0AEE58F00A0135
:1097E0004051F3CFEBFF00010A01402B0001D8A448
:1097F000CDD70901FA970A01416B0001D8960901FA
:10980000FAB7D8860001D8B661EF4CF00AEE58F0EE
:109810000A014151EB500B6E2E0E0B5C0001D8A4D7
:109820005DEF4CF0050E0A01415D0AEE58F0EB5079
:1098300001015F6F040E0A01415D0AEE58F0EB5022
:109840000101606F030E0A01415D0AEE58F0EB5012
:109850000101616F020E0A01415D0AEE58F0EB5002
:109860000101626F0A0141050AEE58F0EB50010157
:10987000636F0A0141290AEE58F0EB500101646F51
:10988000020E0A0141250AEE58F0EB500101656F06
:10989000030E0A0141250AEE58F0EB500101666FF4
:1098A000040E0A0141250AEE58F0EB500101676FE2
:1098B0000901FA8700015FEF4CF00A01412B00011A
:1098C0009CD7226A216A206A62C11FF02A6A010EAF
:1098D000296E860E286EA00E276E02EC02F022C0C2
:1098E000A0F021C09FF020C09EF01FC09DF0226A12
:1098F000216A206A63C11FF02A6A296A270E286E2E
:10990000100E276E02EC02F022C034F021C033F0BA
:1099100020C032F01FC031F031509D2732509E23BD
:1099200033509F233450A023226A216A206A64C1E5
:109930001FF02A6A296A030E286EE80E276E02ECD1
:1099400002F022C034F021C033F020C032F01FC03A
:1099500031F031509D2732509E2333509F23345095
:10996000A023226A216A206A65C11FF02A6A296A37
:10997000286A640E276E02EC02F022C034F021C087
:1099800033F020C032F01FC031F031509D273250EB
:109990009E2333509F233450A023226A216A206AD9
:1099A00066C11FF02A6A296A286A0A0E276E02EC2D
:1099B00002F022C034F021C033F020C032F01FC0CA
:1099C00031F031509D2732509E2333509F23345025
:1099D000A0230101675100019D259D6F000E9E216E
:1099E0009E6F000E9F219F6F000EA021A06F326A14
:1099F0005FC131F03250640DF3CF32F03150640D5D
:109A0000F3CF31F0F4503226366A60C135F036506B
:109A10000A0DF3CF36F035500A0DF3CF35F0F45080
:109A2000362635503126365032220101615131241B
:109A30000001D16F0A013F2B0901FA950001D89668
:109A40000901FAB5D8860001D8B63CEF4DF000EE1A
:109A500042F00A013F51EB500B6E2C0E0B5C0001E3
:109A6000D8A438EF4DF00901FA8500013AEF4DF026
:109A70000A013F2B0001E2D70A013F2900EE42F024
:109A8000EB500101686F0A013F2B0901FA950001B3
:109A9000D8960901FAB5D8860001D8B665EF4DF021
:109AA00000EE42F00A013F51EB500B6E2C0E0B5CA6
:109AB0000001D8A461EF4DF00901FA85000163EFC0
:109AC0004DF00A013F2B0001E2D70A013F2900EEC9
:109AD00042F0EBCF0BF00BC064FA020E3F2500EE14
:109AE00042F0EBCF0BF00BC065FA030E3F2500EE02
:109AF00042F0EBCF0BF00BC066FA040E3F2500EEF0
:109B000042F0EBCF0BF00BC067FA050E3F2500EEDD
:109B100042F0EBCF0BF00BC068FA060E3F2500EECB
:109B200042F0EBCF0BF00BC069FA070E3F2500EEB9
:109B300042F0EBCF0BF00BC06AFA0901FA950A016B
:109B4000406B0001070E0A01405D0001D8B0D4EF60
:109B50004DF00AEE64F00A014051EB500B6E2C0EF2
:109B60000B5C0001D8A4BEEF4DF0F36A0AEE64F07E
:109B70000A014051F3CFEBFF0901FA850001D896A5
:109B80000901FAA5D8860001D8B6CEEF4DF0F36AE8
:109B90000AEE64F00A014051F3CFEBFF00010A0125
:109BA000402B0001D8A4CDD70901FA970A01416BD7
:109BB0000001D8960901FAB7D8860001D8B62EEF71
:109BC0004EF00AEE64F00A014151EB500B6E2E0E7E
:109BD0000B5C0001D8A42AEF4EF0020E0A01415D91
:109BE0000001D8B0F9EF4DF00101696B000101EF00
:109BF0004EF0020E0A01415D0AEE64F0EB500101E5
:109C0000696F0001010E0A01415D0001D8B00EEF3D
:109C10004EF001016A6B000115EF4EF00A0141059B
:109C20000AEE64F0EB5001016A6F00010A0141295C
:109C30000AEE64F0EB5001016B6F020E0A01412540
:109C40000AEE64F0EB5001016C6F0901FA87000124
:109C50002CEF4EF00A01412B0001AAD70A0E010198
:109C6000695D0001D8A037EF4EF00101696B00017A
:109C70000A0E01016A5D0001D8A041EF4EF001011A
:109C80006A6B00010A0E01016B5D0001D8A04BEF69
:109C90004EF001016B6B00010A0E01016C5D0001C9
:109CA000D8A055EF4EF001016C6B0001326A69C11A
:109CB00031F032C02EF031502D6EE80DF3CF31F07F
:109CC000F4CF32F02E50E80DF35032262D50030D14
:109CD000F3503226366A6AC135F03650640DF3CF40
:109CE00036F03550640DF3CF35F0F450362635504C
:109CF000312636503222366A6BC135F036500A0DA5
:109D0000F3CF36F035500A0DF3CF35F0F450362648
:109D1000355031263650322201016C5131246D6F9D
:109D2000000E32206E6F270E0A01426F00010A01F9
:109D300042290B6E01EEA2F0D8904235E926000EC2
:109D4000EA22EECF0FF0EFCF10F001EEA2F0D890A4
:109D50000B34E926000EEA220FC0EEFF10C0EFFF21
:109D6000010E425F0001D8B0E1D76EC1A3F16DC111
:109D7000A2F1C46BC36BC26BC16B0A01746B0001AF
:109D80000A0174510101345D0001D8A0E1EF4EF0E9
:109D900001EEA2F0D8900A017435E926000EEA22FD
:109DA000EECF0BF0EFCF0CF00B500001C1270C50A1
:109DB000C223000EC323C4230A01742B0001D8A4BC
:109DC000DED7336A346A01013429316E000E326AFB
:109DD0003222C4C022F0C3C021F0C2C020F0C1C0F2
:109DE0001FF034C02AF033C029F032C028F031C04F
:109DF00027F08BEC01F020C0C6F01FC0C5F003EEC9
:109E00001EF0D8902335E926000EEA22C5C0EEFFE9
:109E1000C6C0EFFF03EE1EF0D8902335E926000EF2
:109E2000EA22EECF0BF0EFCF0CF00B50285D0C5078
:109E300029590001D8B029EF4FF003EE1EF0D89059
:109E400001012335E926000EEA22EECF28F1EFCFFB
:109E500029F10001C46BC36BC26BC16B0A01746B47
:109E60000001280E0A01745D0001D8B051EF4FF0D7
:109E700001EEA2F0D8900A017435E926000EEA221C
:109E8000EECF0BF0EFCF0CF00B500001C1270C50C0
:109E9000C223000EC323C4230A01742B0001D8A4DB
:109EA000DFD7C4C022F0C3C021F0C2C020F0C1C0BF
:109EB0001FF02A6A296A286A280E276E8BEC01F0A7
:109EC00020C03AF51FC039F50501395101012A5D5D
:109ED00005013A5101012B590001D8B074EF4FF040
:109EE0003AC52BF139C52AF10A013F2B0901FA9530
:109EF0000001D8960901FAB5D8860001D8B696EFC8
:109F00004FF000EE42F00A013F51EB500B6E2C0E69
:109F10000B5C0001D8A492EF4FF00901FA85000113
:109F200094EF4FF00A013F2B0001E2D70A013F29CD
:109F300000EE42F0EBCF0BF00BC06BFA020E3F25A8
:109F400000EE42F0EBCF0BF00BC06CFA030E3F2596
:109F500000EE42F0EBCF0BF00BC06DFA040E3F2584
:109F600000EE42F0EBCF0BF00BC06EFA050E3F2572
:109F700000EE42F0EBCF0BF00BC06FFA060E3F2560
:109F800000EE42F0EBCF0BF00BC070FA070E3F254E
:109F900000EE42F0EBCF0BF00BC071FA0901FA951D
:109FA0000A01406B0001070E0A01405D0001D8B0B4
:109FB00005EF50F00AEE6BF00A014051EB500B6ECA
:109FC0002C0E0B5C0001D8A4EFEF4FF0F36A0AEE01
:109FD0006BF00A014051F3CFEBFF0901FA85000154
:109FE000D8960901FAA5D8860001D8B6FFEF4FF040
:109FF000F36A0AEE6BF00A014051F3CFEBFF000168
:10A000000A01402B0001D8A4CDD70901FA970A0113
:10A01000416B0001D8960901FAB7D8860001D8B67D
:10A0200065EF50F00AEE6BF00A014151EB500B6EF8
:10A030002E0E0B5C0001D8A461EF50F0030E0A0154
:10A04000415D0001D8B02AEF50F001016F6B0001B3
:10A0500032EF50F0030E0A01415D0AEE6BF0EB5057
:10A0600001016F6F0001020E0A01415D0001D8B0CD
:10A070003FEF50F00101706B000147EF50F0020E0E
:10A080000A01415D0AEE6BF0EB500101706F0001B7
:10A09000010E0A01415D0001D8B054EF50F00101FA
:10A0A000716B00015BEF50F00A0141050AEE6BF0A5
:10A0B000EB500101716F00010901FA87000163EFA4
:10A0C00050F00A01412B0001A4D7040E01016F5D7D
:10A0D0000001D8A06EEF50F001016F6B00010A0E75
:10A0E0000101705D0001D8A078EF50F00101706BA4
:10A0F00000010A0E0101715D0001D8A082EF50F04D
:10A100000101716B0001326A6FC131F03250640D90
:10A11000F3CF32F03150640DF3CF31F0F4503226EA
:10A12000366A70C135F036500A0DF3CF36F035502F
:10A130000A0DF3CF35F0F45036263550312636501F
:10A140003222010171513124446F000E3220456FDB
:10A1500030530001D8A4D3EF50F001014553000162
:10A16000D8A4BAEF50F001013151445D0001D8A0EC
:10A17000C2EF50F001013151445F000E455B000118
:10A18000D0EF50F001014451315D446F451DD8B00E
:10A19000010F456F44516808446F010E4555456FE6
:10A1A0000001EEEF50F0010131514427000E45232C
:10A1B000010E455D0001D8A0EDEF50F0D8A4E8EF06
:10A1C00050F0680E0101445D0001D8A0EDEF50F0A1
:10A1D000680E0101445F010E455B0001130E0A0188
:10A1E000426F00010A0142290B6E01EEF4F0D89093
:10A1F0004235E926000EEA22EECF0FF0EFCF10F045
:10A2000001EEF4F0D8900B34E926000EEA220FC0DC
:10A21000EEFF10C0EFFF010E425F0001D8B0E1D7A2
:10A2200045C1F5F144C1F4F10A019F6BA06B746B59
:10A2300000010A0174510101345D0001D8A06DEFE5
:10A2400051F001EEF4F0D8900A017435E926000EC1
:10A25000EA22EECF0BF0EFCF0CF00AEE75F0D890BB
:10A260007435E926000EEA220BC0EEFF0CC0EFFFAA
:10A270000AEE75F0D8907435E926000EEA22EECF8A
:10A280001FF0EFCF20F0020E75EC01F00B6E030E05
:10A290000B5C0001D8A44FEF51F00A019F2B000185
:10A2A0000AEE75F0D8900A017435E926000EEA220C
:10A2B000EECF1FF0EFCF20F0020E75EC01F00B6E29
:10A2C0000B520001D8A467EF51F00A01A02B000146
:10A2D0000A01742B0001D8A4ABD70A019F530001D7
:10A2E000D8B4D3EF51F00A01A0530001D8B4D3EF92
:10A2F00051F00A019F51A0250B6E0C6A0C3601012A
:10A300003429116E000E126A122212500C5C0001E8
:10A31000D8A4D3EF51F011500B5CD8A4D3EF51F077
:10A320000A01746B00010A0174510101345D0001DE
:10A33000D8A0D3EF51F00AEE75F0D8900A01743529
:10A34000E926000EEA22EECF1FF0EFCF20F0020E3A
:10A3500075EC01F00B6E0B520001D8A4CDEF51F05B
:10A360000AEE75F0D8900A017435E926000EEA224B
:10A37000EECF0FF0EFCF10F0680E0F240B6E010E32
:10A3800010200C6E0AEE75F0D8907435E926000E98
:10A39000EA220BC0EEFF0CC0EFFF00010A01742B94
:10A3A0000001D8A4BFD7C46BC36BC26BC16B0A01D9
:10A3B000746B00010A0174510101345D0001D8A0E1
:10A3C000FBEF51F00AEE75F0D8900A017435E926DA
:10A3D000000EEA22EECF0BF0EFCF0CF00B50000195
:10A3E000C1270C50C223000EC323C4230A01742BBF
:10A3F0000001D8A4DED7336A346A01013429316EF2
:10A40000000E326A3222C4C022F0C3C021F0C2C0A2
:10A4100020F0C1C01FF034C02AF033C029F032C090
:10A4200028F031C027F08BEC01F020C0CAF01FC02B
:10A43000C9F0010E0001CA5DD8A02BEF52F0D8A4DC
:10A4400027EF52F0680EC95DD8A02BEF52F0680ECE
:10A45000C95F010ECA5B04EE1EF0D89001012335DE
:10A46000E926000EEA22C9C0EEFFCAC0EFFF0A01CA
:10A470003F2B0901FA950001D8960901FAB5D88653
:10A480000001D8B659EF52F000EE42F00A013F51F8
:10A49000EB500B6E2C0E0B5C0001D8A455EF52F064
:10A4A0000901FA85000157EF52F00A013F2B000124
:10A4B000E2D70A013F2900EE42F0EB500101726F32
:10A4C000020E0A013F2500EE42F0EB500101736FCE
:10A4D000030E0A013F2500EE42F0EB500101746FBC
:10A4E000040E0A013F2500EE42F0EB500101756FAA
:10A4F000050E0A013F2500EE42F0EB500101766F98
:10A50000060E0A013F2500EE42F0EB500101776F85
:10A5100000019453D8B499EF52F09651010A900E6D
:10A52000D8B49519D8A499EF52F045C196F044C11A
:10A5300095F09453D8B4A9EF52F095C0DEFF96C0C1
:10A54000DEFF42EC0FF01AEE72F05BEC02F0ACEFC3
:10A5500052F00A01736B726B0001130E0A01426F15
:10A5600000010A0142290B6E01EE78F0D8904235C5
:10A57000E926000EEA22EECF0FF0EFCF10F001EE49
:10A5800078F0D8900B34E926000EEA220FC0EEFFD7
:10A5900010C0EFFF010E425F0001D8B0E1D773CACF
:10A5A00079F172CA78F1C46BC36BC26BC16B0A01DB
:10A5B000746B00010A0174510101345D0001D8A0DF
:10A5C000FBEF52F001EE78F0D8900A017435E926DD
:10A5D000000EEA22EECF0BF0EFCF0CF00B50000193
:10A5E000C1270C50C223000EC323C4230A01742BBD
:10A5F0000001D8A4DED7336A346A01013429316EF0
:10A60000000E326A3222C4C022F0C3C021F0C2C0A0
:10A6100020F0C1C01FF034C02AF033C029F032C08E
:10A6200028F031C027F08BEC01F020C0C8F01FC02B
:10A63000C7F002EE1EF0D8902335E926000EEA227C
:10A64000C7C0EEFFC8C0EFFF0A01725101012E5DC5
:10A650000A01735101012F590001D8B038EF53F0AE
:10A6600073CA2FF172CA2EF145C12DF144C12CF1EC
:10A6700073CA20F072CA1FF0030E75EC01F00501D9
:10A680001E6F73CA20F072CA1FF0020E75EC01F043
:10A690001F6F73CA20F072CA1FF0010E75EC01F033
:10A6A000206F73CA20F072CA1FF0000E75EC01F023
:10A6B000216F020E0001B95DD8A473EF53F0D89654
:10A6C0008BB3D886D8B673EF53F0CC51CB11D8A446
:10A6D00070EF53F0A2EC29F0CEC0CCF0CDC0CBF09F
:10A6E000CB07000ECC5B03EE1EF0D89001012335A2
:10A6F000E926000EEA22EECF0BF0EFCF0CF00C5261
:10A700000001D8A489EF53F01F0E0B5CD8A0C1EF55
:10A7100054F03D0E0501385D0001D8A0BEEF54F0A5
:10A720001A6A7C0E196E120E186E920E176E9DC06C
:10A7300013F09EC014F09FC015F0A0C016F05CECA2
:10A7400009F050EC08F016C029F515C028F514C022
:10A7500027F513C026F5D15158EC09F029C51AF098
:10A7600028C519F027C518F026C517F0B6EC07F074
:10A7700016C029F515C028F514C027F513C026F515
:10A78000570E0101685D0001D8A4CAEF53F0800E96
:10A790000501271B00011A6A7C0E196E120E186E35
:10A7A000920E176E99C013F09AC014F09BC015F06A
:10A7B0009CC016F05CEC09F050EC08F016C025F5D2
:10A7C00015C024F514C023F513C022F5D05158EC60
:10A7D00009F025C51AF024C519F023C518F022C5C3
:10A7E00017F0B6EC07F016C025F515C024F514C017
:10A7F00023F513C022F5530E01015E5D0001D8A4BC
:10A8000005EF54F0800E0501231B000105012A53BA
:10A810000001D8B4A9EF54F022C5DEFF23C5DEFF46
:10A8200024C5DEFF25C5DEFF26C5DEFF27C5DEFF0A
:10A8300028C5DEFF29C5DEFF2AC5DEFF2BC5DEFFEA
:10A840002CC5DEFF2DC5DEFF2EC5DEFF2FC5DEFFCA
:10A8500030C5DEFF31C5DEFFD2EC17F015EE34F067
:10A860004AEC02F037C522F036C521F035C520F09C
:10A8700034C51FF02A6A0F0E296E420E286E400E54
:10A88000276E8BEC01F020C033F51FC032F5226A31
:10A89000216A33C520F032C51FF02A6A0F0E296ED7
:10A8A000420E286E400E276E02EC02F022C034F0F9
:10A8B00021C033F020C032F01FC031F0315005010B
:10A8C000345F3250355B3350365B3450375BD8964B
:10A8D00037BFD8860001D8B6A1EF54F00501355135
:10A8E0003611371106E1650E345D0001D8A0A1EFE5
:10A8F00054F00501345108011C27050135510801A8
:10A900001D230501365108011E2305013751080199
:10A910001F2325C52DF524C52CF523C52BF522C5F0
:10A920002AF529C531F528C530F527C52FF526C5E7
:10A930002EF50501376B366B356B346B0001A6EFD6
:10A9400054F00501376B366B356B346B0001B9EF92
:10A9500054F025C52DF524C52CF523C52BF522C5AE
:10A960002AF529C531F528C530F527C52FF526C5A7
:10A970002EF50501386B0001C0EF54F00501382BAE
:10A980000001AEEF5CF00901FA950A013F6B00018E
:10A99000D8960901FAB5D8860001D8B6E5EF54F08B
:10A9A00000EE42F00A013F51EB500B6E2C0E0B5C97
:10A9B0000001D8A4E1EF54F00901FA850001E3EFAA
:10A9C00054F00A013F2B0001E2D70901FA950A0170
:10A9D0003F2B0001D8960901FAB5D8860001D8B6F8
:10A9E00007EF55F000EE42F00A013F51EB500B6EBD
:10A9F0002C0E0B5C0001D8A403EF55F00901FA8579
:10AA0000000105EF55F00A013F2B0001E2D70A01D2
:10AA10003F2B0901FA950001D8960901FAB5D886AD
:10AA20000001D8B629EF55F000EE42F00A013F517F
:10AA3000EB500B6E2C0E0B5C0001D8A425EF55F0EB
:10AA40000901FA85000127EF55F00A013F2B0001AB
:10AA5000E2D70A013F2900EE42F0EBCF0BF00BC02A
:10AA60004DFA020E3F2500EE42F0EBCF0BF00BC08B
:10AA70004EFA030E3F2500EE42F0EBCF0BF00BC079
:10AA80004FFA040E3F2500EE42F0EBCF0BF00BC067
:10AA900050FA050E3F2500EE42F0EBCF0BF00BC055
:10AAA00051FA060E3F2500EE42F0EBCF0BF00BC043
:10AAB00052FA070E3F2500EE42F0EBCF0BF00BC031
:10AAC00053FA080E3F2500EE42F0EBCF0BF00BC01F
:10AAD00054FA090E3F2500EE42F0EBCF0BF00BC00D
:10AAE00055FA0A0E3F2500EE42F0EBCF0BF00BC0FB
:10AAF00056FA0B0E3F2500EE42F0EBCF0BF00BC0E9
:10AB000057FA0901FA950A01406B00010B0E0A0180
:10AB1000405D0001D8B0B8EF55F00AEE4DF00A01E3
:10AB20004051EB500B6E2C0E0B5C0001D8A4A2EF31
:10AB300055F0F36A0AEE4DF00A014051F3CFEBFFF6
:10AB40000901FA850001D8960901FAA5D886000105
:10AB5000D8B6B2EF55F0F36A0AEE4DF00A01405153
:10AB6000F3CFEBFF00010A01402B0001D8A4CDD7A1
:10AB70000901FA970A01416B0001D8960901FAB759
:10AB8000D8860001D8B618EF56F00AEE4DF00A014B
:10AB90004151EB500B6E2E0E0B5C0001D8A414EF4C
:10ABA00056F0040E0A01415D0AEE4DF0EB50010132
:10ABB000566F030E0A01415D0AEE4DF0EB500101A4
:10ABC000576F020E0A01415D0AEE4DF0EB50010194
:10ABD000586F0A0141050AEE4DF0EB500101596F23
:10ABE0000A0141290AEE4DF0EB5001015A6F020EA5
:10ABF0000A0141250AEE4DF0EB5001015B6F030E97
:10AC00000A0141250AEE4DF0EB5001015C6F040E84
:10AC10000A0141250AEE4DF0EB5001015D6F09017B
:10AC2000FA87000116EF56F00A01412B0001A4D764
:10AC3000226A216A206A58C11FF02A6A010E296E11
:10AC4000860E286EA00E276E02EC02F022C09CF049
:10AC500021C09BF020C09AF01FC099F0226A216A9F
:10AC6000206A59C11FF02A6A296A270E286E100E21
:10AC7000276E02EC02F022C034F021C033F020C075
:10AC800032F01FC031F03150992732509A2333509F
:10AC90009B2334509C23226A216A206A5AC11FF0E8
:10ACA0002A6A296A030E286EE80E276E02EC02F06B
:10ACB00022C034F021C033F020C032F01FC031F088
:10ACC0003150992732509A2333509B2334509C2380
:10ACD000226A216A206A5BC11FF02A6A296A286AEF
:10ACE000640E276E02EC02F022C034F021C033F073
:10ACF00020C032F01FC031F03150992732509A23D2
:10AD000033509B2334509C23226A216A206A5CC101
:10AD10001FF02A6A296A286A0A0E276E02EC02F0DE
:10AD200022C034F021C033F020C032F01FC031F017
:10AD30003150992732509A2333509B2334509C230F
:10AD400001015D5100019925996F000E9A219A6FBA
:10AD5000000E9B219B6F000E9C219C6F01015651A0
:10AD60000A0DF3CF31F0F4CF32F057513124000106
:10AD7000D06F0A013F2B0901FA950001D89609010D
:10AD8000FAB5D8860001D8B6DBEF56F000EE42F0F7
:10AD90000A013F51EB500B6E2C0E0B5C0001D8A446
:10ADA000D7EF56F00901FA850001D9EF56F00A01F4
:10ADB0003F2B0001E2D70A013F2900EE42F0EB50A1
:10ADC00001015E6F0A013F2B0901FA950001D89637
:10ADD0000901FAB5D8860001D8B604EF57F000EEA5
:10ADE00042F00A013F51EB500B6E2C0E0B5C000140
:10ADF000D8A400EF57F00901FA85000102EF57F0DF
:10AE00000A013F2B0001E2D70A013F2900EE42F080
:10AE1000EBCF0BF00BC058FA020E3F2500EE42F0CC
:10AE2000EBCF0BF00BC059FA030E3F2500EE42F0BA
:10AE3000EBCF0BF00BC05AFA040E3F2500EE42F0A8
:10AE4000EBCF0BF00BC05BFA050E3F2500EE42F096
:10AE5000EBCF0BF00BC05CFA060E3F2500EE42F084
:10AE6000EBCF0BF00BC05DFA070E3F2500EE42F072
:10AE7000EBCF0BF00BC05EFA080E3F2500EE42F060
:10AE8000EBCF0BF00BC05FFA090E3F2500EE42F04E
:10AE9000EBCF0BF00BC060FA0A0E3F2500EE42F03C
:10AEA000EBCF0BF00BC061FA0B0E3F2500EE42F02A
:10AEB000EBCF0BF00BC062FA0C0E3F2500EE42F018
:10AEC000EBCF0BF00BC063FA0901FA950A01406B56
:10AED00000010B0E0A01405D0001D8B09BEF57F056
:10AEE0000AEE58F00A014051EB500B6E2C0E0B5C31
:10AEF0000001D8A485EF57F0F36A0AEE58F00A0172
:10AF00004051F3CFEBFF0901FA850001D896090102
:10AF1000FAA5D8860001D8B695EF57F0F36A0AEE85
:10AF200058F00A014051F3CFEBFF00010A01402B1A
:10AF30000001D8A4CDD70901FA970A01416B00019D
:10AF4000D8960901FAB7D8860001D8B603EF58F0B1
:10AF50000AEE58F00A014151EB500B6E2E0E0B5CBD
:10AF60000001D8A4FFEF57F0050E0A01415D0AEE7B
:10AF700058F0EB5001015F6F040E0A01415D0AEECB
:10AF800058F0EB500101606F030E0A01415D0AEEBB
:10AF900058F0EB500101616F020E0A01415D0AEEAB
:10AFA00058F0EB500101626F0A0141050AEE58F0BA
:10AFB000EB500101636F0A0141290AEE58F0EB5092
:10AFC0000101646F020E0A0141250AEE58F0EB50B0
:10AFD0000101656F030E0A0141250AEE58F0EB509E
:10AFE0000101666F040E0A0141250AEE58F0EB508C
:10AFF0000101676F0901FA87000101EF58F00A01AA
:10B00000412B00019CD7226A216A206A62C11FF08D
:10B010002A6A010E296E860E286EA00E276E02EC9B
:10B0200002F022C0A0F021C09FF020C09EF01FC0FF
:10B030009DF0226A216A206A63C11FF02A6A296A88
:10B04000270E286E100E276E02EC02F022C034F09C
:10B0500021C033F020C032F01FC031F031509D27A5
:10B0600032509E2333509F233450A023226A216AFA
:10B07000206A64C11FF02A6A296A030E286EE80E4E
:10B08000276E02EC02F022C034F021C033F020C061
:10B0900032F01FC031F031509D2732509E23335083
:10B0A0009F233450A023226A216A206A65C11FF0C1
:10B0B0002A6A296A286A640E276E02EC02F022C00E
:10B0C00034F021C033F020C032F01FC031F03150D5
:10B0D0009D2732509E2333509F233450A023226A51
:10B0E000216A206A66C11FF02A6A296A286A0A0E44
:10B0F000276E02EC02F022C034F021C033F020C0F1
:10B1000032F01FC031F031509D2732509E23335012
:10B110009F233450A0230101675100019D259D6F9D
:10B12000000E9E219E6F000E9F219F6F000EA0219A
:10B13000A06F326A5FC131F03250640DF3CF32F04C
:10B140003150640DF3CF31F0F4503226366A60C1CD
:10B1500035F036500A0DF3CF36F035500A0DF3CFE7
:10B1600035F0F45036263550312636503222010162
:10B17000615131240001D16F0A013F2B0901FA9579
:10B180000001D8960901FAB5D8860001D8B6DEEFDD
:10B1900058F000EE42F00A013F51EB500B6E2C0EBE
:10B1A0000B5C0001D8A4DAEF58F00901FA85000120
:10B1B000DCEF58F00A013F2B0001E2D70A013F29DA
:10B1C00000EE42F0EB500101686F0A013F2B0901CC
:10B1D000FA950001D8960901FAB5D8860001D8B6CB
:10B1E00007EF59F000EE42F00A013F51EB500B6EB1
:10B1F0002C0E0B5C0001D8A403EF59F00901FA856D
:10B20000000105EF59F00A013F2B0001E2D70A01C6
:10B210003F2900EE42F0EBCF0BF00BC064FA020EB8
:10B220003F2500EE42F0EBCF0BF00BC065FA030EAA
:10B230003F2500EE42F0EBCF0BF00BC066FA040E98
:10B240003F2500EE42F0EBCF0BF00BC067FA050E86
:10B250003F2500EE42F0EBCF0BF00BC068FA060E74
:10B260003F2500EE42F0EBCF0BF00BC069FA070E62
:10B270003F2500EE42F0EBCF0BF00BC06AFA09015C
:10B28000FA950A01406B0001070E0A01405D0001BA
:10B29000D8B076EF59F00AEE64F00A014051EB5055
:10B2A0000B6E2C0E0B5C0001D8A460EF59F0F36A12
:10B2B0000AEE64F00A014051F3CFEBFF0901FA8571
:10B2C0000001D8960901FAA5D8860001D8B670EF1A
:10B2D00059F0F36A0AEE64F00A014051F3CFEBFF34
:10B2E00000010A01402B0001D8A4CDD70901FA972B
:10B2F0000A01416B0001D8960901FAB7D88600010E
:10B30000D8B6D0EF59F00AEE64F00A014151EB5083
:10B310000B6E2E0E0B5C0001D8A4CCEF59F0020E80
:10B320000A01415D0001D8B09BEF59F00101696B42
:10B330000001A3EF59F0020E0A01415D0AEE64F02C
:10B34000EB500101696F0001010E0A01415D00012E
:10B35000D8B0B0EF59F001016A6B0001B7EF59F0B6
:10B360000A0141050AEE64F0EB5001016A6F000129
:10B370000A0141290AEE64F0EB5001016B6F020EE5
:10B380000A0141250AEE64F0EB5001016C6F0901DE
:10B39000FA870001CEEF59F00A01412B0001AAD72C
:10B3A0000A0E0101695D0001D8A0D9EF59F0010131
:10B3B000696B00010A0E01016A5D0001D8A0E3EF8C
:10B3C00059F001016A6B00010A0E01016B5D000179
:10B3D000D8A0EDEF59F001016B6B00010A0E0101DD
:10B3E0006C5D0001D8A0F7EF59F001016C6B000112
:10B3F000326A69C131F032C02EF031502D6EE80D45
:10B40000F3CF31F0F4CF32F02E50E80DF350322666
:10B410002D50030DF3503226366A6AC135F036508E
:10B42000640DF3CF36F03550640DF3CF35F0F450A2
:10B4300036263550312636503222366A6BC135F009
:10B4400036500A0DF3CF36F035500A0DF3CF35F0F4
:10B45000F4503626355031263650322201016C51D7
:10B4600031246D6F000E32206E6F270E0A01426F7D
:10B4700000010A0142290B6E01EEA2F0D89042357C
:10B48000E926000EEA22EECF0FF0EFCF10F001EE2A
:10B49000A2F0D8900B34E926000EEA220FC0EEFF8E
:10B4A00010C0EFFF010E425F0001D8B0E1D76EC1BE
:10B4B000A3F16DC1A2F1C46BC36BC26BC16B0A0176
:10B4C000746B00010A0174510101345D0001D8A0C0
:10B4D00083EF5AF001EEA2F0D8900A017435E92604
:10B4E000000EEA22EECF0BF0EFCF0CF00B50000174
:10B4F000C1270C50C223000EC323C4230A01742B9E
:10B500000001D8A4DED7336A346A01013429316ED0
:10B51000000E326A3222C4C022F0C3C021F0C2C081
:10B5200020F0C1C01FF034C02AF033C029F032C06F
:10B5300028F031C027F08BEC01F020C0C6F01FC00E
:10B54000C5F003EE1EF0D8902335E926000EEA225E
:10B55000C5C0EEFFC6C0EFFF03EE1EF0D890233546
:10B56000E926000EEA22EECF0BF0EFCF0CF00B50E5
:10B57000285D0C5029590001D8B0CBEF5AF003EEEA
:10B580001EF0D89001012335E926000EEA22EECF05
:10B5900028F1EFCF29F10001C46BC36BC26BC16B03
:10B5A0000A01746B0001280E0A01745D0001D8B015
:10B5B000F3EF5AF001EEA2F0D8900A017435E926B3
:10B5C000000EEA22EECF0BF0EFCF0CF00B50000193
:10B5D000C1270C50C223000EC323C4230A01742BBD
:10B5E0000001D8A4DFD7C4C022F0C3C021F0C2C07C
:10B5F00020F0C1C01FF02A6A296A286A280E276E27
:10B600008BEC01F020C02BF11FC02AF10A013F2B67
:10B610000901FA950001D8960901FAB5D88600010A
:10B62000D8B628EF5BF000EE42F00A013F51EB5034
:10B630000B6E2C0E0B5C0001D8A424EF5BF009010B
:10B64000FA85000126EF5BF00A013F2B0001E2D7EB
:10B650000A013F2900EE42F0EBCF0BF00BC06BFA72
:10B66000020E3F2500EE42F0EBCF0BF00BC06CFA60
:10B67000030E3F2500EE42F0EBCF0BF00BC06DFA4E
:10B68000040E3F2500EE42F0EBCF0BF00BC06EFA3C
:10B69000050E3F2500EE42F0EBCF0BF00BC06FFA2A
:10B6A000060E3F2500EE42F0EBCF0BF00BC070FA18
:10B6B000070E3F2500EE42F0EBCF0BF00BC071FA06
:10B6C0000901FA950A01406B0001070E0A01405D6D
:10B6D0000001D8B097EF5BF00AEE6BF00A01405121
:10B6E000EB500B6E2C0E0B5C0001D8A481EF5BF0CD
:10B6F000F36A0AEE6BF00A014051F3CFEBFF090148
:10B70000FA850001D8960901FAA5D8860001D8B6B5
:10B7100091EF5BF0F36A0AEE6BF00A014051F3CF50
:10B72000EBFF00010A01402B0001D8A4CDD709018D
:10B73000FA970A01416B0001D8960901FAB7D88639
:10B740000001D8B6F7EF5BF00AEE6BF00A01415149
:10B75000EB500B6E2E0E0B5C0001D8A4F3EF5BF0E8
:10B76000030E0A01415D0001D8B0BCEF5BF001019E
:10B770006F6B0001C4EF5BF0030E0A01415D0AEE3E
:10B780006BF0EB5001016F6F0001020E0A01415D89
:10B790000001D8B0D1EF5BF00101706B0001D9EF6F
:10B7A0005BF0020E0A01415D0AEE6BF0EB50010105
:10B7B000706F0001010E0A01415D0001D8B0E6EF93
:10B7C0005BF00101716B0001EDEF5BF00A014105D7
:10B7D0000AEE6BF0EB500101716F00010901FA876D
:10B7E0000001F5EF5BF00A01412B0001A4D7040E24
:10B7F00001016F5D0001D8A000EF5CF001016F6BEB
:10B8000000010A0E0101705D0001D8A00AEF5CF092
:10B810000101706B00010A0E0101715D0001D8A0E9
:10B8200014EF5CF00101716B0001326A6FC131F0FD
:10B830003250640DF3CF32F03150640DF3CF31F05C
:10B84000F4503226366A70C135F036500A0DF3CF07
:10B8500036F035500A0DF3CF35F0F450362635501A
:10B86000312636503222010171513124446F000ECD
:10B870003220456F30530001D8A465EF5CF0010120
:10B8800045530001D8A44CEF5CF001013151445DF7
:10B890000001D8A054EF5CF001013151445F000E6B
:10B8A000455B000162EF5CF001014451315D446F82
:10B8B000451DD8B0010F456F44516808446F010E13
:10B8C0004555456F000180EF5CF00101315144277F
:10B8D000000E4523010E455D0001D8A07FEF5CF00E
:10B8E000D8A47AEF5CF0680E0101445D0001D8A095
:10B8F0007FEF5CF0680E0101445F010E455B0001C3
:10B9000004EE1EF0D89001012335E926000EEA224C
:10B9100044C1EEFF45C1EFFF0A013F2B0901FA9533
:10B920000001D8960901FAB5D8860001D8B6AEEF65
:10B930005CF000EE42F00A013F51EB500B6E2C0E12
:10B940000B5C0001D8A4AAEF5CF00901FA850001A4
:10B95000ACEF5CF00A013F2B0001E2D71200DDECF6
:10B96000CEF0820E026E800E096E306A540E2F6E7B
:10B97000066805684EEC00F0D8A0F3D70A01A16F65
:10B98000640EA15D0001D8A414EF5DF00A01A56B5F
:10B99000A36BA26B00010A01A3530001D8A402EF1C
:10B9A0005DF0640E0A01A25D0001D8B002EF5DF007
:10B9B00001014B51FFEC00F00A01A351100DF3CF30
:10B9C00032F0A251100DF3CF31F0F4503226314A4B
:10B9D000322A3250FFEC00F03150FFEC00F0E4EC82
:10B9E00000F0A46FDE0EA45D0001D8A4FAEF5CF0B5
:10B9F0000A01A52B00010A01A22BD8B4A32B000138
:10BA0000D8A4C8D7820E026E400E096E306A540E5A
:10BA10002F6E066A056A200E016E0A01A55190EC90
:10BA200000F00001B3EF62F0650E0A01A15D0001B4
:10BA3000D8A493EF5DF00A01A56BA36BA26B000184
:10BA40000A01A3530001D8A457EF5DF0640E0A0168
:10BA5000A25D0001D8B057EF5DF001014B51FFEC42
:10BA600000F00A01A351100DF3CF32F0A251100DD6
:10BA7000F3CF31F0F4503226314A322A3250FFEC03
:10BA800000F03150FFEC00F0E4EC00F0A46FDE0EAB
:10BA9000A45D0001D8A44FEF5DF00A01A52B0001C1
:10BAA0000A01A22BD8B4A32B0001D8A4C8D70A013D
:10BAB000A551100DF3CF31F0F4CF32F031040B6EFD
:10BAC000000E32580C6EA36BA26B00010A01A2514A
:10BAD0000B5CA3510C580001D8A091EF5DF001015F
:10BAE0004B51FFEC00F00A01A351FFEC00F0A25112
:10BAF000FFEC00F0E4EC00F0A46F820E026E400E4A
:10BB0000096E306A540E2F6E066A056A200E016EA9
:10BB1000A45190EC00F0A22BD8B4A32B0001D8A420
:10BB2000D4D7B3EF62F0660E0A01A15D0001D8A47C
:10BB3000A2EF5DF0DDECCEF00A0E8C6FB8EF32F0C4
:10BB4000B3EF62F0670E0A01A15D0001D8A4EBEF2C
:10BB50005DF00A01A36BA26B00010A01A24BA32BAB
:10BB6000A3530001D8A4BCEF5DF00B0E0A01A25D47
:10BB70000001D8A0BDEF5DF0F4D6820E026E800EFB
:10BB8000096E306A540E2F6E130E066E880E056E07
:10BB90004EEC00F0D8A0E0D70A01A16FA1CADEFFE9
:10BBA000000175EC66F0FF0EDB50DD520901FA8BE7
:10BBB000E8A0FA9B820E026E400E096E306A540EA7
:10BBC0002F6E066A056A200E016E7B0E90EC00F067
:10BBD0000001B3EF62F0680E0A01A15D0001D8A474
:10BBE00011EF5FF0820E026E800E096E306A540E05
:10BBF0002F6E130E066E880E056E4EEC00F0D8A068
:10BC0000B0D60101316F820E026E800E096E306A6D
:10BC1000540E2F6E130E066E880E056E4EEC00F05D
:10BC20000001D8A09ED60101306F820E026E800EF8
:10BC3000096E306A540E2F6E130E066E880E056E56
:10BC40004EEC00F00001D8A08CD60101326F820EBC
:10BC5000026E800E096E306A540E2F6E130E066E41
:10BC6000880E056E4EEC00F00001D8A07AD60101D6
:10BC7000336F820E026E800E096E306A540E2F6E84
:10BC8000130E066E880E056E4EEC00F00001D8A073
:10BC900068D60101346F820E026E800E096E306A22
:10BCA000540E2F6E130E066E880E056E4EEC00F0CD
:10BCB0000001D8A056D601013B6F820E026E800EA5
:10BCC000096E306A540E2F6E130E066E880E056EC6
:10BCD0004EEC00F00001D8A044D601013A6F820E6C
:10BCE000026E800E096E306A540E2F6E130E066EB1
:10BCF000880E056E4EEC00F00001D8A032D601018E
:10BD0000396F820E026E800E096E306A540E2F6EED
:10BD1000130E066E880E056E4EEC00F00001D8A0E2
:10BD200020D60101466FAA6A460EA96E315146EC33
:10BD300001F00A0E54EC01F0AA6A4C0EA96E3051C3
:10BD400046EC01F00A0E54EC01F0AA6A470EA96E07
:10BD5000325146EC01F00A0E54EC01F0AA6A480E8A
:10BD6000A96E335146EC01F00A0E54EC01F0AA6AB8
:10BD7000490EA96E345146EC01F00A0E54EC01F064
:10BD8000AA6A4D0EA96E3B5146EC01F00A0E54EC26
:10BD900001F0AA6A4E0EA96E3A5146EC01F00A0E65
:10BDA00054EC01F0AA6A4B0EA96E395146EC01F031
:10BDB0000A0E54EC01F0AA6A4A0EA96E465146ECEE
:10BDC00001F00A0E54EC01F0820E026E400E096E74
:10BDD000306A540E2F6E066A056A200E016EFF0E41
:10BDE00090EC00F0010E335D0001D8A402EF5FF08B
:10BDF00001013251020DF3CFCDF0F4CFCEF00001AE
:10BE00000FEF5FF0010132513C0DF3CF31F0F4CF71
:10BE100032F0D89031340001CD6F3234CE6FB3EFB1
:10BE200062F0690E0A01A15D0001D8A446EF5FF03F
:10BE3000820E026E400E096E306A540E2F6E066A34
:10BE4000056A200E016E0101255190EC00F0820E72
:10BE5000026E400E096E306A540E2F6E066A056A35
:10BE6000200E016E265190EC00F0820E026E400E04
:10BE7000096E306A540E2F6E066A056A200E016E36
:10BE8000245190EC00F00001B3EF62F06A0E0A0159
:10BE9000A15D0001D8A4F3EF5FF0460E3DEC01F088
:10BEA0000101316F820E026E400E096E306A540E2F
:10BEB0002F6E066A056A200E016E315190EC00F07B
:10BEC0004C0E3DEC01F0306F820E026E400E096E9A
:10BED000306A540E2F6E066A056A200E016E3051CC
:10BEE00090EC00F0470E3DEC01F0326F820E026ED6
:10BEF000400E096E306A540E2F6E066A056A200ED7
:10BF0000016E325190EC00F0480E3DEC01F0336FC1
:10BF1000820E026E400E096E306A540E2F6E066A53
:10BF2000056A200E016E335190EC00F0490E3DEC95
:10BF300001F0346F820E026E400E096E306A540EAC
:10BF40002F6E066A056A200E016E345190EC00F0E7
:10BF50004D0E3DEC01F03B6F820E026E400E096EFD
:10BF6000306A540E2F6E066A056A200E016E3B5130
:10BF700090EC00F04E0E3DEC01F03A6F820E026E36
:10BF8000400E096E306A540E2F6E066A056A200E46
:10BF9000016E3A5190EC00F04B0E3DEC01F0396F20
:10BFA000820E026E400E096E306A540E2F6E066AC3
:10BFB000056A200E016E395190EC00F04A0E3DECFE
:10BFC00001F0466F820E026E400E096E306A540E0A
:10BFD0002F6E066A056A200E016E465190EC00F045
:10BFE0000001B3EF62F06B0E0A01A15D0001D8A45D
:10BFF00018EF60F0D7EC67F0820E026E400E096E0B
:10C00000306A540E2F6E066A056A200E016EFF0E0E
:10C0100090EC00F00801286BAA6A450EA96E285121
:10C0200046EC01F00A0E54EC01F00001B3EF62F0AF
:10C030006C0E0A01A15D0001D8A439EF60F0DE6A40
:10C04000DE6AFA0EDE6E160EDE6E060EDE6EE4ECB4
:10C05000A8F0820E026E400E096E306A540E2F6EEA
:10C06000066A056A200E016ECC0E90EC00F0B3EF6C
:10C0700062F06D0E0A01A15D0001D8A444EF60F0EA
:10C0800003EC68F0B3EF62F06E0E0A01A15D0001EF
:10C09000D8A471EF60F0640E0A01A66F0001D20E01
:10C0A0000A01A65D0001D8B06FEF60F0AA6AA6CAC7
:10C0B000A9FF3FEC01F00A01A76F820E026E400E4D
:10C0C000096E306A540E2F6E066A056A200E016EE4
:10C0D000A75190EC00F0A62B0001D8A4DFD7B3EF56
:10C0E00062F06F0E0A01A15D0001D8A4E1EF60F0DB
:10C0F0000A01A86B00010A01A82B0B0EA85D000124
:10C10000D8A491EF60F0820E026E400E096E306A84
:10C11000540E2F6E066A056A200E016ED20E90EC48
:10C1200000F00B0E0A01A85D0001D8B0DFEF60F04F
:10C13000640E0A01A66F0001D20E0A01A65D00017D
:10C14000D8B0D1EF60F0820E026E400E096E306AF8
:10C15000540E2F6E066A056A200E016E0A01A65162
:10C1600090EC00F0820E026E800E096E306A540E62
:10C170002F6E070E066ED00E056E4EEC00F000011D
:10C18000D8A0B8D70A01A76FAA6AA6CAA9FFA75163
:10C1900046EC01F00A0E54EC01F0A62B0001D8A4E5
:10C1A000CAD7820E026E400E096E306A540E2F6E90
:10C1B000066A056A200E016EDE0E90EC00F0B3EF09
:10C1C00062F0700E0A01A15D0001D8A4EAEF60F0F0
:10C1D000B3EF62F0710E0A01A15D0001D8A434EF43
:10C1E00061F00A01A36B0F0EA26F00010A01A353B5
:10C1F0000001D8A424EF61F00A01A2290001D8B4FB
:10C2000024EF61F0A3CAAAFFA2CAA9FFFF0E46EC61
:10C2100001F00A0E54EC01F0820E026E400E096E1F
:10C22000306A540E2F6E066A056A200E016E0A01EE
:10C23000A25190EC00F0A35190EC00F0A22BD8B4E6
:10C24000A32B0001D8A4D1D7820E026E400E096E36
:10C25000306A540E2F6E066A056A200E016EFE0EBD
:10C2600090EC00F0B3EF62F0720E0A01A15D0001E4
:10C27000D8A4BFEF61F00A01A36BA26B0001FF0E0F
:10C280000A01A35D0001D8A050EF61F0D8A475EFBA
:10C2900061F0FF0E0A01A25D0001D8B075EF61F0F8
:10C2A00001014C51FFEC00F00A01A351FFEC00F03A
:10C2B000A251FFEC00F0FF0EFDEC00F00A0E54EC72
:10C2C00001F0820E026E400E096E306A540E2F6E1F
:10C2D000066A056A200E016E010E90EC00F0A22B9A
:10C2E000D8B4A32B0001D8A4C9D70A01A36BA26BB1
:10C2F0000001FF0E0A01A35D0001D8A08AEF61F0E2
:10C30000D8A4AFEF61F0FF0E0A01A25D0001D8B022
:10C31000AFEF61F001014E51FFEC00F00A01A351B3
:10C32000FFEC00F0A251FFEC00F0FF0EFDEC00F07E
:10C330000A0E54EC01F0820E026E400E096E306A55
:10C34000540E2F6E066A056A200E016E010E90ECE7
:10C3500000F0A22BD8B4A32B0001D8A4C9D7820E19
:10C36000026E400E096E306A540E2F6E066A056A20
:10C37000200E016EFE0E90EC00F0B3EF62F0730E33
:10C380000A01A15D0001D8A444EF62F00A01A36B89
:10C39000A26B0001FF0E0A01A35D0001D8A0DBEF34
:10C3A00061F0D8A4FDEF61F0FF0E0A01A25D00016B
:10C3B000D8B0FDEF61F001014C51FFEC00F00A0133
:10C3C000A351FFEC00F0A251FFEC00F0E4EC00F010
:10C3D000A46F820E026E400E096E306A540E2F6EEC
:10C3E000066A056A200E016EA45190EC00F0A22BA3
:10C3F000D8B4A32B0001D8A4CCD70A01A36BA26B9D
:10C400000001FF0E0A01A35D0001D8A012EF62F047
:10C41000D8A434EF62F0FF0E0A01A25D0001D8B08B
:10C4200034EF62F001014E51FFEC00F00A01A3511C
:10C43000FFEC00F0A251FFEC00F0E4EC00F0A46F80
:10C44000820E026E400E096E306A540E2F6E066A1E
:10C45000056A200E016EA45190EC00F0A22BD8B416
:10C46000A32B0001D8A4CCD7820E026E400E096E19
:10C47000306A540E2F6E066A056A200E016E7B0E1E
:10C4800090EC00F0B3EF62F0740E0A01A15D0001C0
:10C49000D8A47EEF62F00A01A66B0001FF0E0A012C
:10C4A000A65D0001D8B06EEF62F0AA6AA6CAA9FF25
:10C4B0003FEC01F00A01A46F820E026E400E096E7D
:10C4C000306A540E2F6E066A056A200E016EA45162
:10C4D00090EC00F0A62B0001D8A4DFD7820E026EEC
:10C4E000400E096E306A540E2F6E066A056A200EE1
:10C4F000016E7B0E90EC00F0B3EF62F0750E0A0156
:10C50000A15D0001D8A4B2EF62F0820E026E800E2F
:10C51000096E306A540E2F6E070E066ED00E056E31
:10C520004EEC00F0D8A0F1D70A01A46FAA6A020E5F
:10C53000A96EA45146EC01F00A0E54EC01F0A46976
:10C54000020E3DEC01F0A46F820E026E400E096EE9
:10C55000306A540E2F6E066A056A200E016EA451D1
:10C5600090EC00F00001B1EF5CF012000A01B66B34
:10C57000B56BAB6BAA6B0001060E0A01AB5D000147
:10C58000D8A0CDEF62F0D8A4ECEF62F0400E0A0123
:10C59000AA5D0001D8B0ECEF62F001014B51FFEC55
:10C5A00000F00A01AB51FFEC00F0AA51FFEC00F0E3
:10C5B000E4EC00F0A96FDE0EA95D0001D8A4E5EF60
:10C5C00062F0ABCAB6FAAACAB5FA0A01AA2BD8B465
:10C5D000AB2B0001D8A4CFD70A01B651B511000189
:10C5E000D8A4F7EF62F0F8EC64F0F7EF64F0010123
:10C5F0004B51FFEC00F00B0E0A01B525316E000E19
:10C60000B621326E3250FFEC00F03150FFEC00F0FA
:10C61000E4EC00F0B86FB8CABEF001014B51FFEC7A
:10C6200000F00C0E0A01B525316E000EB621326EF7
:10C630003250FFEC00F03150FFEC00F0E4EC00F081
:10C64000B96FB9CABDF001014B51FFEC00F00D0EFE
:10C650000A01B525316E000EB621326E3250FFEC64
:10C6600000F03150FFEC00F0E4EC00F0BA6FBACA11
:10C67000BCF001014B51FFEC00F00E0E0A01B52594
:10C68000316E000EB621326E3250FFEC00F03150A8
:10C69000FFEC00F0E4EC00F0BB6FBBCABBF0D89637
:10C6A0000001BEBFD886D8B66FEF63F0F30EBB5D56
:10C6B000FF0EBC59010EBD59000EBE59D8A06FEF38
:10C6C00063F0010EB96FAA6A450EA96E010E46EC21
:10C6D00001F0010E0801286F0001F6EF64F001017E
:10C6E0004B51FFEC00F00A01B505316E000EB65952
:10C6F000326E3250FFEC00F03150FFEC00F0E4EC11
:10C7000000F0A96FA92B01014C51FFEC00F00F0EB6
:10C710000A01B525316E000EB621326E3250FFECA3
:10C7200000F03150FFEC00F0A951FDEC00F0050ED7
:10C7300054EC01F001014C51FFEC00F0100E0A0125
:10C74000B525316E000EB621326E3250FFEC00F08E
:10C750003150FFEC00F0DE0EFDEC00F0050E54EC65
:10C7600001F001014F510A0DF3CF31F0F4CF32F057
:10C77000505131240A01BC6F01014C51FFEC00F013
:10C78000110E0A01B525316E000EB621326E3250FF
:10C79000FFEC00F03150FFEC00F0BC51FDEC00F07C
:10C7A000050E54EC01F0010151510A0DF3CF31F0A7
:10C7B000F4CF32F0525131240A01BC6F01014C51C7
:10C7C000FFEC00F0120E0A01B525316E000EB62105
:10C7D000326E3250FFEC00F03150FFEC00F0BC51F3
:10C7E000FDEC00F0050E54EC01F0010153510A0D6F
:10C7F000F3CF31F0F4CF32F0545131240A01BC6F41
:10C8000001014C51FFEC00F0130E0A01B525316E09
:10C81000000EB621326E3250FFEC00F03150FFECCA
:10C8200000F0BC51FDEC00F0050E54EC01F00101EC
:10C8300072510A0DF3CF31F0F4CF32F0735131243D
:10C840000A01BC6F01014C51FFEC00F0140E0A010B
:10C85000B525316E000EB621326E3250FFEC00F07D
:10C860003150FFEC00F0BC51FDEC00F0050E54EC33
:10C8700001F0010174510A0DF3CF31F0F4CF32F021
:10C88000755131240A01BC6F01014C51FFEC00F0DD
:10C89000150E0A01B525316E000EB621326E3250EA
:10C8A000FFEC00F03150FFEC00F0BC51FDEC00F06B
:10C8B000050E54EC01F0010176510A0DF3CF31F071
:10C8C000F4CF32F0775131240A01BC6F01014C5191
:10C8D000FFEC00F0160E0A01B525316E000EB621F0
:10C8E000326E3250FFEC00F03150FFEC00F0BC51E2
:10C8F000FDEC00F0050E54EC01F00001BB2B000E26
:10C90000BC23BD23BE23BEC0B8FABDC0B9FABCC0AB
:10C91000BAFABBC0BBFABB07000EBC5BBD5BBE5B1B
:10C920001B0E0A01B5250001BF6F000E0A01B621DA
:10C930000001C06F01014C51FFEC00F0170E0A011D
:10C94000B525316E000EB621326E3250FFEC00F08C
:10C950003150FFEC00F0B851FDEC00F0050E54EC46
:10C9600001F001014C51FFEC00F0180E0A01B52551
:10C97000316E000EB621326E3250FFEC00F03150B5
:10C98000FFEC00F0B951FDEC00F0050E54EC01F0A5
:10C9900001014C51FFEC00F0190E0A01B525316E72
:10C9A000000EB621326E3250FFEC00F03150FFEC39
:10C9B00000F0BA51FDEC00F0050E54EC01F001015D
:10C9C0004C51FFEC00F01A0E0A01B525316E000E35
:10C9D000B621326E3250FFEC00F03150FFEC00F027
:10C9E000BB51FDEC00F0050E54EC01F0000112000B
:10C9F000A30E0A01BE6FA20EBF6FC16BC06BBF5109
:10CA0000FFEC00F0C151FFEC00F0C051FFEC00F072
:10CA1000010EFDEC00F0050E54EC01F0BE51FFECF0
:10CA200000F0C151FFEC00F0C051FFEC00F0E4EC6D
:10CA300000F0C26FBF51FFEC00F0010EC025316E57
:10CA4000000EC121326E3250FFEC00F03150FFEC8D
:10CA500000F0DE0EFDEC00F0050E54EC01F0BE51CE
:10CA6000FFEC00F0010EC025316E000EC121326EC8
:10CA70003250FFEC00F03150FFEC00F0E4EC00F03D
:10CA8000C26F01014F510A0DF3CF31F0F4CF32F0F4
:10CA9000505131240A01C36FBF51FFEC00F0020E68
:10CAA000C025316E000EC121326E3250FFEC00F015
:10CAB0003150FFEC00F0C351FDEC00F0050E54ECDA
:10CAC00001F0010151510A0DF3CF31F0F4CF32F0F2
:10CAD000525131240A01C36FBF51FFEC00F0030E25
:10CAE000C025316E000EC121326E3250FFEC00F0D5
:10CAF0003150FFEC00F0C351FDEC00F0050E54EC9A
:10CB000001F0010153510A0DF3CF31F0F4CF32F0AF
:10CB1000545131240A01C36FBF51FFEC00F0040EE1
:10CB2000C025316E000EC121326E3250FFEC00F094
:10CB30003150FFEC00F0C351FDEC00F0050E54EC59
:10CB400001F0010172510A0DF3CF31F0F4CF32F050
:10CB5000735131240A01C36FBF51FFEC00F0050E81
:10CB6000C025316E000EC121326E3250FFEC00F054
:10CB70003150FFEC00F0C351FDEC00F0050E54EC19
:10CB800001F0010174510A0DF3CF31F0F4CF32F00E
:10CB9000755131240A01C36FBF51FFEC00F0060E3E
:10CBA000C025316E000EC121326E3250FFEC00F014
:10CBB0003150FFEC00F0C351FDEC00F0050E54ECD9
:10CBC00001F0010176510A0DF3CF31F0F4CF32F0CC
:10CBD000775131240A01C36FBF51FFEC00F0070EFB
:10CBE000C025316E000EC121326E3250FFEC00F0D4
:10CBF0003150FFEC00F0C351FDEC00F0050E54EC99
:10CC000001F0B06BAF6B060EAE6F400EAD6FB0CAE9
:10CC1000C3FABF51FFEC00F0080EC025316E000EC4
:10CC2000C121326E3250FFEC00F03150FFEC00F0C9
:10CC3000C351FDEC00F0050E54EC01F0AFCAC3FA8D
:10CC4000BF51FFEC00F0090EC025316E000EC1216E
:10CC5000326E3250FFEC00F03150FFEC00F0C35167
:10CC6000FDEC00F0050E54EC01F0AECAC3FABF5162
:10CC7000FFEC00F00A0EC025316E000EC121326EAD
:10CC80003250FFEC00F03150FFEC00F0C351FDECEE
:10CC900000F0050E54EC01F0ADCAC3FABF51FFEC31
:10CCA00000F00B0EC025316E000EC121326E3250E5
:10CCB000FFEC00F03150FFEC00F0C351FDEC00F050
:10CCC000050E54EC01F00001BE6BBD6B060EBC6F8F
:10CCD0003F0EBB6F0C0E0A01C0250001BF6F000E96
:10CCE0000A01C1210001C06F1200A30E0A01CD6F1D
:10CCF000A20ECE6FAB0ECF6FAA0ED06FFF0EDBCFA2
:10CD0000C4FADD520901FA9D0A01C451100DF3CF96
:10CD100031F0F4CF32F0080E315CE26F000E325881
:10CD2000E36FCD51FFEC00F0E351FFEC00F0E25176
:10CD3000FFEC00F0E4EC00F0DA6FC451100DF3CF1B
:10CD400031F0F4CF32F0070E315CE26F000E325852
:10CD5000E36FCD51FFEC00F0E351FFEC00F0E25146
:10CD6000FFEC00F0E4EC00F0DB6FC451100DF3CFEA
:10CD700031F0F4CF32F0060E315CE26F000E325823
:10CD8000E36FCD51FFEC00F0E351FFEC00F0E25116
:10CD9000FFEC00F0E4EC00F0DC6FC451100DF3CFB9
:10CDA00031F0F4CF32F0050E315CE26F000E3258F4
:10CDB000E36FCD51FFEC00F0E351FFEC00F0E251E6
:10CDC000FFEC00F0E4EC00F0DD6FDACAC8FADBCA71
:10CDD000C7FADCCAC6FADDCAC5FAC451100DF3CFD2
:10CDE00031F0F4CF32F0040E315CE26F000E3258B5
:10CDF000E36FCD51FFEC00F0E351FFEC00F0E251A6
:10CE0000FFEC00F0E4EC00F0DA6FC451100DF3CF4A
:10CE100031F0F4CF32F0030E315CE26F000E325885
:10CE2000E36FCD51FFEC00F0E351FFEC00F0E25175
:10CE3000FFEC00F0E4EC00F0DB6FC451100DF3CF19
:10CE400031F0F4CF32F0020E315CE26F000E325856
:10CE5000E36FCD51FFEC00F0E351FFEC00F0E25145
:10CE6000FFEC00F0E4EC00F0DC6FC451100DF3CFE8
:10CE700031F0F4CF32F03104E26F000E3258E36F3C
:10CE8000CD51FFEC00F0E351FFEC00F0E251FFEC7C
:10CE900000F0E4EC00F0DD6FDACACCFADBCACBFAC2
:10CEA000DCCACAFADDCAC9FAC8CAD9FAC7CAD8FAE6
:10CEB000C6CAD7FAC5CAD6FA00010A01D651C95D59
:10CEC000D751CA59D851CB59D951CC59D951CC196C
:10CED000D8B0800A0001D8A8CFEF67F0D8960A0131
:10CEE000D9BFD8860001D8B6A6EF67F00A01D9539A
:10CEF0000AE1D85108E1FF0ED65DFF0ED7590001B7
:10CF0000D8A0A6EF67F00A01D629E26F000ED7215C
:10CF1000E36FCF51FFEC00F0E351FFEC00F0E25182
:10CF2000FFEC00F0E4EC00F0D56F820E026E400ED4
:10CF3000096E306A540E2F6E066A056A200E016E65
:10CF4000D55190EC00F00001C5EF67F0D7CAE3FAC5
:10CF5000D6CAE2FA0A01CD51FFEC00F0E351FFEC32
:10CF600000F0E251FFEC00F0E4EC00F0D56F820E2F
:10CF7000026E400E096E306A540E2F6E066A056A04
:10CF8000200E016ED55190EC00F000010A01D62B65
:10CF9000000ED723D823D9230001D8A08DD70901AB
:10CFA000FA8DE86AFABD010EDE6E000112000A0178
:10CFB000E96BE86B0001060E0A01E95D0001D8A0EB
:10CFC000ECEF67F0D8A402EF68F0400E0A01E85DCC
:10CFD0000001D8B002EF68F0A20EFFEC00F00A01E9
:10CFE000E951FFEC00F0E851FFEC00F0000EFDEC21
:10CFF00000F0050E54EC01F0E82BD8B4E92B000149
:10D00000D8A4D8D712000A01EC6BEB6B00017F0E9D
:10D010000A01EC5D0001D8A018EF68F0D8A459EF20
:10D0200068F0F00E0A01EB5D0001D8B059EF68F02E
:10D03000820E026E800E096E306A540E2F6E130E31
:10D04000066E880E056E4EEC00F0D8A0B1EF5CF0D5
:10D050000A01EA6FA00EFFEC00F0EC51FFEC00F0CB
:10D06000EB51FFEC00F0EA51FDEC00F00A0E54EC3D
:10D0700001F0A10EFFEC00F0EC51FFEC00F0EB51E1
:10D08000FFEC00F0E4EC00F0ED6F820E026E400E5B
:10D09000096E306A540E2F6E066A056A200E016E04
:10D0A000ED5190EC00F0EB2BD8B4EC2B0001D8A4A0
:10D0B000ADD71200DDECCEF00A01EE6B640EF06F1E
:10D0C0000001C80E0A01F05D0001D8B07CEF68F0E5
:10D0D000AA6AF0CAA9FF3FEC01F00A01FB6FFB2925
:10D0E0000001D8A476EF68F0F0CAEEFA0B0E0A0140
:10D0F000F0270001D8A0E4D70A01EE530001D8B40C
:10D100001EEF6CF0206AEECA1FF0000E75EC01F005
:10D110000A01EF6FDE6ADE6A030EDE6E110EDE6E4E
:10D12000070EDE6E0001E4ECA8F0EFCADEFF4D0E44
:10D13000DE6E060EDE6EBBECCCF0DE6ADE6A710ED1
:10D14000DE6E630EDE6E070EDE6EE4ECA8F0A0C0AD
:10D1500022F09FC021F09EC020F09DC01FF02A6ADF
:10D16000296A286A0A0E276E02EC02F022C034F007
:10D1700021C033F020C032F01FC031F034C022F0A3
:10D1800033C021F032C020F031C01FF02A6A296A72
:10D19000286A060E276E8BEC01F022C0F8FA21C037
:10D1A000F7FA20C0F6FA1FC0F5FA226A216A206A4F
:10D1B000D1C01FF02A6A0F0E296E420E286E400E53
:10D1C000276E02EC02F022C034F021C033F020C000
:10D1D00032F01FC031F031500A01F5273250F623EA
:10D1E0003350F7233450F8239CC022F09BC021F029
:10D1F0009AC020F099C01FF02A6A296A286A0A0E8C
:10D20000276E02EC02F022C034F021C033F020C0BF
:10D2100032F01FC031F034C022F033C021F032C0F0
:10D2200020F031C01FF02A6A296A286A060E276E8C
:10D230008BEC01F022C0F4FA21C0F3FA20C0F2FA1C
:10D240001FC0F1FA226A216A206AD0C01FF02A6A40
:10D250000F0E296E420E286E400E276E02EC02F071
:10D2600022C034F021C033F020C032F01FC031F0B2
:10D270003150F1273250F2233350F3233450F4234A
:10D28000F96BFA6BF8CA22F0F7CA21F0F6CA20F05F
:10D29000F5CA1FF0010E7FEC01F0F96FF8CA22F019
:10D2A000F7CA21F0F6CA20F0F5CA1FF0000E7FEC95
:10D2B00001F0FA6FF9510A0DF3CF31F0F4CF32F0EB
:10D2C000FA513124FB6F040EEE25AA6AA96EAA3624
:10D2D000FB5146EC01F00A0E54EC01F0040EEE2571
:10D2E000AA6AA96EAA363FEC01F0FB6FF8CA22F0D9
:10D2F000F7CA21F0F6CA20F0F5CA1FF02A6A296A97
:10D30000286A640E276E8BEC01F022C0F8FA21C067
:10D31000F7FA20C0F6FA1FC0F5FAF96BFA6BF8CAF3
:10D3200022F0F7CA21F0F6CA20F0F5CA1FF0010E6C
:10D330007FEC01F0F96FF8CA22F0F7CA21F0F6CAC3
:10D3400020F0F5CA1FF0000E7FEC01F0FA6FF951E2
:10D350000A0DF3CF31F0F4CF32F0FA513124FB6FE4
:10D36000030EEE25AA6AA96EAA36FB5146EC01F01F
:10D370000A0E54EC01F0030EEE25AA6AA96EAA3635
:10D380003FEC01F0FB6FF8CA22F0F7CA21F0F6CAB1
:10D3900020F0F5CA1FF02A6A296A286A640E276EEF
:10D3A0008BEC01F022C0F8FA21C0F7FA20C0F6FA9F
:10D3B0001FC0F5FAF96BFA6BF8CA22F0F7CA21F030
:10D3C000F6CA20F0F5CA1FF0010E7FEC01F0F96FEC
:10D3D000F8CA22F0F7CA21F0F6CA20F0F5CA1FF009
:10D3E000000E7FEC01F0FA6FF9510A0DF3CF31F026
:10D3F000F4CF32F0FA513124FB6F020EEE25AA6A07
:10D40000A96EAA36FB5146EC01F00A0E54EC01F06D
:10D41000020EEE25AA6AA96EAA363FEC01F0FB6F58
:10D42000F8CA22F0F7CA21F0F6CA20F0F5CA1FF0B8
:10D430002A6A296A286A640E276E8BEC01F022C0E2
:10D44000F8FA21C0F7FA20C0F6FA1FC0F5FAF96B16
:10D45000FA6BF8CA22F0F7CA21F0F6CA20F0F5CA32
:10D460001FF0010E7FEC01F0F96FF8CA22F0F7CA45
:10D4700021F0F6CA20F0F5CA1FF0000E7FEC01F093
:10D48000FA6FF9510A0DF3CF31F0F4CF32F0FA51BF
:10D490003124FB6FEE29A96E000EAA6AAA22FB5165
:10D4A00046EC01F00A0E54EC01F0EE29A96E000ED4
:10D4B000AA6AAA223FEC01F0FB6FF8CA22F0F7CA71
:10D4C00021F0F6CA20F0F5CA1FF02A6A296A286AF4
:10D4D000640E276E8BEC01F022C0F8FA21C0F7FA37
:10D4E00020C0F6FA1FC0F5FAFA6BF8CA22F0F7CAA4
:10D4F00021F0F6CA20F0F5CA1FF0000E7FEC01F013
:10D50000FA6FFACAFBFAAA6AEECAA9FFFB5146EC07
:10D5100001F00A0E54EC01F0AA6AEECAA9FF3FEC32
:10D5200001F0FB6FF96BFA6BF4CA22F0F3CA21F039
:10D53000F2CA20F0F1CA1FF0010E7FEC01F0F96F82
:10D54000F4CA22F0F3CA21F0F2CA20F0F1CA1FF0A7
:10D55000000E7FEC01F0FA6FF9510A0DF3CF31F0B4
:10D56000F4CF32F0FA513124FB6F080EEE25AA6A8F
:10D57000A96EAA36FB5146EC01F00A0E54EC01F0FC
:10D58000080EEE25AA6AA96EAA363FEC01F0FB6FE1
:10D59000F4CA22F0F3CA21F0F2CA20F0F1CA1FF057
:10D5A0002A6A296A286A640E276E8BEC01F022C071
:10D5B000F4FA21C0F3FA20C0F2FA1FC0F1FAF96BB5
:10D5C000FA6BF4CA22F0F3CA21F0F2CA20F0F1CAD1
:10D5D0001FF0010E7FEC01F0F96FF4CA22F0F3CADC
:10D5E00021F0F2CA20F0F1CA1FF0000E7FEC01F02A
:10D5F000FA6FF9510A0DF3CF31F0F4CF32F0FA514E
:10D600003124FB6F070EEE25AA6AA96EAA36FB51DC
:10D6100046EC01F00A0E54EC01F0070EEE25AA6A62
:10D62000A96EAA363FEC01F0FB6FF4CA22F0F3CAF0
:10D6300021F0F2CA20F0F1CA1FF02A6A296A286A8A
:10D64000640E276E8BEC01F022C0F4FA21C0F3FACD
:10D6500020C0F2FA1FC0F1FAF96BFA6BF4CA22F09B
:10D66000F3CA21F0F2CA20F0F1CA1FF0010E7FECDC
:10D6700001F0F96FF4CA22F0F3CA21F0F2CA20F0E7
:10D68000F1CA1FF0000E7FEC01F0FA6FF9510A0D9C
:10D69000F3CF31F0F4CF32F0FA513124FB6F060EA4
:10D6A000EE25AA6AA96EAA36FB5146EC01F00A0ED5
:10D6B00054EC01F0060EEE25AA6AA96EAA363FECDC
:10D6C00001F0FB6FF4CA22F0F3CA21F0F2CA20F095
:10D6D000F1CA1FF02A6A296A286A640E276E8BEC49
:10D6E00001F022C0F4FA21C0F3FA20C0F2FA1FC000
:10D6F000F1FAF96BFA6BF4CA22F0F3CA21F0F2CA1C
:10D7000020F0F1CA1FF0010E7FEC01F0F96FF4CAAE
:10D7100022F0F3CA21F0F2CA20F0F1CA1FF0000E85
:10D720007FEC01F0FA6FF9510A0DF3CF31F0F4CF2D
:10D7300032F0FA513124FB6F050EEE25AA6AA96E6C
:10D74000AA36FB5146EC01F0050EEE25AA6AA96E39
:10D75000AA363FEC01F0FB6F0A0E54EC01F0570EB5
:10D760000101685D0001D8A4CDEF6BF0090E0A013C
:10D77000EE25AA6AA96EAA36010E46EC01F00A0E41
:10D7800054EC01F0090EEE25AA6AA96EAA363FEC08
:10D7900001F0FB6F0001E1EF6BF0090E0A01EE25CD
:10D7A000AA6AA96EAA36000E46EC01F00A0E54ECE5
:10D7B00001F0090EEE25AA6AA96EAA363FEC01F027
:10D7C000FB6F0001530E01015E5D0001D8A400EF64
:10D7D0006CF00A0E0A01EE25AA6AA96EAA36010E9D
:10D7E00046EC01F00A0E54EC01F0090EEE25AA6A8F
:10D7F000A96EAA363FEC01F0FB6F000114EF6CF04C
:10D800000A0E0A01EE25AA6AA96EAA36000E46EC97
:10D8100001F00A0E54EC01F0090EEE25AA6AA96E79
:10D82000AA363FEC01F0FB6F00010F0E246EA00E34
:10D8300055EC01F0DDECCEF02DEF6CF00B0EDE6E52
:10D840004A0EDE6E010EDE6EBBECCCF0070E246ECF
:10D85000D00E55EC01F0DDECCEF08B831200D896A3
:10D860008BA3D886D8B636EF6CF08B8DD8968BA16B
:10D87000D886D8B676EF6CF004EE1EF0D890010191
:10D880002335E926000EEA22EECF0BF0EFCF0CF0A5
:10D890000BC0DEFF0CC0DEFF89C0DEFF8AC0DEFFEA
:10D8A000010EDE6E0001B3EC0EF01AEEFCF05BEC44
:10D8B00002F00A01FD530001D8A466EF6CF01F0EC0
:10D8C0000A01FC5D0001D8A06CEF6CF08B918B8D90
:10D8D000A7ECBFF074EF6CF0A7ECBFF0FCCADEFF62
:10D8E000FDCADEFF17ECC0F078EF6CF0CDEC0FF066
:10D8F0001200DE6ADE6A890EDE6E200EDE6EDE6AE1
:10D90000E4ECA8F0DE6ADE6A8A0EDE6E2F0EDE6EB2
:10D91000030EDE6EE4ECA8F0DE6ADE6A1C0EDE6E3C
:10D92000DE6A080EDE6EE4ECA8F0DE6ADE6AD70E70
:10D93000DE6E870EDE6E080EDE6EE4ECA8F0D89682
:10D940008BABD886D8B6B9EF6CF0DE6ADE6AA90E6A
:10D95000DE6E060EDE6E0A0EDE6EE4ECA8F0DE6A07
:10D96000DE6ADF0EDE6E3C0EDE6E0A0EDE6EE4EC6C
:10D97000A8F0DE6ADE6AC90EDE6E2B0EDE6E080EC1
:10D98000DE6EE4ECA8F00101376B0001DE6AFCEC0E
:10D990008EF09853D8A4D0EF6CF0F7D7F6EF6CF078
:10D9A000010E985DD8A4DCEF6CF00801276B000134
:10D9B000B8EF32F0F6EF6CF0040E985DD8A4EEEFFD
:10D9C0006CF0D8968BABD886D8B6EBEF6CF08BEFBB
:10D9D0006DF0ECEF6CF0D9D7F6EF6CF0020E985DBD
:10D9E000D8A4F5EF6CF0F6EF6CF0CFD7DDECCEF00D
:10D9F000AAEC0AF0010EDE6E13EC48F0D0C0B1F0D4
:10DA00001A6A7C0E196E120E186E920E176E99C05D
:10DA100013F09AC014F09BC015F09CC016F05CEC9B
:10DA200009F050EC08F016C0A4F015C0A3F014C023
:10DA3000A2F013C0A1F0D05158EC09F0A4C01AF024
:10DA4000A3C019F0A2C018F0A1C017F0B6EC07F0FF
:10DA500016C0A4F015C0A3F014C0A2F013C0A1F02A
:10DA6000530E01015E5D0001D8A439EF6DF0800E08
:10DA7000A21BD1C0B3F01A6A7C0E196E120E186E7A
:10DA8000920E176E9DC013F09EC014F09FC015F04B
:10DA9000A0C016F05CEC09F050EC08F016C0A8F03D
:10DAA00015C0A7F014C0A6F013C0A5F0D15158ECD2
:10DAB00009F0A8C01AF0A7C019F0A6C018F0A5C0B8
:10DAC00017F0B6EC07F016C0A8F015C0A7F014C008
:10DAD000A6F013C0A5F0570E0101685D0001D8A49F
:10DAE00074EF6DF0800EA61B010E0101376FDE6A28
:10DAF000DE6A890EDE6E200EDE6EDE6A0001E4EC68
:10DB0000A8F0DE6ADE6A8A0EDE6E2F0EDE6E030E6F
:10DB1000DE6EE4ECA8F0DE6ADE6A1C0EDE6EDE6A03
:10DB2000080EDE6EE4ECA8F0DE6ADE6AD90EDE6E68
:10DB3000870EDE6E080EDE6EE4ECA8F0D8968BAB96
:10DB4000D886D8B6B8EF6DF0DE6ADE6AA90EDE6E52
:10DB5000060EDE6E0A0EDE6EE4ECA8F0DE6ADE6A09
:10DB6000DF0EDE6E3C0EDE6E0A0EDE6EE4ECA8F01A
:10DB7000DE6A010EDE6EC90EDE6E2B0EDE6E080E44
:10DB8000DE6EE4ECA8F0DE6ADE6AC70EDE6E2B0EF7
:10DB9000DE6E080EDE6EE4ECA8F0C80E54EC01F068
:10DBA000DE6AFCEC8EF09853D8A4DAEF6DF0F8D76B
:10DBB00000EF6EF0010E985DD8A4E6EF6DF008015D
:10DBC000276B0001B8EF32F000EF6EF0040E985DA5
:10DBD000D8A4F8EF6DF0D8968BABD886D8B6F5EF11
:10DBE0006DF085EF6EF0F6EF6DF0DAD700EF6EF0C6
:10DBF000030E985DD8A4FFEF6DF000EF6EF0D0D764
:10DC0000DDECCEF0AAEC0AF0010EDE6E13EC48F06B
:10DC100045C1D4F044C1D3F0D0C0B2F01A6A7C0E32
:10DC2000196E120E186E920E176E99C013F09AC0EC
:10DC300014F09BC015F09CC016F05CEC09F050ECA1
:10DC400008F016C0ACF015C0ABF014C0AAF013C0B9
:10DC5000A9F0D05158EC09F0ACC01AF0ABC019F0E3
:10DC6000AAC018F0A9C017F0B6EC07F016C0ACF0C7
:10DC700015C0ABF014C0AAF013C0A9F0530E0101F7
:10DC80005E5D0001D8A447EF6EF0800EAA1BD1C0E4
:10DC9000B4F01A6A7C0E196E120E186E920E176E80
:10DCA0009DC013F09EC014F09FC015F0A0C016F0E8
:10DCB0005CEC09F050EC08F016C0B0F015C0AFF005
:10DCC00014C0AEF013C0ADF0D15158EC09F0B0C0A3
:10DCD0001AF0AFC019F0AEC018F0ADC017F0B6EC36
:10DCE00007F016C0B0F015C0AFF014C0AEF013C00E
:10DCF000ADF0570E0101685D0001D8A482EF6EF00F
:10DD0000800EAE1B020E0101376F0001A1C0DEFFC5
:10DD1000A2C0DEFFA3C0DEFFA4C0DEFFA5C0DEFF01
:10DD2000A6C0DEFFA7C0DEFFA8C0DEFFA9C0DEFFE1
:10DD3000AAC0DEFFABC0DEFFACC0DEFFADC0DEFFC1
:10DD4000AEC0DEFFAFC0DEFFB0C0DEFFD2EC17F02A
:10DD50001BEE00F04AEC02F003CB22F002CB21F0E4
:10DD600001CB20F000CB1FF02A6A0F0E296E420E65
:10DD7000286E400E276E8BEC01F020C03DF11FC0D5
:10DD80003CF1226A216A3DC120F03CC11FF02A6AA1
:10DD90000F0E296E420E286E400E276E02EC02F026
:10DDA00022C034F021C033F020C032F01FC031F067
:10DDB00031500B01005D0101406F32500B010159E0
:10DDC0000101416F33500B0102590101426F345080
:10DDD0000B0103590101436F43C122F042C121F0FD
:10DDE00041C120F040C11FF02A6A296A286A640EE6
:10DDF000276E02EC02F022C043F121C042F120C0A4
:10DE000041F11FC040F13D530001D8A40FEF6FF066
:10DE1000B40E01013C5D0001D8A019EF6FF0B40E03
:10DE200001013C5D3E6F000E3D593F6F000120EF48
:10DE30006FF0B40E01013C253E6F000E3D213F6F97
:10DE40000001010E0101395D0001D8A456EF6FF009
:10DE500043C122F042C121F041C120F040C11FF076
:10DE60002A6A296A286A210E276E02EC02F022C073
:10DE700034F021C033F020C032F01FC031F034C084
:10DE800022F033C021F032C020F031C01FF02A6AE6
:10DE9000296A286A0A0E276E8BEC01F022C043F132
:10DEA00021C042F120C041F11FC040F18B83010E1F
:10DEB0000801276F00018B8B22EF35F01200DE6A1C
:10DEC000FCEC8EF0010E985DD8A476EF6FF093EC29
:10DED000D2F0D8968BB3D886D8B674EF6FF008011D
:10DEE000276B0001B8EF32F0AFEF6FF0020E985DD4
:10DEF000D8A484EF6FF08B837AECCEF0D7EC99F056
:10DF00007AECCEF0AFEF6FF0030E985DD8A492EFED
:10DF10006FF08B837AECCEF0D7EC99F07AECCEF000
:10DF2000AFEF6FF0040E985DD8A499EF6FF0AFEFEC
:10DF30006FF0050E985DD8A4AFEF6FF0D8968BB355
:10DF4000D886D8B6ADEF6FF08DC03BFA8CC08DF09F
:10DF50003BCA8CF08B8322EF35F0AFEF6FF0AAEC69
:10DF60000AF0DE6A13EC48F0BBEC70F01BEE0CF02C
:10DF70004AEC02F0D8960B010FBFD8860001D8B644
:10DF8000D7EF6FF03D0E0B010C5D860E0D59010EA3
:10DF90000E59000E0F590001D8A0D7EF6FF00B01FA
:10DFA0000F6B010E0E6F860E0D6F3C0E0C6F000195
:10DFB0000FCB22F00ECB21F00DCB20F00CCB1FF0BD
:10DFC0002A6A296A286A0A0E276E8BEC01F022C0A1
:10DFD0000FFB21C00EFB20C00DFB1FC00CFB0FCBA5
:10DFE00022F00ECB21F00DCB20F00CCB1FF0000E59
:10DFF0007FEC01F00B01066F0FCB22F00ECB21F06E
:10E000000DCB20F00CCB1FF02A6A296A286A0A0E71
:10E01000276E8BEC01F022C00FFB21C00EFB20C04D
:10E020000DFB1FC00CFB050E065D0001D8A022EF02
:10E0300070F00B010C2B000E0D230E230F2300019B
:10E0400022EF70F00B01066B086B096B0FCB22F00F
:10E050000ECB21F00DCB20F00CCB1FF0020E7FEC8D
:10E0600001F0066F0FCB22F00ECB21F00DCB20F08C
:10E070000CCB1FF0010E7FEC01F0086F0FCB22F0EC
:10E080000ECB21F00DCB20F00CCB1FF0000E7FEC5F
:10E0900001F0096F326A06CB31F03250640DF3CFD4
:10E0A00032F03150640DF3CF31F0F4503226366A3D
:10E0B00008CB35F036500A0DF3CF36F035500A0D47
:10E0C000F3CF35F0F4503626355031263650322213
:10E0D00009513124046F000E3220056FD8960101DA
:10E0E00038B1D8860001D8B682EF70F0DE6ADE6AF9
:10E0F000C50EDE6E820EDE6E090EDE6EE4ECA8F05A
:10E100008CEF70F0DE6ADE6AC30EDE6E820EDE6EAB
:10E11000090EDE6EE4ECA8F004CBDEFF05CBDEFFDB
:10E12000DE6A010EDE6EDE6A4CEC7BF0D8968BA3C5
:10E13000D886D8B6B8EF70F0010139530001D8A4E1
:10E14000AEEF70F0DE6ADE6A0C0EDE6E820EDE6E00
:10E150000D0EDE6EE4ECA8F0B8EF70F0DE6ADE6A59
:10E160000A0EDE6E820EDE6E0D0EDE6EE4ECA8F0A0
:10E170008B93A5D61200C0EC11F01BEE18F04AEC00
:10E1800002F0010E0101395D0001D8A4F6EF70F034
:10E190001BCB22F01ACB21F019CB20F018CB1FF0AB
:10E1A0002A6A296A286A210E276E02EC02F022C030
:10E1B00034F021C033F020C032F01FC031F034C041
:10E1C00022F033C021F032C020F031C01FF02A6AA3
:10E1D000296A286A0A0E276E8BEC01F022C01BFB0D
:10E1E00021C01AFB20C019FB1FC018FB0B011851DE
:10E1F0000001D55D0B01106F19510001D6590B01BB
:10E20000116F1A510001D7590B01126F1B510001F8
:10E21000D8590B01136F13CB22F012CB21F011CB85
:10E2200020F0105132EC02F0106F20C011FB21C021
:10E2300012FB22C013FB1351121111111011000116
:10E24000D8A42BEF71F03FCB13FB3ECB12FB3DCBA1
:10E2500011FB3CCB10FB13CB3FFB12CB3EFB11CB96
:10E260003DFB10CB3CFB1BCBD8F01ACBD7F019CB26
:10E27000D6F018CBD5F004EE1EF0D890010123356E
:10E28000E926000EEA22EECF0BF0EFCF0CF00BC028
:10E29000DEFF0CC0DEFFD3C0DEFFD4C0DEFFDE6ACF
:10E2A0000001B3EC0EF01BEE1CF05BEC02F0B6517B
:10E2B000640DF3CF1FFBB551640DF3CF1EFBF4507B
:10E2C0000B011F270001B851640DF3CF21FBB7519B
:10E2D000640DF3CF20FBF4500B012127236B3AC1CF
:10E2E00022FB010139530001D8A491EF71F00B0119
:10E2F00023510A0DF3CF32F022510A0DF3CF31F042
:10E30000F450322632C020F031C01FF0246A210EB2
:10E31000236EEBEC01F0226F20C023FB0001B2EF73
:10E3200071F0010E0101395D0001D8A49AEF71F07E
:10E33000B1EF71F00B0123510A0DF3CF32F02251EE
:10E340000A0DF3CF31F0F450322632C020F031C044
:10E350001FF0246A210E236EEBEC01F0226F20C027
:10E3600023FB0001D896010138A1D8860001D8B658
:10E370006DEF72F00B011D530001D8A4FEEF71F098
:10E380005B0E0B011C5D0001D8B0FEEF71F00B01BC
:10E3900022511825146F23511921156F000E1A21CF
:10E3A000166F000E1B21176F1E51145F1F51155B56
:10E3B000000E165B000E175B205114272151152308
:10E3C000000E162317231051142711511523125133
:10E3D00016231351172317CB22F016CB21F015CBA0
:10E3E00020F0145132EC02F0146F20C015FB21C054
:10E3F00016FB22C017FB00016BEF72F00B011D53DF
:10E400000001D8A40BEF72F05B0E0B011C5D000144
:10E41000D8A06AEF72F00B012251185D146F2351DE
:10E420001959156F000E1A59166F000E1B59176FE8
:10E430001E51145F1F51155B000E165B000E175B1B
:10E440002051142721511523000E16231723105194
:10E45000145D115115591251165913511759135171
:10E460001719D8B0800A0001D8B84FEF72F00B012D
:10E470001451105D146F15511159156F1651125921
:10E48000166F17511359176FE86A010138A1010F70
:10E49000D8B43891D8A43881000158EF72F00B013C
:10E4A0001051145F1151155B1251165B1351175B1C
:10E4B000000117CB22F016CB21F015CB20F00B0179
:10E4C000145132EC02F0146F20C015FB21C016FB72
:10E4D00022C017FB00011EEF73F00B011D5300015A
:10E4E000D8A47AEF72F05A0E0B011C5D0001D8A07F
:10E4F000B1EF72F00B0122511825146F235119212D
:10E50000156F000E1A21166F000E1B21176F1E517A
:10E5100014271F511523000E162317232051145FB3
:10E520002151155B000E165B000E175B105114276E
:10E5300011511523125116231351172317CB22F013
:10E5400016CB21F015CB20F0145132EC02F0146FF1
:10E5500020C015FB21C016FB22C017FB00011EEFD7
:10E5600073F00B011D530001D8A41DEF73F05A0E78
:10E570000B011C5D0001D8B01DEF73F00B0122519F
:10E58000185D146F23511959156F000E1A59166F23
:10E59000000E1B59176F1E5114271F511523000E13
:10E5A000162317232051145F2151155B000E165BB3
:10E5B000000E175B1051145D115115591251165967
:10E5C0001351175913511719D8B0800A0001D8B840
:10E5D00002EF73F00B011451105D146F15511159B6
:10E5E000156F16511259166F17511359176FE86AA4
:10E5F000010138A1010FD8B43891D8A438810001A5
:10E600000BEF73F00B011051145F1151155B125198
:10E61000165B1351175B000117CB22F016CB21F0CC
:10E6200015CB20F00B01145132EC02F0146F20C016
:10E6300015FB21C016FB22C017FB0001010E0101D2
:10E640003B5D0001D8A462EF73F0010140510B0162
:10E65000145D010141510B011559010142510B019A
:10E660001659010143510B011759010143510B0187
:10E670001719D8B0800A0001D8B862EF73F03CC116
:10E68000DEFF3DC1DEFF14CBDEFF15CBDEFF16CB78
:10E69000DEFF17CBDEFF04EE1EF0D890010123351C
:10E6A000E926000EEA22EECF0BF0EFCF0CF00BC004
:10E6B000DEFF0CC0DEFF000185EC10F01BEE14F055
:10E6C0004AEC02F00B011E5305E11F530001D8B4C0
:10E6D00095EF73F0D8960B011BBFD8860001D8B612
:10E6E00087EF73F00B011B5310E11A530EE11F511A
:10E6F000195D0001D8A087EF73F007E10B011851F5
:10E700001E5D0001D8B087EF73F0000E01D0010E3E
:10E710003B6EE86A010138B1010E3B140001D8B428
:10E7200094EF73F00101389100010B01205305E1D2
:10E7300021530001D8B4C8EF73F0D8960B011BBF6A
:10E74000D8860001D8B6BAEF73F00B011B5310E165
:10E750001A530EE12151195D0001D8A0BAEF73F0F0
:10E7600007E10B011851205D0001D8B0BAEF73F03A
:10E77000000E01D0010E3B6E010E010138B1E86AB6
:10E780003B140001D8B4C7EF73F0010138810001D8
:10E79000D896010138A1D8860001D8B603EF74F0ED
:10E7A000080130530001D8B403EF74F00801305170
:10E7B000640DF3CF3AFBF4CF3BFBD8960B0117BFA8
:10E7C000D8860001D8B603EF74F00B01175310E19F
:10E7D00016530EE13B51155D0001D8A003EF74F014
:10E7E00007E10B0114513A5D0001D8B003EF74F05A
:10E7F00008012F290001D8B403EF74F08B832FC8D0
:10E800008CF022EF35F014CBDEFF15CBDEFF16CBFC
:10E81000DEFF17CBDEFF1200FF0EDBCF50FBDD5219
:10E8200097510B0DF3CF31F0F4CF32F0640E312459
:10E830000B01656FAA6A65CBA9FF3FEC01F0416F40
:10E840006529A96E000EAA6AAA223FEC01F0426F68
:10E85000020E6525AA6AA96EAA363FEC01F0436F45
:10E86000030E6525AA6AA96EAA363FEC01F0446F33
:10E87000040E6525AA6AA96EAA363FEC01F0456F21
:10E88000050E6525AA6AA96EAA363FEC01F0466F0F
:10E89000060E6525AA6AA96EAA363FEC01F0476FFD
:10E8A000070E6525AA6AA96EAA363FEC01F0486FEB
:10E8B000080E6525AA6AA96EAA363FEC01F0496FD9
:10E8C000090E6525AA6AA96EAA363FEC01F04A6FC7
:10E8D0000A0E6525AA6AA96EAA363FEC01F04B6FB5
:10E8E00041290001D8A483EF74F00B016D6B6C6BB0
:10E8F0006B696A69716B706B766B776B786B796B30
:10E900000001E2EF76F0226A216A206A41CB1FF013
:10E91000050E2A6EF50E296EE10E286E276A02ECAE
:10E9200002F022C05CFB21C05BFB20C05AFB1FC071
:10E9300059FB226A216A206A42CB1FF02A6A0F0E15
:10E94000296E420E286E400E276E02EC02F022C0A5
:10E9500034F021C033F020C032F01FC031F031500C
:10E960000B01592732505A2333505B2334505C2318
:10E97000226A216A206A43CB1FF02A6A296A270E7D
:10E98000286E100E276E02EC02F022C034F021C077
:10E9900033F020C032F01FC031F0315059273250CF
:10E9A0005A2333505B2334505C23226A216A206A45
:10E9B00044CB1FF02A6A296A286A640E276E02EC8B
:10E9C00002F022C034F021C033F020C032F01FC06A
:10E9D00031F03150592732505A2333505B23345091
:10E9E0005C2345515925596F000E5A215A6F000E6C
:10E9F0005B215B6F000E5C215C6F010E4A5D0001C4
:10EA0000D8A40AEF75F0D880000E0B0159575A5759
:10EA10005B575C570001226A216A206A46CB1FF0CF
:10EA20002A6A0F0E296E420E286E400E276E02ECE7
:10EA300002F022C058FB21C057FB20C056FB1FC06C
:10EA400055FB226A216A206A47CB1FF02A6A296A8D
:10EA5000270E286E100E276E02EC02F022C034F052
:10EA600021C033F020C032F01FC031F031500B0113
:10EA70005527325056233350572334505823226A97
:10EA8000216A206A48CB1FF02A6A296A286A640E24
:10EA9000276E02EC02F022C034F021C033F020C017
:10EAA00032F01FC031F031505527325056233350C9
:10EAB00057233450582349515525556F000E562180
:10EAC000566F000E5721576F000E5821586F010ED8
:10EAD0004B5D0001D8A474EF75F0D880000E0B01D7
:10EAE000555756575757585700011A6A240E196E32
:10EAF000740E186E920E176E55CB13F056CB14F0A1
:10EB000057CB15F058CB16F05CEC09F050EC08F040
:10EB100016C060FB15C05FFB14C05EFB13C05DFB3D
:10EB20001A6A240E196E740E186E920E176E59CB57
:10EB300013F05ACB14F05BCB15F05CCB16F05CEC09
:10EB400009F050EC08F016C064FB15C063FB14C05C
:10EB500062FB13C061FB1A6A7C0E196E120E186EEE
:10EB6000920E176E9DC013F09EC014F09FC015F05A
:10EB7000A0C016F05CEC09F050EC08F016C054FB95
:10EB800015C053FB14C052FB13C051FBD15158ECBC
:10EB900009F054CB1AF053CB19F052CB18F051CBEB
:10EBA00017F0B6EC07F016C054FB15C053FB14C0A9
:10EBB00052FB13C051FB570E0101685D0001D8A440
:10EBC000E5EF75F0800E0B01521B00011A6A7C0EF6
:10EBD000196E120E186E920E176E99C013F09AC02D
:10EBE00014F09BC015F09CC016F05CEC09F050ECE2
:10EBF00008F016C04FFB15C04EFB14C04DFB13C0F0
:10EC00004CFBD05158EC09F04FCB1AF04ECB19F019
:10EC10004DCB18F04CCB17F0B6EC07F016C04FFBFD
:10EC200015C04EFB14C04DFB13C04CFB530E01012D
:10EC30005E5D0001D8A420EF76F0800E0B014D1B25
:10EC400000014CCBDEFF4DCBDEFF4ECBDEFF4FCBCA
:10EC5000DEFF51CBDEFF52CBDEFF53CBDEFF54CBCA
:10EC6000DEFF5DCBDEFF5ECBDEFF5FCBDEFF60CB8A
:10EC7000DEFF61CBDEFF62CBDEFF63CBDEFF64CB6A
:10EC8000DEFFD2EC17F01BEE66F04AEC02F069CB27
:10EC900022F068CB21F067CB20F066CB1FF02A6A08
:10ECA0000F0E296E420E286E400E276E8BEC01F07F
:10ECB00020C071FB1FC070FB226A216A71CB20F05B
:10ECC00070CB1FF02A6A0F0E296E420E286E400E7E
:10ECD000276E02EC02F022C034F021C033F020C0D5
:10ECE00032F01FC031F031500B01665D6A6F325057
:10ECF00067596B6F335068596C6F345069596D6F39
:10ED0000370E505D010ED8A4000E3B6E380E505DDC
:10ED1000010ED8A4000E3B100001D8B4E1EF76F04C
:10ED200003EE1EF0D89001012335E926000EEA22F9
:10ED3000EECF0BF0EFCF0CF00BC0DEFF0CC0DEFF10
:10ED40006ACBDEFF6BCBDEFF6CCBDEFF6DCBDEFF75
:10ED5000000129EC17F01BEE7BF05BEC02F07CCBA2
:10ED600020F07BCB1FF0246A3C0E236EEBEC01F00D
:10ED70000B017A6F206A7ACB1FF0010E75EC01F05F
:10ED8000766F206A7ACB1FF0000E75EC01F0776F7A
:10ED90007CCB20F07BCB1FF0246A3C0E236EEBEC87
:10EDA00001F027C07AFB206A7ACB1FF0010E75ECC8
:10EDB00001F0786F206A7ACB1FF0000E75EC01F03D
:10EDC000796F0001010E0101395D0001D8A47DEFCA
:10EDD00077F00B017F916DBF0CD0A00E6A5D860E9F
:10EDE0006B59010E6C59000E6D590001D8B075EFCA
:10EDF00077F06DCB22F06CCB21F06BCB20F06ACB9F
:10EE00001FF02A6A296A286A210E276E02EC02F096
:10EE100022C034F021C033F020C032F01FC031F0E6
:10EE200034C022F033C021F032C020F031C01FF0D6
:10EE30002A6A296A286A0A0E276E8BEC01F022C022
:10EE40006DFB21C06CFB20C06BFB1FC06AFBD8961A
:10EE50000B016DBFD8860001D8B66EEF77F00B01BD
:10EE60006D530AE16C5108E1E80E6A5D030E6B59BF
:10EE70000001D8A06EEF77F06DCB22F06CCB21F0C3
:10EE80006BCB20F06ACB1FF02A6A296A030E286E2A
:10EE9000E80E276E02EC02F022C034F021C033F0FD
:10EEA00020C032F01FC031F034C022F033C021F056
:10EEB00032C020F031C01FF02A6A296A170E286E6E
:10EEC000BC0E276E8BEC01F022C06DFB21C06CFBE9
:10EED00020C06BFB1FC06AFB0B017F8100016BCB65
:10EEE0006FFB6ACB6EFB7AEF77F0030E0B016F6F4F
:10EEF000E70E6E6F00019EEF77F0D8960B016DBFA5
:10EF0000D8860001D8B699EF77F00B016D530AE16E
:10EF10006C5108E1FF0E6A5DFF0E6B590001D8A02D
:10EF200099EF77F00B016D6B6C6B030E6B6FE70E57
:10EF30006A6F00016BCB6FFB6ACB6EFB010E0101A8
:10EF4000465D0001D8A4C0EF77F004EE1EF0D89023
:10EF500001012335E926000EEA22EECF0BF0EFCFB8
:10EF60000CF00BC0DEFF0CC0DEFF70CBDEFF71CB00
:10EF7000DEFF000175EC0EF01BEE70F05BEC02F0B2
:10EF8000330E0B01505D0001D8A4ECEF77F070CB8D
:10EF9000DEFF71CBDEFFDE6A010EDE6EDE6A4CEC58
:10EFA0007BF004EE1EF0D89001012335E926000E17
:10EFB000EA22EECF0BF0EFCF0CF00BC0DEFF0CC05F
:10EFC000DEFF010EDE6E010EDE6E0A0EDE6E000149
:10EFD0004CEC7BF009EF7AF0340E0B01505D000130
:10EFE000D8A417EF78F070CBDEFF71CBDEFFDE6ABE
:10EFF000010EDE6EDE6A4CEC7BF003EE1EF0D89064
:10F0000001012335E926000EEA22EECF0BF0EFCF07
:10F010000CF00BC0DEFF0CC0DEFF010EDE6EDE6A00
:10F02000140EDE6E00014CEC7BF009EF7AF0350E29
:10F030000B01505D0001D8A43FEF78F070CBDEFFEC
:10F0400071CBDEFF42EC0FF01BEE7DF05BEC02F0CB
:10F0500070CBDEFF71CBDEFFDE6A010EDE6EDE6A94
:10F060004CEC7BF07DCBDEFF7ECBDEFF010EDE6E57
:10F07000DE6A140EDE6E4CEC7BF009EF7AF0360E91
:10F080000B01505D0001D8A4EAEF78F070CBDEFFF1
:10F0900071CBDEFFDE6A010EDE6EDE6A4CEC7BF0C9
:10F0A0006FCB20F06ECB1FF0030E246EE80E0AEC3F
:10F0B00000F03B6E010E0B017FB1E86A3B140001CA
:10F0C000D8B4A0EF78F0D8960901FAAFD88600013D
:10F0D000D8B66EEF78F0ABECCEF08B836ECBDEFF64
:10F0E0006FCBDEFF010EDE6E010EDE6EDE6A4CECD3
:10F0F0007BF00901FA9FD89600018BA3D886D8B679
:10F100009EEF78F0010139530001D8A494EF78F014
:10F11000DE6ADE6A0C0EDE6E820EDE6E040EDE6EBF
:10F12000E4ECA8F09EEF78F0DE6ADE6A0A0EDE6E8E
:10F13000820EDE6E040EDE6EE4ECA8F0E8EF78F0EE
:10F14000D8960901FABFD8860001D8B6ABEF78F09F
:10F15000ABECCEF08B836FCB20F06ECB1FF0246A2C
:10F160000A0E236EEBEC01F00B016E6F20C06FFBFB
:10F170006ECBDEFF6FCBDEFF010EDE6EDE6ADE6A77
:10F1800000014CEC7BF00901FA8FD89600018BA3AB
:10F19000D886D8B6E8EF78F0010139530001D8A439
:10F1A000DEEF78F0DE6ADE6A370EDE6E820EDE6E2D
:10F1B000040EDE6EE4ECA8F0E8EF78F0DE6ADE6ABA
:10F1C000390EDE6E820EDE6E040EDE6EE4ECA8F00A
:10F1D00009EF7AF0370E0B01505D0001D8A408EF5B
:10F1E00079F070CBDEFF71CBDEFFDE6A010EDE6EE2
:10F1F000DE6A4CEC7BF0DE6A76CBDEFF77CBDEFF9F
:10F2000078CBDEFF79CBDEFFD2EC82F009EF7AF02B
:10F21000380E0B01505D0001D8A4B2EF79F06FCB2E
:10F2200020F06ECB1FF0030E246EE80E07EC00F00A
:10F230003B6E010E0B017FB1E86A3B140001D8B4AC
:10F240005EEF79F0D8960901FAAFD8860001D8B6FA
:10F250002DEF79F07AECCEF08B836ECBDEFF6FCBA7
:10F26000DEFFDE6A010EDE6EDE6A4CEC7BF0090129
:10F27000FA9FD89600018BA3D886D8B65CEF79F0B8
:10F28000010139530001D8A452EF79F0DE6ADE6A39
:10F290000C0EDE6E820EDE6E0D0EDE6EE4ECA8F05D
:10F2A0005CEF79F0DE6ADE6A0A0EDE6E820EDE6EDA
:10F2B0000D0EDE6EE4ECA8F0A5EF79F0D89609010A
:10F2C000FABFD8860001D8B669EF79F07AECCEF0B3
:10F2D0008B836FCB20F06ECB1FF0246A0A0E236E57
:10F2E000EBEC01F00B016E6F20C06FFB6ECBDEFF0D
:10F2F0006FCBDEFFDE6ADE6ADE6A00014CEC7BF07B
:10F300000901FA8FD89600018BA3D886D8B6A5EF4D
:10F3100079F0010139530001D8A49BEF79F0DE6A3E
:10F32000DE6A370EDE6E820EDE6E0D0EDE6EE4ECF1
:10F33000A8F0A5EF79F0DE6ADE6A390EDE6E820E85
:10F34000DE6E0D0EDE6EE4ECA8F0DE6A76CBDEFF3C
:10F3500077CBDEFF78CBDEFF79CBDEFFD2EC82F01D
:10F3600009EF7AF0390E0B01505D0001D8A407EFC8
:10F370007AF004EE1EF0D89001012335E926000E44
:10F38000EA22EECF0BF0EFCF0CF00BC0DEFF0CC08B
:10F39000DEFF010EDE6E010EDE6E0A0EDE6E000175
:10F3A0004CEC7BF0A7ECBFF0010146530001D8A460
:10F3B000FFEF79F004EE1EF0D89001012335E92625
:10F3C000000EEA22EECF0BF0EFCF0CF00BC0DEFF09
:10F3D0000CC0DEFF70CBDEFF71CBDEFF010EDE6EF8
:10F3E0000001B3EC0EF01BEE80F05BEC02F080CB82
:10F3F000DEFF81CBDEFF17ECC0F005EF7AF070CBBB
:10F40000DEFF71CBDEFF17ECC0F009EF7AF0B8EF4A
:10F4100032F012001BEE88F05BEC02F0D8968BA362
:10F42000D886D8B61BEF7AF0380E0B01856F380EF0
:10F43000866F380E876F000189CB20F088CB1FF0D4
:10F44000030E246EE80E236EEBEC01F00B01826FCD
:10F4500089CB32F088CB31F0366A82CB35F036C0BA
:10F460002EF035502D6EE80DF3CF35F0F4CF36F099
:10F470002E50E80DF35036262D50030DF35036264E
:10F480003550315E3650325A32C020F031C01FF054
:10F49000246A640E236EEBEC01F0836F89CB32F0AB
:10F4A00088CB31F0366A82CB35F036C02EF035503D
:10F4B0002D6EE80DF3CF35F0F4CF36F02E50E80D79
:10F4C000F35036262D50030DF35036263550315E5D
:10F4D0003650325A366A83CB35F03650640DF3CF4E
:10F4E00036F03550640DF3CF35F0F45036263550F4
:10F4F000315E3650325A32C020F031C01FF0246ADB
:10F500000A0E236EEBEC01F0846FDE6A570EDE6E9E
:10F51000000106ECBEF0170E0B018A6F8351865D69
:10F520000001D8B49AEF7AF083CBDEFF8ACBDEFFFE
:10F53000DDECC4F083CB86FB620E0B018A6F845135
:10F54000875D0001D8B4ABEF7AF084CBDEFF8ACBC5
:10F55000DEFFDDECC4F084CB87FB0B017F9382538D
:10F560000001D8B4C8EF7AF0010E0B018B6F8A6BE3
:10F570008251855D0001D8B4C6EF7AF082CBDEFF00
:10F580008ACBDEFF8BCBDEFFBBECCCF00B017F83A5
:10F590000001E86A0B017FB3010EDE6E000112006C
:10F5A0001BEE8CF05BEC02F01BEE8EF05BEC02F0DD
:10F5B0000B018E518C5D8F518D590001D8B0EBEF4E
:10F5C0007AF0DE6ADE6A050EDE6EDE6ADE6AE4EC82
:10F5D000A8F00DEF7BF00B018D518F5D0001D8A4D9
:10F5E00004EF7BF00B018C518E5D0001D8A404EF79
:10F5F0007BF0DE6ADE6A070EDE6EDE6A070EDE6E06
:10F60000E4ECA8F00DEF7BF0DE6ADE6A090EDE6E38
:10F61000DE6A0A0EDE6EE4ECA8F012001BEE90F03B
:10F620005BEC02F01BEE92F05BEC02F00B019251EE
:10F63000905D935191590001D8B029EF7BF0DE6ABB
:10F64000DE6AAF0EDE6EDE6ADE6AE4ECA8F04BEF37
:10F650007BF00B019151935D0001D8A442EF7BF048
:10F660000B019051925D0001D8A442EF7BF0DE6A5D
:10F67000DE6AB10EDE6EDE6A030EDE6EE4ECA8F02A
:10F680004BEF7BF0DE6ADE6AB30EDE6EDE6A040EDE
:10F69000DE6EE4ECA8F01200FF0EDBCFA4FBDD521F
:10F6A000FF0EDB50DD520B017F87E8A07F97FF0E36
:10F6B000DB50DD527F85E8A07F951BEE9EF05BEC72
:10F6C00002F0D89600018BA3D886D8B675EF7BF0F0
:10F6D000430E0B019B6F430E9C6F430E9D6F430EB9
:10F6E000986F430E996F430E9A6F00010B01946B54
:10F6F000956B966B976BD8967FA5D8860001D8B688
:10F70000B9EF7CF00A0E0B01A26F0D0E00018C5DAB
:10F71000D8A48EEF7BF0040E0B01A26F0001D896E7
:10F720000B017FA7D8860001D8B6EDEF7BF09FCB09
:10F7300020F09ECB1FF0020E75EC01F00B01946FD0
:10F740009FCB20F09ECB1FF0010E75EC01F0956F62
:10F750009FCB20F09ECB1FF0000E75EC01F0966F52
:10F76000976BA4CBA3FB9451985D0001D8B4C1EF73
:10F770007BF0A2CBDEFFA3CBDEFF94CBDEFFC7EC9A
:10F78000C4F094CB98FB290E0B01A425A36F9551CF
:10F79000995D0001D8B4D5EF7BF0A2CBDEFFA3CBFF
:10F7A000DEFF95CBDEFFC7ECC4F095CB99FB520E84
:10F7B0000B01A425A36F96519A5D0001D8B4E9EF1F
:10F7C0007BF0A2CBDEFFA3CBDEFF96CBDEFFC7EC48
:10F7D000C4F096CB9AFBB7EF7CF09FCB20F09ECB8A
:10F7E0001FF0030E75EC01F00B01946F9FCB20F01E
:10F7F0009ECB1FF0020E75EC01F0956F9FCB20F0B1
:10F800009ECB1FF0010E75EC01F0966F9FCB20F0A0
:10F810009ECB1FF0000E75EC01F0976F9453000122
:10F82000D8A466EF7CF0A4CBA3FB0B019551985DA7
:10F830000001D8B424EF7CF0A2CBDEFFA3CBDEFF27
:10F8400095CBDEFFC7ECC4F095CB98FB2D0E0B01DA
:10F85000A425A36F9651995D0001D8B438EF7CF0D0
:10F86000A2CBDEFFA3CBDEFF96CBDEFFC7ECC4F05E
:10F8700096CB99FB5A0E0B01A425A36F97519A5D65
:10F880000001D8B44CEF7CF0A2CBDEFFA3CBDEFFAF
:10F8900097CBDEFFC7ECC4F097CB9AFB5B0E0B0156
:10F8A000A425A56F050EDE6EA5CBDEFF0001B7EC2B
:10F8B000BEF02E0E0B01A425A56F050EDE6EA5CBA6
:10F8C000DEFF000193ECBEF0B7EF7CF0A4CBA3FB0E
:10F8D0000B019451985D0001D8B477EF7CF0A2CB76
:10F8E000DEFFA3CBDEFF94CBDEFFC7ECC4F094CBEE
:10F8F00098FB2D0E0B01A425A36F9551995D000176
:10F90000D8B48BEF7CF0A2CBDEFFA3CBDEFF95CB90
:10F91000DEFFC7ECC4F095CB99FB5A0E0B01A42572
:10F92000A36F96519A5D0001D8B49FEF7CF0A2CBF3
:10F93000DEFFA3CBDEFF96CBDEFFC7ECC4F096CB99
:10F940009AFB2E0E0B01A425A56F050EDE6EA5CB2E
:10F95000DEFF0001B7ECBEF05B0E0B01A425A56F26
:10F96000050EDE6EA5CBDEFF000193ECBEF000EFCE
:10F970007EF0206A8CC01FF0010E75EC01F00B6E5A
:10F98000080E0B5CD8A4CAEF7CF00B01A26B00013F
:10F99000D9EF7CF00D0E8C5DD8A4D5EF7CF0040E71
:10F9A0000B01A26F0001D8EF7CF0010E0B01A26FDA
:10F9B0000001D8960B017FA7D8860001D8B636EF94
:10F9C0007DF09FCB20F09ECB1FF0020E75EC01F076
:10F9D0000B01946F9FCB20F09ECB1FF0010E75ECB6
:10F9E00001F0956F9FCB20F09ECB1FF0000E75ECC1
:10F9F00001F0966FA4CBA3FB94519B5D0001D8B49A
:10FA00000AEF7DF0A2CBDEFFA3CBDEFF94CBDEFFBF
:10FA1000C7ECC4F094CB9BFB290E0B01A425A36F6C
:10FA200095519C5D0001D8B41EEF7DF0A2CBDEFFA6
:10FA3000A3CBDEFF95CBDEFFC7ECC4F095CB9CFBE0
:10FA4000520E0B01A425A36F96519D5D0001D8B401
:10FA500032EF7DF0A2CBDEFFA3CBDEFF96CBDEFF45
:10FA6000C7ECC4F096CB9DFB00EF7EF09FCB20F05F
:10FA70009ECB1FF0030E75EC01F00B01946F9FCB32
:10FA800020F09ECB1FF0020E75EC01F0956F9FCB1E
:10FA900020F09ECB1FF0010E75EC01F0966F9FCB0E
:10FAA00020F09ECB1FF0000E75EC01F0976F945381
:10FAB0000001D8A4AFEF7DF0A4CBA3FB0B019551BF
:10FAC0009B5D0001D8B46DEF7DF0A2CBDEFFA3CB30
:10FAD000DEFF95CBDEFFC7ECC4F095CB9BFB2D0E74
:10FAE0000B01A425A36F96519C5D0001D8B481EF52
:10FAF0007DF0A2CBDEFFA3CBDEFF96CBDEFFC7EC13
:10FB0000C4F096CB9CFB5A0E0B01A425A36F975112
:10FB10009D5D0001D8B495EF7DF0A2CBDEFFA3CBB5
:10FB2000DEFF97CBDEFFC7ECC4F097CB9DFB530EF7
:10FB30000B01A425A56F010EDE6EA5CBDEFF000133
:10FB4000FEECBEF0260E0B01A425A56F010EDE6EA5
:10FB5000A5CBDEFF0001DAECBEF000EF7EF0A4CB17
:10FB6000A3FB0B0194519B5D0001D8B4C0EF7DF065
:10FB7000A2CBDEFFA3CBDEFF94CBDEFFC7ECC4F04D
:10FB800094CB9BFB2D0E0B01A425A36F95519C5D7F
:10FB90000001D8B4D4EF7DF0A2CBDEFFA3CBDEFF13
:10FBA00095CBDEFFC7ECC4F095CB9CFB5A0E0B0146
:10FBB000A425A36F96519D5D0001D8B4E8EF7DF0B8
:10FBC000A2CBDEFFA3CBDEFF96CBDEFFC7ECC4F0FB
:10FBD00096CB9DFB260E0B01A425A56F010EDE6EB4
:10FBE000A5CBDEFF0001FEECBEF0530E0B01A425F9
:10FBF000A56F010EDE6EA5CBDEFF0001DAECBEF0D4
:10FC00001200D8968BA3D886D8B648EF7EF0DE6A6D
:10FC1000DE6A1F0EDE6EDE6A010EDE6EE4ECA8F018
:10FC2000DE6ADE6A210EDE6EDE6A050EDE6EE4EC52
:10FC3000A8F0010E0101395D0001D8A42BEF7EF080
:10FC4000DE6ADE6A390EDE6EDE6A090EDE6EE4EC16
:10FC5000A8F034EF7EF0DE6ADE6A370EDE6EDE6A12
:10FC6000090EDE6EE4ECA8F0DE6ADE6A150EDE6ECA
:10FC7000070EDE6E0C0EDE6EE4ECA8F0DE6ADE6AC5
:10FC8000130EDE6E5A0EDE6E0C0EDE6EE4ECA8F085
:10FC90000B01A76B29C120F028C11FF0000E75ECE5
:10FCA00001F0A76F920EA66FA7CBDEFFA6CBDEFFFB
:10FCB000010EDE6E000129ECCAF00B01A76B29C111
:10FCC00020F028C11FF0010E75EC01F0A76F840E23
:10FCD000A66FA7CBDEFFA6CBDEFF010EDE6E000116
:10FCE00029ECCAF0010EDE6EBEECD1F0800E0B01E5
:10FCF000A76FA7CBDEFF0001DAECD1F0030EDE6EBA
:10FD00004CECD2F0030EDE6E4CECD2F00B01A76B84
:10FD100029C120F028C11FF0020E75EC01F0A76F79
:10FD2000720EA66FA7CBDEFFA6CBDEFF010EDE6E46
:10FD3000000129ECCAF00B01A76B29C120F028C1F2
:10FD40001FF0030E75EC01F0A76F640EA66FA7CB32
:10FD5000DEFFA6CBDEFF010EDE6E000129ECCAF04D
:10FD60000B01A76B2BC120F02AC11FF0000E75EC10
:10FD700001F0A76F3E0EA66FA7CBDEFFA6CBDEFF7E
:10FD8000010EDE6E000129ECCAF00B01A76B2BC13E
:10FD900020F02AC11FF0010E75EC01F0A76F300EA4
:10FDA000A66FA7CBDEFFA6CBDEFF010EDE6E000145
:10FDB00029ECCAF0010EDE6EBEECD1F02C0E0B0168
:10FDC000A76FA7CBDEFF0001DAECD1F0030EDE6EE9
:10FDD0004CECD2F0030EDE6E4CECD2F00B01A76BB4
:10FDE0002BC120F02AC11FF0020E75EC01F0A76FA5
:10FDF0001E0EA66FA7CBDEFFA6CBDEFF010EDE6ECA
:10FE0000000129ECCAF00B01A76B2BC120F02AC11D
:10FE10001FF0030E75EC01F0A76F100EA66FA7CBB5
:10FE2000DEFFA6CBDEFF010EDE6E000129ECCAF07C
:10FE3000010139530001D8A428EF7FF01FC8AFFBA0
:10FE40001EC8AEFB1DC8ADFB1CC8ACFB58EF7FF055
:10FE50001FC822F01EC821F01DC820F01CC81FF0CA
:10FE60002A6A296A030E286EE80E276E02EC02F059
:10FE700022C034F021C033F020C032F01FC031F076
:10FE800034C022F033C021F032C020F031C01FF066
:10FE90002A6A296A070E286E3C0E276E8BEC01F049
:10FEA00022C0AFFB21C0AEFB20C0ADFB1FC0ACFB2E
:10FEB0000B01A76BAFCB22F0AECB21F0ADCB20F086
:10FEC000ACCB1FF0010E7FEC01F0A76F920EA66F76
:10FED000A7CBDEFFA6CBDEFF050EDE6E000129EC10
:10FEE000CAF00B01A76BAFCB22F0AECB21F0ADCBAC
:10FEF00020F0ACCB1FF0020E7FEC01F0A76F840E58
:10FF0000A66FA7CBDEFFA6CBDEFF050EDE6E0001DF
:10FF100029ECCAF0050EDE6EBEECD1F0800E0B01AE
:10FF2000A76FA7CBDEFF0001DAECD1F0030EDE6E87
:10FF30004CECD2F0030EDE6E4CECD2F00B01A76B52
:10FF4000AFCB22F0AECB21F0ADCB20F0ACCB1FF08D
:10FF5000030E7FEC01F0A76F720EA66FA7CBDEFF3A
:10FF6000A6CBDEFF050EDE6E000129ECCAF00B0108
:10FF7000A76BAFCB22F0AECB21F0ADCB20F0ACCB5A
:10FF80001FF0040E7FEC01F0A76F640EA66FA7CBE5
:10FF9000DEFFA6CBDEFF050EDE6E000129ECCAF007
:10FFA0000B01A76BAFCB22F0AECB21F0ADCB20F095
:10FFB000ACCB1FF0050E7FEC01F0A76F560EA66FBD
:10FFC000A7CBDEFFA6CBDEFF050EDE6E000129EC1F
:10FFD000CAF00B01A76BAFCB22F0AECB21F0ADCBBB
:10FFE00020F0ACCB1FF0060E7FEC01F0A76F480E9F
:10FFF000A66FA7CBDEFFA6CBDEFF050EDE6E0001EF
:020000040001F9
:1000000029ECCAF09CC022F09BC021F09AC020F0DD
:1000100099C01FF02A6A296A286A0A0E276E02EC24
:1000200002F022C034F021C033F020C032F01FC0F3
:1000300031F034C022F033C021F032C020F031C0A2
:100040001FF02A6A296A286A060E276E8BEC01F0D7
:1000500022C0ABFB21C0AAFB20C0A9FB1FC0A8FB8C
:10006000226A216A206AD0C01FF02A6A0F0E296E08
:10007000420E286E400E276E02EC02F022C034F0D1
:1000800021C033F020C032F01FC031F031500B01DD
:10009000A8273250A9233350AA233450AB23530E40
:1000A00001015E5D0001D8A47CEF80F0010EDE6EE0
:1000B000CCECD1F0380E0B01A76FA7CBDEFF00010F
:1000C00006ECD2F00C0EDE6E5AECD2F00C0EDE6EA8
:1000D0005AECD2F00C0EDE6E5AECD2F00C0EDE6E44
:1000E0005AECD2F00C0EDE6E5AECD2F00C0EDE6E34
:1000F0005AECD2F09AEF80F0010EDE6ECCECD1F02B
:10010000380E0B01A76FA7CBDEFF000106ECD2F083
:10011000DE6A5AECD2F0DE6A5AECD2F0DE6A5AECB1
:10012000D2F0DE6A5AECD2F0DE6A5AECD2F0DE6A25
:100130005AECD2F00B01A76BABCB22F0AACB21F08B
:10014000A9CB20F0A8CB1FF0010E7FEC01F0A76F28
:10015000920EA66FA7CBDEFFA6CBDEFF0D0EDE6EE6
:10016000000129ECCAF00B01A76BABCB22F0AACBA4
:1001700021F0A9CB20F0A8CB1FF0020E7FEC01F0FC
:10018000A76F840EA66FA7CBDEFFA6CBDEFF0D0EFA
:10019000DE6E000129ECCAF00B01A76BABCB22F09D
:1001A000AACB21F0A9CB20F0A8CB1FF0030E7FEC47
:1001B00001F0A76F760EA66FA7CBDEFFA6CBDEFF02
:1001C0000D0EDE6E000129ECCAF00B01A76BABCB64
:1001D00022F0AACB21F0A9CB20F0A8CB1FF0040E6F
:1001E0007FEC01F0A76F680EA66FA7CBDEFFA6CB52
:1001F000DEFF0D0EDE6E000129ECCAF00B01A76BCD
:10020000ABCB22F0AACB21F0A9CB20F0A8CB1FF0DA
:10021000050E7FEC01F0A76F5A0EA66FA7CBDEFF8D
:10022000A6CBDEFF0D0EDE6E000129ECCAF0020E39
:10023000DE6ECCECD1F05E0E0B01A76FA7CBDEFF1C
:10024000000106ECD2F0C00EDE6E5AECD2F0C00E09
:10025000DE6E5AECD2F00B01A76BABCB22F0AACB2F
:1002600021F0A9CB20F0A8CB1FF0060E7FEC01F007
:10027000A76F480EA66FA7CBDEFFA6CBDEFF0D0E45
:10028000DE6E000129ECCAF00B01A76BABCB22F0AC
:10029000AACB21F0A9CB20F0A8CB1FF0070E7FEC52
:1002A00001F0A76F3A0EA66FA7CBDEFFA6CBDEFF4D
:1002B0000D0EDE6E000129ECCAF0A0C022F09FC036
:1002C00021F09EC020F09DC01FF02A6A296A286A8A
:1002D0000A0E276E02EC02F022C034F021C033F087
:1002E00020C032F01FC031F034C022F033C021F002
:1002F00032C020F031C01FF02A6A296A286A060E2F
:10030000276E8BEC01F022C0ABFB21C0AAFB20C002
:10031000A9FB1FC0A8FB226A216A206AD1C01FF076
:100320002A6A0F0E296E420E286E400E276E02ECCE
:1003300002F022C034F021C033F020C032F01FC0E0
:1003400031F031500B01A8273250A9233350AA2392
:100350003450AB23570E0101685D0001D8A4D7EFDC
:1003600081F0050EDE6ECCECD1F02A0E0B01A76FEA
:10037000A7CBDEFF000106ECD2F00C0EDE6E5AECCD
:10038000D2F00C0EDE6E5AECD2F00C0EDE6E5AEC91
:10039000D2F00C0EDE6E5AECD2F00C0EDE6E5AEC81
:1003A000D2F00C0EDE6E5AECD2F0F5EF81F0050EB5
:1003B000DE6ECCECD1F02A0E0B01A76FA7CBDEFFCF
:1003C000000106ECD2F0DE6A5AECD2F0DE6A5AEC9A
:1003D000D2F0DE6A5AECD2F0DE6A5AECD2F0DE6A73
:1003E0005AECD2F0DE6A5AECD2F00B01A76BABCB21
:1003F00022F0AACB21F0A9CB20F0A8CB1FF0010E50
:100400007FEC01F0A76F920EA66FA7CBDEFFA6CB05
:10041000DEFF090EDE6E000129ECCAF00B01A76BAE
:10042000ABCB22F0AACB21F0A9CB20F0A8CB1FF0B8
:10043000020E7FEC01F0A76F840EA66FA7CBDEFF44
:10044000A6CBDEFF090EDE6E000129ECCAF00B011F
:10045000A76BABCB22F0AACB21F0A9CB20F0A8CB85
:100460001FF0030E7FEC01F0A76F760EA66FA7CBEF
:10047000DEFFA6CBDEFF090EDE6E000129ECCAF01E
:100480000B01A76BABCB22F0AACB21F0A9CB20F0BC
:10049000A8CB1FF0040E7FEC01F0A76F680EA66FCB
:1004A000A7CBDEFFA6CBDEFF090EDE6E000129EC36
:1004B000CAF00B01A76BABCB22F0AACB21F0A9CBE2
:1004C00020F0A8CB1FF0050E7FEC01F0A76F5A0EAD
:1004D000A66FA7CBDEFFA6CBDEFF090EDE6E000106
:1004E00029ECCAF0060EDE6ECCECD1F05E0E0B01EC
:1004F000A76FA7CBDEFF000106ECD2F0C00EDE6EC8
:100500005AECD2F0C00EDE6E5AECD2F00B01A76BA3
:10051000ABCB22F0AACB21F0A9CB20F0A8CB1FF0C7
:10052000060E7FEC01F0A76F480EA66FA7CBDEFF8B
:10053000A6CBDEFF090EDE6E000129ECCAF00B012E
:10054000A76BABCB22F0AACB21F0A9CB20F0A8CB94
:100550001FF0070E7FEC01F0A76F3A0EA66FA7CB36
:10056000DEFFA6CBDEFF090EDE6E000129ECCAF02D
:100570000B01A76BABCB22F0AACB21F0A9CB20F0CB
:10058000A8CB1FF0080E7FEC01F0A76F2C0EA66F12
:10059000A7CBDEFFA6CBDEFF090EDE6E000129EC45
:1005A000CAF01200FF0EDBCFB3FBDD52FF0EDBCF34
:1005B000B2FBDD52FF0EDBCFB1FBDD52FF0EDBCF16
:1005C000B0FBDD52FF0EDB50DD520B017F89E8A04E
:1005D0007F99D89600018BA3D886D8B601EF83F017
:1005E000630E0B01B76F630EB66F630EB56F630ECC
:1005F000B46F630EBB6F630EBA6F630EB96F630E99
:10060000B86F0001D8960B017FB9D8860001D8B623
:1006100042EF83F0020EDE6ECCECD1F0560EDE6EB1
:1006200006ECD2F00B01BE6B0001040E0B01BE5DA7
:100630000001D8B025EF83F03F0EDE6E5AECD2F009
:100640000B01BE2B0001D8A4EFD7050EDE6ECCEC5B
:10065000D1F0560EDE6E06ECD2F00B01BE6B00013F
:10066000040E0B01BE5D0001D8B040EF83F0FC0E1C
:10067000DE6E5AECD2F00B01BE2B0001D8A4EFD7EE
:1006800078EF83F0020EDE6EBEECD1F04E0EDE6E21
:10069000DAECD1F00B01BE6B0001040E0B01BE5D64
:1006A0000001D8B05DEF83F03F0EDE6E4CECD2F06F
:1006B0000B01BE2B0001D8A4EFD7050EDE6EBEECF9
:1006C000D1F04E0EDE6EDAECD1F00B01BE6B000104
:1006D000040E0B01BE5D0001D8B078EF83F0FC0E74
:1006E000DE6E4CECD2F00B01BE2B0001D8A4EFD78C
:1006F000D8960B017FB9D8860001D8B6CFEF83F02A
:10070000090E0B01BD6FBC6BB051B45D0001D8B4D4
:1007100092EF83F0BDCBDEFFBCCBDEFFB0CBDEFFC4
:10072000C7ECC4F0B0CBB4FB280E0B01BC6FB151C9
:10073000B55D0001D8B4A5EF83F0BDCBDEFFBCCB27
:10074000DEFFB1CBDEFFC7ECC4F0B1CBB5FB540E7E
:100750000B01BC6FB251B65D0001D8B4B8EF83F0A5
:10076000BDCBDEFFBCCBDEFFB2CBDEFFC7ECC4F0FF
:10077000B2CBB6FB7C0E0B01BC6FB351B75D000171
:10078000D8B4CBEF83F0BDCBDEFFBCCBDEFFB3CB69
:10079000DEFFC7ECC4F0B3CBB7FB1CEF84F0010E57
:1007A0000B01BD6FBC6BB051B85D0001D8B4E1EF77
:1007B00083F0BDCBDEFFBCCBDEFFB0CBDEFFC7ECF2
:1007C000C4F0B0CBB8FB280E0B01BC6FB151B95DC2
:1007D0000001D8B4F4EF83F0BDCBDEFFBCCBDEFF6D
:1007E000B1CBDEFFC7ECC4F0B1CBB9FB540E0B01AB
:1007F000BC6FB251BA5D0001D8B407EF84F0BDCB35
:10080000DEFFBCCBDEFFB2CBDEFFC7ECC4F0B2CB69
:10081000BAFB7C0E0B01BC6FB351BB5D0001D8B4B9
:100820001AEF84F0BDCBDEFFBCCBDEFFB3CBDEFF27
:10083000C7ECC4F0B3CBBBFB1200FF0EDB50DD52A4
:100840000B017F8BE8A07F9B030E0001836F840E5A
:10085000826F0A0E986F0B0E08012A6FDC0E296F4B
:10086000F2942AC8D7FF29C8D6FF0B01D06B00012C
:100870000B01D16B0001F2A44AEF84F00B0E0801CA
:100880002A6FDC0E296FF2942AC8D7FF29C8D6FF39
:100890000B01D06B0001D6CF29F8D7CF2AF8D89614
:1008A0008BB3D886D8B658EF84F0DE6AFCEC8EF0B5
:1008B000010E985DD8A481EF84F0D8960B017FBB20
:1008C000D8860001D8B66AEF84F08B83CCEF85F030
:1008D0007FEF84F03E0E8C5DD8A474EF84F08B83A0
:1008E0005FEF8BF07FEF84F0400E8C5DD8A47DEF3E
:1008F00084F052EF88F07FEF84F022EF35F0B8EF0C
:1009000084F0020E985DD8A4A0EF84F03C0E8227FC
:10091000000E8323030E835DD8A09AEF84F0D8A441
:1009200097EF84F0850E825DD8A09AEF84F0836BF8
:100930003C0E826F010E0B01D16F0001B8EF84F005
:10094000030E985DD8A4B8EF84F03C0E825F000ED1
:10095000835B83518211D8A4B2EF84F0030E836FBE
:10096000840E826F010E0B01D16F0001B8EF84F08D
:1009700083C020F082C01FF0246A3C0E236EEBEC93
:1009800001F00B01C36F206AC3CB1FF0010E75ECA1
:1009900001F0BF6F206AC3CB1FF0000E75EC01F0B1
:1009A000C06FC16BC26B010EDE6EBFCBDEFFC0CB72
:1009B000DEFFC1CBDEFFC2CBDEFF0001D2EC82F056
:1009C000010E0B01D15D0001D8A4ECEF84F0C80E3C
:1009D00054EC01F0BEEF85F03E0E8C5DD8A4BEEF66
:1009E00085F02AC820F029C81FF0880E246EB80EA2
:1009F00004EC00F03B6E010E0B01D053D8A4000EA6
:100A00003B140001D8B4BEEF85F0AAEC0AF0DE6A10
:100A100013EC48F0BBEC70F01BEEC4F04AEC02F0B3
:100A2000D8960B01C7BFD8860001D8B62DEF85F048
:100A30003D0E0B01C45D860EC559010EC659000E50
:100A4000C7590001D8A02DEF85F00B01C76B010E2F
:100A5000C66F860EC56F3C0EC46F0001C7CB22F077
:100A6000C6CB21F0C5CB20F0C4CB1FF02A6A296A7F
:100A7000286A640E276E8BEC01F022C0C7FB21C0F0
:100A8000C6FB20C0C5FB1FC0C4FB0B01CA6BCB6BF0
:100A9000CC6BC7CB22F0C6CB21F0C5CB20F0C4CBAA
:100AA0001FF0020E7FEC01F0CA6FC7CB22F0C6CB5D
:100AB00021F0C5CB20F0C4CB1FF0010E7FEC01F07C
:100AC000CB6FC7CB22F0C6CB21F0C5CB20F0C4CB77
:100AD0001FF0000E7FEC01F0CC6F326ACACB31F010
:100AE0003250640DF3CF32F03150640DF3CF31F05A
:100AF000F4503226366ACBCB35F036500A0DF3CFA0
:100B000036F035500A0DF3CF35F0F4503626355017
:100B1000312636503222CC513124C86F000E32209B
:100B2000C96FC8CBDEFFC9CBDEFF010EDE6E010E42
:100B3000DE6EDE6A00014CEC7BF0010E0B01D06F23
:100B4000D896010138B1D8860001D8B6B4EF85F047
:100B5000DE6ADE6AC50EDE6E820EDE6E010EDE6EAF
:100B6000E4ECA8F0BEEF85F0DE6ADE6AC30EDE6E4E
:100B7000820EDE6E010EDE6EE4ECA8F0D8968BA33A
:100B8000D886D8B6C9EF85F0010E246E900E55ECCC
:100B900001F08B936CD6120008012E6B030E0B0133
:100BA000DF6F0001F2A434EF86F08207000E835B52
:100BB0000D0E08012A6F050E296F2AC8D7FF29C814
:100BC000D6FFF2940001846B83C020F082C01FF036
:100BD000246A3C0E236EEBEC01F00B01D26F206A0D
:100BE000D2CB1FF0010E75EC01F0D36F206AD2CB8F
:100BF0001FF0000E75EC01F0D46F83C020F082C0AE
:100C00001FF0246A3C0E236EEBEC01F027C0D2FBF0
:100C1000206AD2CB1FF0010E75EC01F0D56F206A6F
:100C2000D2CB1FF0000E75EC01F0D66F010EDE6E18
:100C3000D3CBDEFFD4CBDEFFD5CBDEFFD6CBDEFFC2
:100C40000001D2EC82F083518211D8A42DEF86F0FE
:100C500008012E6B0001CFEF87F083C0DEFB82C05E
:100C6000DDFB9FD7FBEF86F0D6CF29F8D7CF2AF848
:100C7000EA0E08012A5D0001D8A04AEF86F0D8A448
:100C800049EF86F0610E0801295D0001D8A04AEF06
:100C900086F087D7880E08012A5DB80ED8B4295D82
:100CA0000001D8B0FBEF86F0010EDE6EFCEC8EF09A
:100CB000010E985DD8A47CEF86F008012E53000148
:100CC000D8A47AEF86F0D8968BB3D886D8B67AEFC8
:100CD00086F008012E6B010E2D6F0001DDECCEF0C9
:100CE0000801276B010E246EF40E55EC01F0000193
:100CF000B8EF32F0FBEF86F0020E985DD8A4A9EFB2
:100D000086F008012E530001D8A4A6EF86F083C018
:100D100020F082C01FF0246A0A0E236EEBEC01F073
:100D2000826F20C083F083510A0DF3CF32F08251DD
:100D30000A0DF3CF31F0F4503226010E3124826FC8
:100D4000000E3220836F020E08012D6F0001FBEFB1
:100D500086F0030E985DD8A4C8EF86F008012E53E4
:100D60000001D8A4C5EF86F0020E08012D5D000138
:100D7000D8A4C2EF86F0030E836F840E826FDE6A02
:100D80001DEC84F0030E08012D6F0001FBEF86F0CF
:100D9000040E985DD8A4D5EF86F00B01D769040E38
:100DA00008012D6F0001FBEF86F0050E985DD8A4B9
:100DB000F8EF86F00B01D7290001D8A4F2EF86F0F6
:100DC00008012E290001D8A4EDEF86F008012E6B52
:100DD0000B01D76B0001F1EF86F008012E690B01C2
:100DE000D76B0001050E08012D6F0001FAEF86F0A8
:100DF00008012D6B0001D6CF29F8D7CF2AF8EA0ECB
:100E000008012A5D0001D8A011EF87F0D8A410EFE7
:100E100087F0610E0801295D0001D8A011EF87F06D
:100E2000C0D60B01D7290001D8A420EF87F00B0111
:100E3000D82B00011FEF87F00B01D76BD86B000197
:100E400008012D530001D8B42CEF87F083C0DAFBE2
:100E500082C0D9FB47EF87F082510B01D95DDB6F70
:100E6000000183510B01DA59DC6FDC530001D8A477
:100E700041EF87F0100E0B01DB5D0001D8A046EFBB
:100E800087F00B01D76B08012E6B2E6900010B0157
:100E9000D7290001D8A46AEF87F00B01DF530001C6
:100EA000D8B468EF87F0DE6A010EDE6E750EDE6E76
:100EB000820EDE6E050EDE6EE4ECA8F0DE6ADE6AFF
:100EC000730EDE6E840EDE6E050EDE6EE4ECA8F0B0
:100ED0000B01DF6B000108012E29010ED8A4000EC2
:100EE0003B6E010E0B01D753D8A4000E3B1400013A
:100EF000D8B49AEF87F0010E0B01DF5D0001D8B482
:100F000097EF87F0DE6A010EDE6E730EDE6E840EE2
:100F1000DE6E050EDE6EE4ECA8F0DE6ADE6A750EAB
:100F2000DE6E820EDE6E050EDE6EE4ECA8F0010EC3
:100F30000B01DF6F0001010E08012E53D8A4000E33
:100F40003B6E010E0B01D753D8A4000E3B140001D9
:100F5000D8B4CBEF87F0020E0B01DF5D0001D8A4FF
:100F6000C8EF87F0DE6A010EDE6E730EDE6E840E51
:100F7000DE6E050EDE6EE4ECA8F0DE6A010EDE6EBB
:100F8000750EDE6E820EDE6E050EDE6EE4ECA8F0EF
:100F9000020E0B01DF6F00018B9303D612000B01D1
:100FA000E06B00011A0E0B01E05D0001D8B0E8EF24
:100FB00087F084ECD2F0C80E54EC01F093ECD2F040
:100FC000C80E54EC01F00B01E02B0001D8A4E9D7C6
:100FD000010EBA5DD8A4F8EF87F0030EB95DD8A46E
:100FE000F8EF87F0020EB96FB6EC62F0020EBA6F3E
:100FF0008DC08CF08B8322EF35F012000B0E0801B0
:101000002A6FDC0E296F2AC8D7FF29C8D6FFF294B1
:1010100000018207000E835B83C020F082C01FF0B6
:10102000246A3C0E236EEBEC01F00B01E16F206AA9
:10103000E1CB1FF0010E75EC01F0E26F206AE1CB0D
:101040001FF0000E75EC01F0E36F83C020F082C04A
:101050001FF0246A3C0E236EEBEC01F027C0E1FB8D
:10106000206AE1CB1FF0010E75EC01F0E46F206AFD
:10107000E1CB1FF0000E75EC01F0E56F010EDE6EA6
:10108000E2CBDEFFE3CBDEFFE4CBDEFFE5CBDEFF32
:101090000001D2EC82F083518211D8A451EF88F084
:1010A0007ED71200030E0B01F96FE80EF86F010EE8
:1010B000FB6F0B0E08012A6FDC0E296F2AC8D7FFC1
:1010C00029C8D6FFF2940001F2A478EF88F08207D5
:1010D000000E835B0B0E08012A6FDC0E296FF29461
:1010E0002AC8D7FF29C8D6FF0001846B79EF88F0A2
:1010F000EAD7F2A48BEF88F08207000E835B0B0E19
:1011000008012A6FDC0E296FF2942AC8D7FF29C87C
:10111000D6FF0001846BD6CF29F8D7CF2AF8EA0E84
:1011200008012A5D0001D8A0A1EF88F0D8A4A0EFA3
:1011300088F0610E0801295D0001D8A0A1EF88F0B8
:10114000D8D7F2A4A5EF88F0D4D783510B01F95D6D
:101150000001D8A4B3EF88F082510B01F85D0001C3
:10116000D8B444EF89F083C020F082C01FF0246A15
:101170003C0E236EEBEC01F00B01F36F206AF3CB16
:101180001FF0010E75EC01F0F46F206AF3CB1FF035
:10119000000E75EC01F0F56F83C020F082C01FF0E7
:1011A000246A3C0E236EEBEC01F027C0F3FB206AAF
:1011B000F3CB1FF0010E75EC01F0F66F206AF3CB54
:1011C0001FF0000E75EC01F0F76F010EDE6EF4CB30
:1011D000DEFFF5CBDEFFF6CBDEFFF7CBDEFF000157
:1011E000D2EC82F083518211D8A4F8EF88F0D7D6E0
:1011F00083C0F9FB82C0F8FBFDCB20F0FCCB1FF0D5
:10120000246A3C0E236EEBEC01F00B01F36F206AB5
:10121000F3CB1FF0010E75EC01F0F46F206AF3CBF5
:101220001FF0000E75EC01F0F56FFDCB20F0FCCB4C
:101230001FF0246A3C0E236EEBEC01F027C0F3FB99
:10124000206AF3CB1FF0010E75EC01F0F66F206AF7
:10125000F3CB1FF0000E75EC01F0F76F0001F2A464
:1012600033EF89F0CBDEDE6AF4CBDEFFF5CBDEFFB9
:10127000F6CBDEFFF7CBDEFFD2EC82F0F2A442EF3A
:1012800089F037D779EF89F0EA0E08012A5D00016D
:10129000D8A056EF89F0D8A455EF89F0610E080167
:1012A000295D0001D8A056EF89F023D7F2A45AEFA8
:1012B00089F01FD79C0E08012A5D400ED8B4295D25
:1012C0000001D8B079EF89F0010EDE6EFCEC8EF0F3
:1012D000010E985DD8A479EF89F0DDECCEF008011D
:1012E000276B010E246EF40E55EC01F00001B8EFEF
:1012F00032F08453D8A47FEF89F00B01FB6B00011F
:101300000B01FB530001D8A408EF8AF02AC820F093
:1013100029C81FF0610E246EA80E04EC00F03B6E8D
:10132000010E8453D8A4000E3B10D8B408EF8AF005
:10133000010E845DD8A4A0EF89F0010E0B01FB6FB4
:101340000001AAEC0AF0DE6A13EC48F0BBEC70F086
:101350001BEEE7F04AEC02F0D8960B01EABFD88604
:101360000001D8B6D0EF89F03D0E0B01E75D860E87
:10137000E859010EE959000EEA590001D8A0D0EF52
:1013800089F00B01EA6B010EE96F860EE86F3C0EE7
:10139000E76F170EFD6F340EFC6F000106EF8AF049
:1013A000EACB22F0E9CB21F0E8CB20F0E7CB1FF02D
:1013B0002A6A296A286A640E276E8BEC01F022C023
:1013C000EAFB21C0E9FB20C0E8FB1FC0E7FB03EEFE
:1013D0001EF0D89001012335E926000EEA22EECF57
:1013E0000BF0EFCF0CF00BC0DEFF0CC0DEFFE7CB45
:1013F000DEFFE8CBDEFFE9CBDEFFEACBDEFF00015C
:1014000029EC17F01BEEFCF05BEC02F0010E846F90
:101410008B936FD61200D8968BB3D886D8B624EFAC
:101420008AF0DE6AFCEC8EF0010E985DD8A424EF01
:101430008AF0D8968BB3D886D8B624EF8AF0080104
:10144000276B0001B8EF32F0AAEC0AF0DE6A13EC69
:1014500048F0BBEC70F01CEE01F04AEC02F004CC5A
:1014600022F003CC21F002CC20F001CC1FF02A6A3C
:10147000296A286A640E276E8BEC01F022C004FCF6
:1014800021C003FC20C002FC1FC001FCD8960C0147
:1014900004BFD8860001D8B669EF8AF00C01045366
:1014A0000AE1035108E1E80E015D030E0259000153
:1014B000D8A069EF8AF00C01046B036B030E026F76
:1014C000E70E016F170E0E6F340E0D6F000188EFDF
:1014D0008AF003EE1EF0D89001012335E926000EB4
:1014E000EA22EECF0BF0EFCF0CF00BC0DEFF0CC00A
:1014F000DEFF01CCDEFF02CCDEFF03CCDEFF04CC3E
:10150000DEFF000129EC17F01CEE0DF05BEC02F0A1
:101510000ECC20F00DCC1FF0246A3C0E236EEBECB9
:1015200001F00C010F6F206A0FCC1FF0010E75EC5B
:1015300001F0106F206A0FCC1FF0000E75EC01F067
:10154000116F0ECC20F00DCC1FF0246A3C0E236EE0
:10155000EBEC01F027C00FFC206A0FCC1FF0010E4E
:1015600075EC01F0126F206A0FCC1FF0000E75ECC5
:1015700001F0136F076B096B0A6B0B6B04CC22F045
:1015800003CC21F002CC20F001CC1FF0020E7FEC46
:1015900001F0076F04CC22F003CC21F002CC20F044
:1015A00001CC1FF0010E7FEC01F0096F04CC22F09A
:1015B00003CC21F002CC20F001CC1FF0000E7FEC18
:1015C00001F00A6F326A07CC31F03250640DF3CF6C
:1015D00032F03150640DF3CF31F0F4503226366AD8
:1015E00009CC35F036500A0DF3CF36F035500A0DE0
:1015F000F3CF35F0F45036263550312636503222AE
:101600000A513124056F000E3220066F05CCDEFF33
:1016100006CCDEFFDE6A010EDE6EDE6A00014CECF7
:101620007BF007CC08FCD8968BA3D886D8B651EFB0
:101630008BF0010139530001D8A42BEF8BF0DE6A47
:10164000DE6A0C0EDE6E820EDE6E0D0EDE6EE4ECD9
:10165000A8F035EF8BF0DE6ADE6A0A0EDE6E820ECF
:10166000DE6E0D0EDE6EE4ECA8F001013B530001CE
:10167000D8A447EF8BF0DE6ADE6A6F0EDE6E820E54
:10168000DE6E090EDE6EE4ECA8F051EF8BF0DE6A40
:10169000DE6A6B0EDE6E820EDE6E090EDE6EE4EC2E
:1016A000A8F0DE6A10CCDEFF11CCDEFF12CCDEFF2C
:1016B00013CCDEFFD2EC82F08B93ADD61200010189
:1016C00039530001D8A471EF8BF0DE6ADE6A0C0E8C
:1016D000DE6E820EDE6E040EDE6EE4ECA8F07BEFB2
:1016E0008BF0DE6ADE6A0A0EDE6E820EDE6E040E9D
:1016F000DE6EE4ECA8F0030E0C01286FE80E276FF5
:10170000010E2A6F2B6B08012E6B0C012C6B010E46
:1017100008012D6F83C02EFC82C02DFC030E0C012E
:10172000316F0B0E08012A6FDC0E296F2AC8D7FF14
:1017300029C8D6FFF2940001F2A4B0EF8BF0820723
:10174000000E835B0B0E08012A6FDC0E296FF294EA
:101750002AC8D7FF29C8D6FF0001846BB1EF8BF0F0
:10176000EAD7F2A4C3EF8BF08207000E835B0B0E67
:1017700008012A6FDC0E296FF2942AC8D7FF29C806
:10178000D6FF0001846BD6CF29F8D7CF2AF8EA0E0E
:1017900008012A5D0001D8A0D9EF8BF0D8A4D8EFBA
:1017A0008BF0610E0801295D0001D8A0D9EF8BF004
:1017B000D8D7F2A4DDEF8BF0D4D783510C01285D8C
:1017C0000001D8A4EBEF8BF082510C01275D0001E2
:1017D000D8B43BEF8CF083C020F082C01FF0246AA5
:1017E0003C0E236EEBEC01F00C01226F206A22CC40
:1017F0001FF0010E75EC01F0236F206A22CC1FF060
:10180000000E75EC01F0246F83C020F082C01FF041
:10181000246A3C0E236EEBEC01F027C022FC206A08
:1018200022CC1FF0010E75EC01F0256F206A22CC4E
:101830001FF0000E75EC01F0266F010EDE6E23CC5A
:10184000DEFF24CCDEFF25CCDEFF26CCDEFF000150
:10185000D2EC82F083518211D8A435EF8CF00801CC
:101860002E6B276B0001CFEF87F083C028FC82C06E
:1018700027FCFCEF8CF0EA0E08012A5D0001D8A0DD
:101880004DEF8CF0D8A44CEF8CF0610E0801295D6F
:101890000001D8A04DEF8CF064D7F2A451EF8CF08A
:1018A00060D79C0E08012A5D400ED8B4295D000166
:1018B000D8B0FCEF8CF0010EDE6EFCEC8EF098538D
:1018C000D8A468EF8CF008012D6B0001FCEF8CF0C0
:1018D000010E985DD8A485EF8CF008012E5300010D
:1018E000D8A483EF8CF0010E08012D6F0001DDEC10
:1018F000CEF00801276B010E246EF40E55EC01F0BA
:101900000001B8EF32F0FCEF8CF0020E985DD8A425
:10191000ACEF8CF008012E530001D8A4A9EF8CF095
:1019200083C020F082C01FF0246A0A0E236EEBEC05
:1019300001F0826F20C083F083510A0DF3CF83F052
:1019400082510A0DF3CF82F0F4508327020E080172
:101950002D6F0001FCEF8CF0030E985DD8A4CCEF46
:101960008CF008012E530001D8A4C9EF8CF0020EB0
:1019700008012D5D0001D8A4C6EF8CF0030E836F23
:10198000840E826F010EDE6E1DEC84F0030E0801E2
:101990002D6F0001FCEF8CF0040E985DD8A4D9EFF8
:1019A0008CF00C012B69040E08012D6F0001FCEF77
:1019B0008CF0050E985DD8A4FCEF8CF00C012B295F
:1019C0000001D8A4F6EF8CF008012E290001D8A45C
:1019D000F1EF8CF008012E6B0C012B6B0001F5EF81
:1019E0008CF008012E690C012B6B0001050E08011B
:1019F0002D6F0001FCEF8CF00C012B290001D8A405
:101A00000BEF8DF00C012C2B00010AEF8DF00C0177
:101A10002B6B2C6B000108012D530001D8B417EF7C
:101A20008DF083C02EFC82C02DFC31EF8DF08251F1
:101A30000C012D5D2F6F000183510C012E59306F69
:101A400030530001D8A42CEF8DF0100E0C012F5D47
:101A50000001D8A030EF8DF00C012B6B08012E692E
:101A600000010C012B290001D8A454EF8DF00C01CA
:101A700031530001D8B452EF8DF0DE6A010EDE6EF4
:101A8000750EDE6E820EDE6E060EDE6EE4ECA8F0E3
:101A9000DE6ADE6A730EDE6E840EDE6E060EDE6EAB
:101AA000E4ECA8F00C01316B000108012E29010EB5
:101AB000D8A4000E3B6E010E0C012B53D8A4000ECF
:101AC0003B140001D8B484EF8DF0010E0C01315DA0
:101AD0000001D8B481EF8DF0DE6A010EDE6E730E68
:101AE000DE6E840EDE6E060EDE6EE4ECA8F0DE6ABC
:101AF000DE6A750EDE6E820EDE6E060EDE6EE4ECC3
:101B0000A8F0010E0C01316F0001010E08012E53E7
:101B1000D8A4000E3B6E010E0C012B53D8A4000E6E
:101B20003B140001D8B4B5EF8DF0020E0C01315D0D
:101B30000001D8A4B2EF8DF0DE6A010EDE6E730EE6
:101B4000DE6E840EDE6E060EDE6EE4ECA8F0DE6A5B
:101B5000010EDE6E750EDE6E820EDE6E060EDE6E1F
:101B6000E4ECA8F0020E0C01316F00018453D8A4FC
:101B7000BCEF8DF00C012A6B00010C012A5300010F
:101B8000D8A4F8EF8EF0D6CF29F8D7CF2AF82AC8F4
:101B900020F029C81FF0610E246EA80E04EC00F09E
:101BA0003B6E010E8453D8A4000E3B10D8B4F8EF5E
:101BB0008EF0010E845DD8A4E1EF8DF0010E0C01D2
:101BC0002A6F0001AAEC0AF0DE6A13EC48F0BBECC5
:101BD00070F01CEE16F04AEC02F0D8960C0119BF1A
:101BE000D8860001D8B60AEF8EF03D0E0C01165DC6
:101BF000860E1759010E1859000E19590001D8A068
